:100000000C94E4140D9468110D943D110D9412118B
:100010000D94E7100D94BC100D9491100D94661082
:100020000D943B100C9415150C9415150C94151586
:100030000C9415150C9415150C9415150C9477CD7E
:100040000C9415150C9415150C9415150C94151588
:100050000C9415150C9415150C9415150D94A60EED
:100060000C9415150C9407B90C94DDB80C94151567
:100070000C9415150C9415150C9415150C94151558
:100080000C9415150C9415150C9415150C94151548
:100090000C94D7BA0C944DBA0C948FBA0C941ACF16
:1000A0000C9415150C9415150C9415150C94151528
:1000B0000C9415150C9415150C9415150C94151518
:1000C0000C9415150C9415150C9415150C94B3B8C7
:1000D0000C9489B80C9415150C945FB80C9435B831
:1000E0000C94151507634236B79BD8A71A39685682
:1000F00018AEBAAB558C1D3CB7CC5763BD6DEDFD4A
:10010000753EF6177231BF000000803F0800000006
:10011000BE922449123EABAAAA2ABECDCCCC4C3EFC
:1001200000000080BEABAAAAAA3E00000000BF00EB
:100130000000803F0000000000084178D3BB4387E7
:10014000D1133D190E3CC3BD4282AD2B3E68EC82FB
:1001500076BED98FE1A93E4C80EFFFBE01C4FF7F80
:100160003F00000000000C94B1690C94A3E70C94CC
:1001700075A80C94B05A0C9458150C9476AB0C944A
:10018000C5CC0C94FA630C9407AA0C9421FA0C9435
:100190003F290C94F8790C94E0280C947AFD0C9487
:1001A0008F770C94CA810C948D6C0C94CD1E0C949A
:1001B0001EA10D9472020D94E4020C94A73A0C94C3
:1001C000D01E0C94594E0D94FC270D94BA010C943A
:1001D000656B0C9455A80D94A5020C94D4150C9441
:1001E00083280C94827F0D9487010C943BBD0C9462
:1001F000C4AA0C945DC50D94AD020C944F210C94CF
:10020000EDA50C94DB590C9439220D94CC010C947F
:10021000DB3A0C94DBD50C94BCA70C940FC50D9461
:100220001A0A0C942D6C0D9489020C94F2630C94B0
:10023000F11C0C9410A10C9428FA0C947BE00C9403
:1002400036C40C94A52B0D94C7010C9432AA0C94BF
:1002500048AA0C94733B0C94AE2B0C94A6750C948A
:1002600092190C94E51D0C94D2BD0C94C2AB0C9465
:10027000E4150C945FAB0C946DB70C9446700C9421
:1002800028BF0C945E1F0C94B3E80C94474C0C945C
:10029000DEAA0C94EB5A0C943B3A0C9437E00C9485
:1002A00059290C9487BD0C9429680C941F6C0C94EC
:1002B000F7AC0D94AC010C943CA90C94F7AE0C94E3
:1002C000B6C50C94FF6A0C94D8150D94C2010C9419
:1002D000FA4B0C9438E40C946CFD0C94B7390C94E4
:1002E00052AA0C94FA150C9415C10C944C1D0C9444
:1002F000D0150C9490D40C94A0220C9487230C94C9
:10030000F5AC0C943D740C94BCE70C94743B0C94C9
:100310009DC80C940C2D0D94470A0C942A1E0C9425
:100320005E3B0C9444210C94FA3B0C949EA20C94DA
:1003300047770C94AD300C947FFA0C942F1D0C94DD
:100340005B4E0C94A6AB0C94854A0D94B0010C94B2
:100350001FA90C9401640C94463A0C94EDC10C94C2
:10036000D5170C9489440C9481B20C94C5AB0D94B0
:10037000B4010C940E210C949B1E0C9468FA0C94FE
:1003800019AD0C94EDA90C9486E80C94661F0C949E
:1003900086310C943B160C9431AD0C94012D0C94C9
:1003A0009A1F0C94B26B0C9410A90C9437640C94A3
:1003B000F1B20C9403AA0C9412E60C94F4710C9410
:1003C00087B60C947D760C94785B0C9491510C94C8
:1003D00039F50C9488730C947AE00D947A020C949D
:1003E0002B640D94BE010C948D1F0C9412210C945F
:1003F00081FD0C94EA640C94581D0C940C210C940F
:1004000036A50C941EAA0C9458C10C94657A0C94D1
:1004100068750C9432160C945B150D9499010C942C
:10042000D5790C94EB280C94D7170C941C3B0C94A6
:10043000523E0C94B3AA0D94EE020C94E16A0D9412
:1004400093020C948EE50C94BE630C941A160C94D3
:1004500010210C9418650C9462290D9491010C9450
:10046000A33B0C94B06B0C94A1AB0C94AA300C94ED
:100470006F590D94C8010C94BE9B0C944F280C949A
:100480005D1E0C94E5E00C94FD210C945E210C940F
:10049000EDAC0C94CD6B0C94A5590C94397A0C945A
:1004A0005E150C943D180C94362F0C94EC640C944F
:1004B00051CC0C94F3A30C946D1F0C946EAF0C9460
:1004C0001A210C940D9A0C94F3AC0C94EA480C94F9
:1004D000889F0C94B8AB0C94181D0C9417C20C9404
:1004E0008BA70C94853A0D94A6010C94F4A50C945A
:1004F0000C640C94A7A90C94426B0C940D230C94DF
:10050000E9E50C9424BD0D949D020D944A0A0C94C7
:10051000AE760C94ABA20C942AB60C94156C0C9489
:1005200055150C94051D0C9442700C94837F0C940B
:10053000EBAC0C9459D60C945F4E0C946BA90C94B4
:10054000F13A0C9498A20C94B73A0C945A1C0C945F
:10055000D25A0C94F1AC0D94B7020C94ACAD0C943F
:10056000A82B0C9424E60C9454AA0C9472280D9495
:100570008D010C9460430C94873A0C94D7B60C947C
:10058000285A0D941B0A0C94A9AB0C94BDAD0D9484
:100590009C010C94123B0C94744C0C943B1D0C94D9
:1005A000CB280C949A6B0C94182C0C94072D0C945B
:1005B000D7AA0C94BB930C9480AB0C94AE6B0C94A8
:1005C000257A0C94DFEE0C947E5B0C9449790C94A4
:1005D000633B0C9473180C94ED630C94659B0C9422
:1005E000E0150C9452160C94B4AA0C94C6180C94F2
:1005F0001BBD0C9445A70C947EEB0D947F020C94CC
:100600004E7A0C948FFD0C94D2D30C9473FD0C9401
:1006100058370C94E1A90C94772A0C9459810C94C6
:1006200080C50C94FE2C0D9495010C949A390C9471
:10063000776C0C94E4B60C9488510C94246B0C9455
:10064000A31F0C94EFAC0D9402030C94523B0C943A
:100650003AFA0C9471B50C940ABD0C941A690C9476
:100660005DA90C946E5A0C9408670C94A7180C940E
:10067000443B0C94DE4C0C9403E60C94F4590C941B
:100680006C9B0C94DEE70C94561E0C9415CC0C94C9
:10069000896B0C94F5630C94EBA10C94A3230C943C
:1006A0005C3A0C944F1F0C9424160C94EA8D0C9415
:1006B0008E430C947B5B0C94D0640C943E1D0C9484
:1006C00044E70D94F8020C9451A30C94DC150C949F
:1006D000363B0D94C1020C94686C0C949DFD0C94F7
:1006E0007BAB0C944B220C94461F0C94B9280D94B0
:1006F000DA020C94CC630C9408210C9417AA0C9485
:10070000CD390C9499BD0C9414210C9459AC0C94D3
:10071000D8A10C944B4B0C94205B0C9417F90C94BF
:1007200065210C9428A30C94941F0C9421220C9402
:1007300077E00C94C74C0C947D490C94837A0D940B
:100740000C030C9490B60C94F9AC0C946C230C94A0
:1007500039210C9451AB0C94CCA20C9412B30C9490
:1007600014440D94E7270C94E8AE0C9406E00C9426
:1007700068160C94014A0C949AA70C9449FA0C94AC
:10078000555A0C9410C90C944A700C947F390D94EE
:10079000A2010C949F5B0C94B21F0C9459E80C942A
:1007A00032C40C94B5AB0C94D9170C9417150C9457
:1007B00008A80C94D44B0C94E9160C947A800C94F1
:1007C000F4B30C9464280C9456440C94F0640C9488
:1007D000DA3B0C940A210C94B4390C9429AA0C9499
:1007E000E8C50C94789B0C94B5AA0C94BDAB0C9402
:1007F0007CE00C9495A90C9457760D94CB020C9444
:1008000076E00C94971C0C9497510C94AEA70C9422
:1008100016210C9428C50C94B44B0C94996A0C9432
:100820008C920C9454B20C940D7A0C949EC40C943B
:10083000E2A30C94FDC00C94AEA90C944FB50C949B
:10084000806F0C9496FD0C94817F0C94491D0C9440
:10085000783A0C9438160C94E8150C94042D0C94EA
:1008600092D50C94DDA90C94ED4A0C94B1200C9413
:1008700031AA0C94EE640C941FAF0C941D230C94BD
:10088000A03B0C9418210C9438F50C9443A30C94C1
:1008900036160C9411650C946A760C94CEC10C94A7
:1008A00047630C940BAB0C94112C0C94AA6B0C9416
:1008B00040A54E414E494E495459494E46CDCCCCA7
:1008C0003D0AD7233C17B7D13877CC2B329595E624
:1008D000241FB14F0A000020410000C84200401C04
:1008E0004620BCBE4CCA1B0E5AAEC59D74636469DB
:1008F0006E6F70737578585B00556E6B6E6F776EA8
:10090000207375666669782000556E6B6E6F776E22
:1009100020636D642000636C724374723A2000455A
:100920004F46002F00496E3A20003D00494E3A00E4
:100930003D004C454741435920494E3A002500C2ED
:10094000B04320483D00204448543232207479702E
:10095000652E20543D00494E3A00204E6F20656DB3
:1009600069742064617461210020436F756E746541
:100970007220747970652E2076616C3D00494E3A84
:100980000020436F756E74657220747970652E2037
:10099000494E434F525245435420496E746572721A
:1009A000757074206E756D62657221212100495247
:1009B000513A002D3E00200023002D3E0020005023
:1009C000656E6465643A2023007261770076616C1D
:1009D0000074656D70007361740068756500666110
:1009E0006E0052474200485356006D6F64650053D5
:1009F0006574436D643A0053746F726564204558A2
:100A0000543A00737566666978436F64653A0020EE
:100A1000666F7220286D73293A004354524C3A2075
:100A20005363686564756C6520636D642000206D98
:100A300073203A0041726D656420666F7220002059
:100A400044697361726D656400584F4E0048414CB3
:100A500054002074696D653A004354524C3A205258
:100A600065733A002054533A0020543A003D005038
:100A7000696E3A004354524C3A20436F6D6D616E7B
:100A80006420626C6F636B656420627920647269B4
:100A9000766572206F72206368616E6E656C206689
:100AA000726F7A656E004354524C3A204F4E3A4171
:100AB0006C7265616479204163746976650A0043EC
:100AC00054524C3A2048414C543A416C726561642E
:100AD0007920496E6163746976650A004354524C0B
:100AE0003A20584F4E3A2044697361626C65640A3B
:100AF000004354524C3A20584F4E3A416C72656153
:100B00006479204163746976650A004354524C3A13
:100B100020584F464620736B69707065642E2050D4
:100B200072657620636D643A004354524C3A205407
:100B300075726E6564206F66662066726F6D3A002E
:100B40004354524C3A20526573746F726564206648
:100B5000726F6D3A004354524C3A2049676E6F727F
:100B600065642C206368616E6E656C20636D643D06
:100B70000020457865633A004354524C3A20416363
:100B8000746976653A004354524C3A2048414C54BB
:100B90003A416C726561647920496E61637469766B
:100BA000650A004354524C3A20584F4E3A2044694B
:100BB0007361626C65640A004354524C3A20584F8A
:100BC0004E3A416C7265616479204163746976655F
:100BD0000A004354524C3A20584F464620736B69E2
:100BE000707065642E205072657620636D643A00E3
:100BF0004354524C3A205475726E6564206F666699
:100C00002066726F6D3A004354524C3A205265731D
:100C1000746F7265642066726F6D3A004354524C73
:100C20003A204E6F7420656E6F756768206D656D34
:100C30006F727920666F722067726F7570206F70A7
:100C400065726174696F6E004354524C3A20556E60
:100C50006B6E6F776E2073756666697800536B698B
:100C60007070656420686F6D696520737475666661
:100C7000002000205375623D00204974656D3D00E1
:100C80004354524C3A2052414D3D004354524C3A49
:100C9000204F75744F664D656D6F72793A2000284C
:100CA0002D292000282B2920002076616C756520D5
:100CB0006973200020756E6B6E6F776E0A005D3D64
:100CC000005B0020696E76616C6964002000206F13
:100CD0006B003A00206661696C6564003A005265F9
:100CE000747279696E67206D6F6462757320434D0D
:100CF000440A004D6F6462757320706F6C6C696E8E
:100D000067206572726F723D002056616C3A200058
:100D10004D423A20004E6F7420737570706F72747C
:100D200065642072656720747970650A00496C6C8F
:100D30006567616C20617267756D656E74730A001A
:100D40004D6F6462757320706F6C6C696E6720659F
:100D500072726F723D002D002050492056616C2048
:100D60003A004D6F6462757320706F6C6C696E67CA
:100D7000206572726F723D002D0020464D20566135
:100D80006C203A004354524C2F706F6C6C3A204FD9
:100D900075744F664D656D6F72793A2000207365EA
:100DA000632072656D61696E696E6700537461746A
:100DB00075732064656666657265640A002D3E0081
:100DC0005075623A20006374726C00454E41424C8B
:100DD0004500465245455A450044495341424C4519
:100DE000002D3E005075623A2000636D640046415C
:100DF0004E5F4F4E4C590044525900434F4F4C00E8
:100E000048454154004155544F002D3E00507562F5
:100E10003A20007365740064656C002D3E005075C7
:100E2000623A20002D3E005075623A2000556E6BEC
:100E30006E6F776E20636D64200A004F4646004F48
:100E40004E004D6F64627573206F70206661696C2F
:100E500065643A004D42206F6B003D00564323000D
:100E600020636D643D003D0056435F6865617423F7
:100E7000004E6F7420737570706F727465642072A9
:100E8000656720747970650A002056616C3A307885
:100E90000020543A00205265673A3078004164647B
:100EA000723A0020002D3E00436F6E7665727469C1
:100EB0006E6720002D3E0057726F6E67204173737E
:100EC00069676E6D656E742000524742783A200063
:100ED00020764C6576656C3A0020436F6E76563A04
:100EE0000020436F6E76533A0020486F743A0043F7
:100EF0006F6C643A0020436F6E766572746564208F
:100F0000563A00436F6E76657274656420533A00FA
:100F10002D3E0057726F6E672041737369676E6D67
:100F2000656E7420002D3E0057726F6E672041730E
:100F30007369676E6D656E74200053617665643AFF
:100F4000000000000000000000004F4E0000000004
:100F50000000004F46460000000000005245535478
:100F60000000000000544F47474C45000000484136
:100F70004C540000000000584F4E000000000000DC
:100F8000584F46460000000000494E435245415329
:100F90004500444543524541534500454E41424C6E
:100FA0004500000044495341424C450000554E461F
:100FB0005245455A4500465245455A4500000041B4
:100FC00055544F000000000046414E5F4F4E4C59B3
:100FD000004849474800000000004D454449554D30
:100FE0000000004C4F5700000000000048454154ED
:100FF0000000000000434F4F4C000000000044522E
:101000005900000000000053544F50000000000041
:101010005247420000000000004853560000000004
:10102000000020537566663A002041543A00436F31
:101030006D706C6574652E2052656D6F76652074D9
:101040006F706963200024636F6D6D616E6400537F
:101050006B697070696E672E2E00436C65616E550A
:10106000702072657461696E656420746F70696365
:101070002000220022004F75744F664D656D6F721F
:101080007921005D20003A5B000A005D00456D702B
:1010900074793A205B000A003A004D41433A00550A
:1010A0004450205379736C6F6720696E697469616D
:1010B0006C697A65642E0A005379736C6F672070CF
:1010C0006172616D733A002E6C6F63616C005365E1
:1010D0007276696365207265636F72643A20006D91
:1010E000444E5320726573706F6E64657220737422
:1010F00061727465642E004572726F72207365743C
:1011000074696E67207570204D444E53207265736C
:10111000706F6E6465722100476F742049502061C2
:101120006464726573733A00276970205B69705B51
:101130002C646E735B2C67775B2C7375626E6574C1
:101140005D5D5D5D27202D2073657420737461746F
:1011500069632049500A004661696C656420746FB8
:1011600020636F6E66696775726520457468657285
:101170006E6574207573696E6720444843502E2055
:10118000596F752063616E20736574206970206DDE
:10119000616E75616C6C792100204D41534B3A00B2
:1011A0002047573A0020444E533A004C6F61646523
:1011B000642066726F6D20666C6173682049503AD6
:1011C000000A7573657320444843500A00537461E4
:1011D0007274696E67206C616E00546F6F206D6170
:1011E0006E79204D51545420636F6E6E656374693F
:1011F0006F6E206572726F72732E20526573746108
:101200007274204C414E00207472792061676169CC
:101210006E20696E2035207365636F6E647300669F
:1012200061696C65642C2072633D0041776169746B
:10123000696E6720666F722072657461696E65649D
:1012400020746F7069637300636F6E6E656374659D
:10125000642061732000202E2E2E0020757365728D
:101260003A003A000A417474656D7074696E6720C3
:101270004D51545420636F6E6E656374696F6E20B8
:10128000746F2000646973636F6E6E656374656468
:10129000005573696E67204D51545420706173730B
:1012A000776F72642066726F6D20636F6E66696718
:1012B000002E6C6F63616C006D444E53206E616D47
:1012C0006520757064617465643A200044657669D0
:1012D0006365204E616D653A004174206C656173F1
:1012E0007420646576696365206E616D6520616E4A
:1012F000642062726F6B6572204950206D75737443
:1013000020626520636F6E6669677572656400248C
:101310006E6F646573004F4E2C4F46462C48414C0F
:10132000542C524553542C584F4E2C584F46462C53
:10133000544F47474C450024666F726D61740065D9
:101340006E756D00246461746174797065006873F2
:101350007600636F6C6F7200302D32353500696E28
:10136000746567657200666C6F617400332E302E91
:10137000310024686F6D696500757074696D652C46
:101380006672656568656170003330663762333652
:101390005F323032332D30342D3130004C69676884
:1013A000744875622000246E616D65005265626943
:1013B0006E6420737563636573732E2049502061DA
:1013C0006464726573733A004572726F723A207288
:1013D0006562696E64206661696C0052656E65774E
:1013E000656420737563636573732E2049502061B3
:1013F0006464726573733A004572726F723A207258
:10140000656E65776564206661696C000A4E6F20C1
:101410006C696E6B00526573746F72696E672063DE
:101420006F6E6669672066726F6D20454550524F3A
:101430004D00416363657074696E6720636F6D6D05
:10144000616E64732E2E2E0A004E6F204D5154543F
:1014500020636F6E66696775726564004C6F6164C6
:10146000696E6720636F6E6669672066726F6D20B4
:10147000706F7274616C2064697361626C65642E54
:101480002075736520676574204F4E20746F20654A
:101490006E61626C6500436F6E66696720697320D8
:1014A00076616C696400436F6E74696E7565207750
:1014B0006974682070726576696F75736C79206CD9
:1014C0006F6164656420636F6E666967003E003C0F
:1014D00000543A0043757272656E74204C414E2080
:1014E000636F6E6669672869702C646E732C67770A
:1014F0002C7375626E6574293A000A557365207401
:101500006865736520636F6D6D616E64733A202743
:1015100068656C7027202D20746869732074657865
:10152000740A276D61632064653A61643A62653AC2
:1015300065663A66653A3030272073657420616EBF
:10154000642073746F7265204D41432D6164647231
:1015500065737320696E20454550524F4D0A2769C7
:1015600070205B69705B2C646E735B2C67775B2CFF
:101570007375626E65745D5D5D5D27202D207365FA
:1015800074207374617469632049500A277361760B
:101590006527202D20736176652063757272656EF4
:1015A0007420636F6E66696720696E204E565241E3
:1015B0004D3B204F4E7C4F4646202D20656E61628C
:1015C0006C652F64697361626C65206175746F73FB
:1015D0006176650A2767657427205B636F6E6669AD
:1015E0006720616464725D27202D20676574206325
:1015F0006F6E6669672066726F6D207072652D630D
:101600006F6E666967757265642055524C20616E15
:10161000642073746F726520616464722C204F4E75
:101620007C4F4646202D20656E61626C652F646993
:101630007361626C6520646F776E6C6F6164206F9C
:101640006E20737461727475700A276C6F61642701
:10165000202D206C6F616420636F6E666967206661
:10166000726F6D204E5652414D0A277077642720C5
:101670002D20646566696E6520616E642073746FE9
:101680007265204D5154542070617373776F72648A
:101690000A276F746170776427202D20646566695E
:1016A0006E6520616E642073746F726520485454B7
:1016B00050204150492070617373776F72640A271C
:1016C0006C6F67205B73657269616C5F6C6F676CD0
:1016D0006576656C5D205B7564705F6C6F676C65CB
:1016E00076656C5D27202D20646566696E65206CCB
:1016F0006F67206C6576656C2028302E2E37290A9E
:10170000276B696C6C27202D2074657374207761BA
:10171000746368646F670A27636C65617227202DA4
:1017200020636C65617220454550524F4D0A277207
:1017300065626F6F7427202D207265626F6F742051
:10174000636F6E74726F6C6C657200536F66742099
:101750007265626F6F74696E672E2E2E0052414D56
:101760003D000A5379736C6F6720000A312D776949
:10177000726520000A6D71747420000A6D6F6462D6
:101780007573207632000A6D6F646275732076314E
:1017900020282B29000A696E7075747320000A696D
:1017A00074656D7320000A436F6E666967757265B4
:1017B000643A0020416464723A006465762300094B
:1017C000445332343832206572726F7200095265A8
:1017D00073657420646F6E650009436865636B69A7
:1017E0006E6720666F7220312D57697265206465BF
:1017F00076696365732E2E2E004453323438322DB1
:101800003130302070726573656E74004572726F8E
:101810007220312D7720696E697420233220467240
:1018200065653A0077737461742E20467265653A77
:10183000005465726D2E20467265653A00457272DD
:101840006F7220312D7720696E6974202331004634
:101850007265653A004453323438325F3130305F5C
:101860004932435F544F5F31575F425249444745C5
:1018700020696E697400444D584F75742E2046726D
:1018800065653A00444D58696E204275666665721A
:1018900020616C6C6F632065727200496E69742000
:1018A000696E2063683A003B003D0050696E3A0063
:1018B0003B003D4C4F5700546865726D6F3A004FC6
:1018C0006E6520776972652052656164790A004609
:1018D0007265653A00444D58206F757420737461C9
:1018E000727465642E204368616E6E656C733A2075
:1018F00000444D5820696E20737461727465642EC3
:10190000204368616E6E656C733A004170706C794B
:10191000696E6720636F6E666967004C6F6164650E
:101920006420455441473A004E6F2073746F7265CE
:101930006420636F6E666967004C6F616465642044
:1019400066726F6D20454550524F4D006C6F61645B
:10195000206661696C656400547279696E67204C19
:101960006F61642066726F6D20454550524F4D0087
:101970004C6F6164696E6720436F6E6669672066AD
:10198000726F6D20454550524F4D00436F6E666932
:1019900067206175746F736176653A000A537973D5
:1019A0006C6F67206465627567206C6576656C3A5C
:1019B0000053657269616C206465627567206C65AF
:1019C00076656C3A0053617665640A00536574204D
:1019D00064796E616D69632049500A004545505233
:1019E0004F4D20636C65617265640A004D5154541B
:1019F0002050617373776F726420757064617465D1
:101A0000640A004F54412050617373776F726420F1
:101A1000757064617465640A00636F756C64206E30
:101A20006F742070617273653A2000557064617440
:101A300065640A004E6F20495020616472657373BB
:101A40000052656C656173696E6720736F636B65C7
:101A50007420616E6420726574727900205361761F
:101A60006564004C6F6164696E672048545450206F
:101A7000636F6E666967206F6E2073746172747530
:101A8000703A004F4646004F4E002B002D00455443
:101A900061673A200047657420455441473A200069
:101AA000485454502F312E310025733A2025730DA0
:101AB0000A0020485454502F312E310D0A486F73BC
:101AC000743A2025730D0A4163636570743A202AC5
:101AD0002F2A0D0A436F6E6E656374696F6E3A202C
:101AE000636C6F73650D0A0025730020000D0A00FA
:101AF000474554006661696C656420746F20636FAC
:101B00006E6E6563740A004552524F523A20536517
:101B1000727665722072657475726E65642000431A
:101B20006F6E666967206E6F74206368616E6765AB
:101B3000640A00446F6E652E0A00436F6E66696723
:101B40002070617273696E67206661696C65640AF2
:101B500000676F7420436F6E6669670A006874746B
:101B60007020726574636F6465200066726565201D
:101B700000436F6E666967205552493A2068747455
:101B8000703A2F2F002044656661756C7420636F76
:101B90006E66696720736572766572207573656419
:101BA0003A20006C617A79686F6D652E7275000A53
:101BB000282B294D554C544956454E54000A282B84
:101BC0002950574D5F52454C4159000A282B294D49
:101BD000444E53000A282D2955415254425249443B
:101BE0004745000A282B295359534C4F47000A28D0
:101BF0002B29504944000A282D294D4350323330B7
:101C00003137000A282D294152544E4554000A28E4
:101C10002D294F5441000A282B29535049204C4567
:101C200044000A282B294D4F544F52204354520050
:101C30000A282B294143204841494552206F6E20F4
:101C400053657269616C33000A282B29434353386A
:101C5000313120262048444331303830000A282BC7
:101C600029524553544152545F4C414E5F4F4E5F91
:101C70004D5154545F4552524F5253000A282D295A
:101C80004841524452455345542C207573696E6740
:101C900020736F6674000A282B29434F554E544514
:101CA00052000A282B29444854000A282B2944535F
:101CB000323438322D313030000A282B294F574921
:101CC0005245000A282D2949504D4F444255530092
:101CD0000A282B294D4F4442555320307830362066
:101CE00061742053657269616C322073706565643C
:101CF0003A39363030000A282B29414441465255A2
:101D00004954204C4544000A282B29444D58000AC8
:101D1000282B2957697A6E657435313030000A28CE
:101D20002B294672656552616D207072696E746907
:101D30006E67000A282B295741544348444F4700F7
:101D40006C617A79686F6D652E7275000A436F6EEB
:101D5000666967207365727665723A003230313198
:101D600030334C0020432B2B2076657273696F6EE5
:101D70003A00333066376233365F323032332D30DB
:101D8000342D3130000A4C617A79686F6D652E729E
:101D900075204C6967687448756220636F6E747251
:101DA0006F6C6C65722000204F464600204F4E003D
:101DB0002042595041535300726561647900247385
:101DC0007461746500757074696D6500667265652F
:101DD0006865617000247374617473002054696DC8
:101DE00065723A00204C6F636B733A002000204C00
:101DF0006F636B733A000A52414D3D002045787085
:101E0000697265640A00202D746172676574207AB6
:101E10006F6E652D0020416C61726D204578706990
:101E20007265640A0020636D643A00204375723A5B
:101E300000205365743A00536176656420746F2006
:101E4000454550524F4D00536176696E6720636F70
:101E50006E66696720746F20454550524F4D2E2E97
:101E600000206973200044656C6574696E672063A7
:101E70006F6E662E2052414D207761733A00537485
:101E80006F707065640053746F7070696E67206363
:101E900068616E6E656C73202E2E2E004E6F74205E
:101EA000756E6C6F636B656420696E2031307320D2
:101EB0002D20636F6E74696E7565202E2E2E005571
:101EC0006E6C6F636B696E6720636F6E6669672007
:101ED0002E2E2E0063637338313120697320616CBC
:101EE000726561647920696E697469616C697A658B
:101EF00064006864633130383020697320616C722B
:101F00006561647920696E697469616C697A656478
:101F10000048444331303830206E6F7420696E6958
:101F20007469616C697A6564006363733831313A4E
:101F30002064617461206E6F7420617661696C61E8
:101F4000626C6500636373383131206E6F74206991
:101F50006E697469616C697A656400203C3C00417B
:101F6000433A200041433A2053657269616C207501
:101F7000736564206279204143202D206469736178
:101F8000626C696E672073657269616C206C6F6743
:101F900067696E6720616E6420636D640041433A37
:101FA000204F7574206F66206D656D6F72790041EA
:101FB000433A20496E69743A200041433A2044650F
:101FC0002D496E69743A200045525200445259001E
:101FD00046414E5F4F4E4C59004845415400434FD7
:101FE0004F4C0041433A204F4B00203E3E200041E1
:101FF000433A200041433A20506F6C6C696E670091
:102000004C4F57004D454449554D004849474800FD
:102010004155544F007261770071756569740073A2
:1020200077696E67006C6F636B00556E6B6E6F77D0
:102030006E207375666669782000556E6B6E6F77DB
:102040006E20636D642000436F756E7465723A2074
:1020500000444D582D4F757420496E69743A200024
:10206000444D582D4F75742073746F703A200041A1
:10207000737369676E65643A00444D5820637472E7
:102080006C3A200069313600016933320002753143
:102090003600037533320004693868000569386C0E
:1020A0000006753868000775386C00087831300014
:1020B00009313030000A44656661756C74207365BF
:1020C0007269616C206D6F6465204E3831207573C4
:1020D000656400384531002600384E31000600386E
:1020E0004532002E00384E32000E00384F31003697
:1020F00000384F32003E003745310024003745326A
:10210000002C00374F31003400374F32003C00378D
:102110004E31000400374E32000C004D4255533A08
:10212000204D6F646275732074656D706C617465A9
:10213000206E6F7420666F756E643A20004D4255B4
:10214000533A20496E76616C69642074656D706CD9
:102150006174652E002C002C002C002C004D425583
:10216000533A20636F6E666967206661696C6564C7
:102170003A004D4255533A20636F6E666967206599
:1021800072726F72004D4255533A20636F6E6669EA
:1021900067206C6F6164656420004D4255533A209E
:1021A0004F7574206F66206D656D6F7279004D42BA
:1021B00055533A20506F6C6C696E67206572726F70
:1021C0007220004D425553443A2049676E6F726544
:1021D00064202D20657175616C20776974682073A7
:1021E00065747465642076616C004D4255533A20E5
:1021F0004164642040533A20006E657874726567CC
:10220000206F7574206F662072616E67650052657D
:1022100063757272656E7420736561726368696E4E
:1022200067206E657874726567004D425553443A75
:10223000204D61707065643A003A002066726F6DDF
:1022400020004D425553443A2020676F74200020EF
:1022500076616C3A0020005265733A200020696E66
:102260007465726E616C2073656E64206572726F46
:1022700072202D206E6F207265674F626A002069A0
:102280006E7465726E616C2073656E642065727227
:102290006F72202D206E6F2074656D706C61746597
:1022A0000020696E7465726E616C2073656E6420C7
:1022B0006572726F72202D206E6F2073746F72655D
:1022C000004D425553443A20656E64506F6C6C204B
:1022D000004D425553443A20506F6C6C2000206EE4
:1022E0006F7420666F756E64004D4255533A20201E
:1022F000706172616D20002073656E64206572727A
:102300006F722E20004D4255533A202000416464E4
:102310002040563A20002056616C3A20004D42552C
:1023200053443A207375666669783A00206F7220CC
:1023300073756666697820004D4255533A204E6F9A
:102340002074656D706C61746520666F722000206A
:1023500064656C74613A002D3E002F002056616C5C
:102360003A004D6F746F723A20696E3A004D6F7487
:102370006F723A2074696D656F757400556E6B6E7F
:102380006F776E20636D64004D6F746F723A2046F4
:102390006F7263656420657865637574696F6E003C
:1023A0004D756C746956656E7420636F6E666967EF
:1023B000206661696C6564004D756C746956656E64
:1023C0007420696E6974004D756C746976656E74FD
:1023D0002044652D496E697400204F75743A0020C1
:1023E0006D33002066726F6D2000204D6178207281
:1023F0006571756573743A002066616E253A002038
:1024000061637469766520563A00546F74616C207C
:10241000563A005049443A20616C726561647920F3
:10242000696E697469616C697A6564005049443AFF
:1024300020496E76616C696420706172616D206103
:10244000727261792E002C002C002C002C00504957
:10245000443A20636F6E666967206661696C6564E3
:102460003A005049443A20636F6E666967206C6F8A
:102470006164656420005049443A20636F6E666968
:1024800067206572726F72005049443A204F75742C
:10249000206F66206D656D6F727900203C414C4D58
:1024A0003E0020443A0020493A0020503A0020697A
:1024B0006E3A00207365743A005049443A20005047
:1024C00049443A20496E76616C696420706172619A
:1024D0006D2061727261792E00536574206F75747E
:1024E00020746F20002050494420616C61726D2E71
:1024F00020002050494420616C61726D3A20636C69
:102500006F736564005049443A20556E6B6E6F7767
:102510006E2073756666697820005049443A2055EC
:102520006E6B6E6F776E20636D6420002053657450
:10253000706F696E743A005049443A200020496E29
:102540007075742076616C75653A005049443A2084
:102550000020696E69740050574D2D4F757420230B
:10256000002073746F700050574D2D4F75742023E9
:10257000003D0050696E3A0020696E697400526532
:102580006C61792D4F75742023002073746F700077
:1025900052656C61792D4F75742023003D3E003AE1
:1025A0000070756220616374696F6E200069646CED
:1025B00065006F66660068656174696E67006661D4
:1025C0006E00647279696E6700636F6F6C696E6725
:1025D0000020697320004F75742000556E6B6E6F7C
:1025E000776E207375666669782000556E6B6E6F26
:1025F000776E20636D642000616374696F6E007292
:10260000656C61794374723A200053686F770020DB
:10261000636D643D002D0020416464723A0064657E
:1026200076230020616C69766500204E6F64653A00
:1026300000312D7769726520636F756E743A2000E2
:10264000312D776972652073686F72746564005B01
:10265000305D3A2000202D202D202D20EFBBBF0023
:102660003E003E31202D200020002E00696E0073B8
:102670005F6F7574006D79686F6D65004354524CDF
:102680002F657865633A204F75744F664D656D6FA1
:1026900072793A2000202D3E2000456D69743A2061
:1026A00000202D3E20004974656D436D643A200082
:1026B000202D3E20004974656D3A2000005EBCE28A
:1026C000613FDD83C29C7E20A3FD1F419DC3217F0E
:1026D000FCA2401E5F01E3BD3E6082DC237D9FC102
:1026E000421CFEA0E1BF5D0380DE3C62BEE0025CF6
:1026F000DF81633D7C22C09E1D43A1FF4618FAA4E2
:1027000027799BC584DA3866E5BB5907DB856739CD
:10271000BAE406581947A5FB7826C49A653BD987C1
:10272000045AB8E6A7F91B45C6987A24F8A6441AB5
:1027300099C7257B3A6486D85B05E7B98CD2306EA1
:10274000EDB3510F4E10F2AC2F7193CD114FADF38D
:10275000702ECC92D38D6F31B2EC0E50AFF1134D81
:10276000CE90722C6D33D18F0C52B0EE326C8ED075
:10277000530DEFB1F0AE4C1291CF2D73CA94762861
:10278000ABF517490856B4EA6937D58B5709EBB54D
:1027900036688AD495CB2977F4AA4816E9B7550B41
:1027A00088D6346A2B7597C94A14F6A8742AC89635
:1027B000154BA9F7B6E80A54D7896B35436F6E6E8F
:1027C00065637465642E00436F6E6E2E2061626FC8
:1027D00072746564003E3E2000496E76616C6964E7
:1027E00020636F6D6D616E64000000200023002681
:1027F0000029002C002F0032000001000003010618
:102800000109013E3E3E004E6F204D414320636F63
:102810006E666967757265643A20736574206669CF
:10282000726D776172652773204D41430A004E6FC8
:102830002076616C696420454550524F4D2064619B
:1028400074612E20496E697469616C697A696E677A
:102850002E0000002200250028002B002E00310051
:10286000340002010000050108010B0100000A0B01
:1028700002090C0D0E08070304010000000000000F
:102880000000000000000000000000000000000048
:102890000000000000000000121110000000000005
:1028A0000000000000000000000000000000000028
:1028B000000000002100240027002A002D00300025
:1028C000330001010000040107010A010102102088
:1028D0002008081020401020408002010201080456
:1028E00002010102040810204080804020100804EA
:1028F0000201800402018040201008040201080443
:102900000201010204081020408001020408102086
:1029100040800505050507050808080802020202AF
:102920000A0A08080404040401010101010101016B
:102930000303030303030303040707070C0C0C0C36
:102940000C0C0C0C0202020206060606060606061F
:102950000B0B0B0B0B0B0B0B57726F6E6720706121
:10296000796C6164004354524C2F7478743A204F50
:1029700075744F664D656D6F72793A2000202D3E5B
:102980002041543A004368616E20747970653A00C2
:102990004E6F2073746F7265642076616C75657319
:1029A000202D2064656661756C743A200053617651
:1029B000656420455441473A0053657420455441AD
:1029C000473A2000E300B10311241FBECFEFD1E24C
:1029D000DEBFCDBF00E00CBF1BE0A0E0B2E0E2E450
:1029E000F0E802E00BBF02C007900D92A039B107DA
:1029F000D9F723E1A0E9BBE001C01D92A93AB207D3
:102A0000E1F714E1C3EED4E100E006C0219701092B
:102A1000802FFE010F94E537C23ED10780E0080702
:102A2000A9F70F94212C0D940F400C940000FC0189
:102A3000848195810895DC011696ED91FC91309783
:102A400039F080858F70823019F4868197810895DE
:102A500090E080E00895FC01A481B581109721F1F8
:102A600018969C9118979F708EEF890F823010F006
:102A700091111AC019964D935D936D937C931C9799
:102A8000A481B58118969C911897907F92601896B2
:102A90009C930480F581E02D8085982F907F90365F
:102AA00019F48F70806A8087089581E090E008951E
:102AB00087E090E008958AE090E0089588E090E053
:102AC0000895FC01238130E090E080E0FC01EE0FEE
:102AD000FF1FE853F44FA081B181A217B30761F43F
:102AE000880F991F880F991FFC01EC54F44F408305
:102AF0005183628373830895A081B181AB2B19F454
:102B000020813181EDCF019685309105F9F6089548
:102B1000FC01238130E090E080E0FC01EE0FFF1F1C
:102B2000E853F44F408151814217530761F4880FF5
:102B3000991F880F991FFC01EC54F44F608171813B
:102B400082819381089540815181452B89F431839D
:102B50002083880F991F880F991FFC01EC54F44FB4
:102B6000108211821282138260E070E0CB0108951E
:102B700001968530910589F6F7CF880F991F880F48
:102B8000991FFC01E456F44F80819181A281B381A9
:102B90000196A11DB11D80839183A283B383089503
:102BA00085E090E00C94BD1584E090E00C94BD1598
:102BB00083E090E00C94BD1582E090E00C94BD158C
:102BC00081E090E00C94BD1590E080E00C94BD1580
:102BD000CF93DF93EC01E881F9810484F585E02D42
:102BE000199529893A892F5F3F4F3A8B298BDF91BD
:102BF000CF910895CF93DF93EC018E8581110DC0A5
:102C000081E090E049895A892C853D854217530718
:102C100008F080E0DF91CF910895E881F981048484
:102C2000F585E02DCE0119958F3F910549F780E09C
:102C300090E0F0CFFC01848595856817790708F44A
:102C4000CB01928B818B0895DC011E962C911E97EF
:102C5000222339F0ED91FC910190F081E02D6FEF8E
:102C600019940895FC0187859089089581E008955D
:102C700090E080E00895FC0122813381232B49F00C
:102C8000868197818130910539F01CF00397039775
:102C900030F090E080E0089581E090E0089582E0D7
:102CA00090E008950F931F93CF93DF9300D000D04F
:102CB0001F921F92CDB7DEB781E028960FB6F89429
:102CC000DEBF0FBECDBFDF91CF911F910F91089551
:102CD00090E080E00895DC011296ED91FC91309730
:102CE00071F090859F70923039F0953041F4CF01AA
:102CF0000E9485FA90E0089581E090E0089590E0C8
:102D000080E0089565E0FC01808191810E94F3F9E3
:102D1000009761F0FC018085859585958595859561
:102D2000181624F4082E000C990B089590E080E00A
:102D300008950F931F93CF93DF93FC01C281D3813A
:102D40002097C9F18B0188858F70853021F5CE01E0
:102D50000E9485FA8017110671F16CF1602FCE0187
:102D60000E94F3F9FC01892B31F180858F7082304C
:102D700039F461857285838594850F942B3606C05E
:102D80008330C9F46185728583859485DF91CF9105
:102D90001F910F910895672B71F4823029F4698592
:102DA0007A858B859C85E9CF833029F469857A857E
:102DB0008B859C85EBCF60E070E0CB01E7CF64EAC8
:102DC0007CE0811102C06FE97CE08EE692E10D9417
:102DD0000615DC0155962C915597273781F4ED9116
:102DE000FC91008CF18DE02D19956FE179E08EE674
:102DF00092E10F9406158EE692E10D94BA120895B1
:102E0000CF93DF93009709F490C0FC012081222327
:102E100009F48BC0EC0163E17EE00F942F30892B25
:102E200009F45FC066EC7DE0CE010F942F30892B52
:102E300009F45AC06AEE7DE0CE010F942F30892B41
:102E400009F455C06AEE79E0CE010F942F30892B3A
:102E500009F450C066EE79E0CE010F942F30892B33
:102E600009F44BC062EE79E0CE010F942F30892B2C
:102E700009F446C06EED79E0CE010F942F30892B16
:102E800009F441C06AED79E0CE010F942F30892B0F
:102E9000E9F166ED79E0CE010F942F30892BC9F16D
:102EA00061ED79E0CE010F942F30892BA9F16DEC03
:102EB00079E0CE010F942F30892B89F167E17EE014
:102EC000CE010F942F30892B69F169EC79E0CE01A6
:102ED0000F942F30892B49F58DE090E0DF91CF9151
:102EE000089582E090E0FACF89E090E0F7CF81E0AA
:102EF00090E0F4CF88E090E0F1CF85E090E0EECF75
:102F000086E090E0EBCF87E090E0E8CF8AE090E0C9
:102F1000E5CF8BE090E0E2CF8CE090E0DFCF83E084
:102F200090E0DCCF84E090E0D9CF90E080E0D6CF95
:102F3000CF92DF92EF92FF920F931F93CF93DF9385
:102F4000CDB7DEB7C154D1090FB6F894DEBF0FBEBE
:102F5000CDBF6C01AB0130E020E060E4CE01019612
:102F60007C010E942DD9F70101900020E9F73197EB
:102F70008F010E191F09A801B701C6010F94723CF9
:102F8000892B11F010E000E0C801CF5BDF4F0FB6D6
:102F9000F894DEBF0FBECDBFDF91CF911F910F918F
:102FA000FF90EF90DF90CF9008950D94922E0D94A6
:102FB000922ECF92DF92EF92FF920F931F93CF93B7
:102FC000DF93CDB7DEB7C054D1090FB6F894DEBF9A
:102FD0000FBECDBF8091F70D9091F80D059709F4C4
:102FE00049C06115710509F445C069017A018B0179
:102FF00040E450E0CE0101960F94803C6FE270E017
:10300000CE0101960F94473C892B41F4980143E08F
:1030100050E060E4CE0101960E942DD94FE350E0CC
:10302000B601CE0101960F94623C0E945FF988239D
:1030300009F18091F70D9091F80D0697D9F48091E0
:10304000870C811117C0B701CE0101960F9451076B
:1030500081E090E0C05CDF4F0FB6F894DEBF0FBE9A
:10306000CDBFDF91CF911F910F91FF90EF90DF9037
:10307000CF90089590E080E0EDCFCF92DF92EF9275
:10308000FF920F931F93CF93DF93CDB7DEB7609777
:103090000FB6F894DEBF0FBECDBF7C016B01CA0135
:1030A000B9012AE0AE014F5F5F4F0F94D330D701D3
:1030B000ED91FC910288F389E02D9801AE014F5FFC
:1030C0005F4FB601C701199560960FB6F894DEBF41
:1030D0000FBECDBFDF91CF911F910F91FF90EF9069
:1030E000DF90CF900895CF92DF92EF92FF920F93EF
:1030F0001F93CF93DF93CDB7DEB760970FB6F894E9
:10310000DEBF0FBECDBF7C016B01BA01A901CE01AC
:1031100001960E9455DAD701ED91FC910288F3895E
:10312000E02D9801AE014F5F5F4FB601C7011995C1
:1031300060960FB6F894DEBF0FBECDBFDF91CF9182
:103140001F910F91FF90EF90DF90CF9008951F9304
:10315000CF93DF93FC01162FC389D489818992898B
:103160009C012F5F3F4F328B218BC80FD91FCE019F
:103170000F944837181721F0612FCE010F94503764
:1031800081E090E0DF91CF911F910895FC0181894A
:103190009289248535858217930740F423893489E1
:1031A000820F931F0F94483790E008958FEF9FEFA1
:1031B00008958F929F92AF92BF92CF92DF92EF923B
:1031C000FF920F931F93CF93DF93E091F90DF0914E
:1031D000FA0D309709F467C0812EF02E932EC22E7F
:1031E000A52ED42EB72EE62EBC01CF010E9441F9A8
:1031F000EC01892B19F481E090E057C088858F702D
:103200008530C9F760E0CE010E94F3F98C0161E0DE
:10321000CE010E94F3F9FC01C185D285D80119962F
:103220002D913C912130310561F13CF46F2DCE019F
:10323000232B09F70E9460CEDECF2230310531F119
:1032400027303105C1F6892BB1F280858F7085302A
:1032500091F6C681D781209771F288858F7084306E
:1032600061F40F2D182D2C2D392D4D2D5A2D6E2D2D
:103270007B2D89859A850E94D9180A80DB81C02D13
:10328000EACF6F2DCE0103960E9460CE6E2DCE0147
:103290000E9460CE6D2DCE0101960E9460CE6C2DF5
:1032A000CE010296C7CF90E080E0DF91CF911F91D1
:1032B0000F91FF90EF90DF90CF90BF90AF909F90D5
:1032C0008F900895CF92DF92EF92FF920F931F930A
:1032D000CF93DF93E091D60BF091D70B3097C9F0E5
:1032E00090859F709530A9F469017A01EB01682FF0
:1032F000CF010E94F3F9FC0190859F70943049F44E
:1033000081859285009729F09601A701BE010E9450
:10331000D918DF91CF911F910F91FF90EF90DF901F
:10332000CF9008958F929F92AF92BF92CF92DF92EB
:10333000EF92FF920F931F93CF93DF938091D40B63
:103340009091D50B892B09F48BC021E030E0D0E0BF
:10335000C0E0CC24C394D12C46010C2E02C0880CB2
:10336000991C0A94E2F7092C000CAA08BB08790101
:1033700084E0E80EF11CC90150E040E060912E02AB
:1033800070912F02FC016817790720F4E0912E025A
:10339000F0912F0260919A0C70919B0CE60FF71F31
:1033A000A081E091D40BF091D50BBC016150710963
:1033B000E60FF71F60816A17F1F06091910B709131
:1033C000920B63307105B4F04091970B5091980BBC
:1033D0006091990B70919A0B482959296A297B2988
:1033E0004093970B5093980B6093990B70939A0BA3
:1033F000A08351E041E00196E816F90609F0BECF3E
:103400004423D9F18091910B9091920B0196909366
:10341000920B8093910B5523E9F0E091D40BF0913E
:10342000D50BE20FF31F028110E0218130E04081D3
:1034300050E03197608170E0CE010E94621980E017
:103440000E94B4D36093930B7093940B8093950B6D
:103450009093960B21969701C430D10509F07CCF4B
:10346000DF91CF911F910F91FF90EF90DF90CF9060
:10347000BF90AF909F908F9008951092920B1092F2
:10348000910BC9CF009789F0FC0120852F70253062
:1034900061F40E94F3F9009741F0FC0120852F7040
:1034A000243019F481859285089590E080E0089594
:1034B000CF92DF92EF92FF920F931F93CF93DF9300
:1034C00000D000D0CDB7DEB78091820C81119CC0B6
:1034D0008091F70D9091F80D02970CF495C08091B2
:1034E000DA0B9091DB0B009709F48EC061EE75E06A
:1034F0000E9441F98C01009709F486C00E9485FA68
:10350000E82EF12CE114F10409F47EC070E060E0D3
:10351000C8010E94421A6C01EA94EF2809F483C0A2
:1035200061E0C8010E94F3F9FC0101851285CE011A
:1035300001960E948EFFCE0101960E94ACFF68EBBF
:1035400070E18DEB91E10F940615B6018DEB91E1E1
:103550000F9410146BE07AE08DEB91E10F9410144E
:103560004AE050E0B8018DEB91E10F94F7136BE066
:103570007AE08DEB91E10F9410146EE07EE08DEB1C
:1035800091E10F9410148DEB91E10F94BA1262E067
:1035900072E08CE892E10E9428C5D0928212C0921B
:1035A000811210938412009383128EE09EE0892B87
:1035B000E9F58FED95E090938612809385128091C6
:1035C000D80B9091D90B009741F070E060E00E9419
:1035D000421A9093840C8093830C8091830C909179
:1035E000840C009731F19093881280938712109287
:1035F0008A121092891281E08093820C6FE970E147
:103600008DEB91E10F94061526960FB6F894DEBF68
:103610000FBECDBFDF91CF911F910F91FF90EF9023
:10362000DF90CF90089502E012E081CF8EE09EE01F
:10363000C2CF81E994E0892B19F48FED95E0D3CFC7
:1036400081E994E0D0CFCF93DF9300D000D01F92D8
:103650001F92CDB7DEB7FC01862F8F706181607F2E
:10366000682B618388E0DE01119601900D928A95A6
:10367000E1F729813A814B815C816D817E818F8167
:10368000988528960FB6F894DEBF0FBECDBFDF91A8
:10369000CF910895CF93DF9300D000D01F921F9257
:1036A000CDB7DEB7FC01608398E0DE011196019092
:1036B0000D929A95E1F729813A814B815C816D8168
:1036C0007E818F81988528960FB6F894DEBF0FBE55
:1036D000CDBFDF91CF9108956F927F928F929F928D
:1036E000AF92BF92CF92DF92EF92FF920F931F9310
:1036F000CF93DF93CDB7DEB7A0970FB6F894DEBFB8
:103700000FBECDBF8C01862E7A01DC018D919C917C
:103710001197892B09F466C01496ED91FC913097AE
:1037200009F460C080818071BFEF6B135DC0B1F49C
:1037300081E0A0960FB6F894DEBF0FBECDBFDF913B
:10374000CF911F910F91FF90EF90DF90CF90BF909E
:10375000AF909F908F907F906F9008954330510568
:1037600039F3818082942FE082226FEB79E08EE63C
:1037700092E10F9406154AE050E0D80113966C913F
:103780008EE692E10F94D0126DEB79E08EE692E135
:103790000F940615D8011496ED91FC9161816F701C
:1037A0004AE050E08EE692E10F94D0126AEB79E0A5
:1037B0008EE692E10F9406154AE050E0682D8EE601
:1037C00092E10F94D0128EE692E10F94BA12D801D2
:1037D0001496ED91FC9181818F70881207C08081D1
:1037E0008F7E808380E0A5CF8111FCCF198E1A8E49
:1037F0001B8E1C8E1D8E1E8E1F8E18A28A8D8F70A2
:103800008A8FD8011496ED91FC9181818F70881573
:10381000A9F1B3E0EB16F10489F168EB79E08EE6EB
:1038200092E10F9406154AE050E0F80163818EE6BC
:1038300092E10F94D01266EB79E08EE692E10F945C
:103840000615D8011496ED91FC9161816F704AE0E4
:1038500050E08EE692E10F94D01263EB79E08EE6B1
:1038600092E10F9406154AE050E0682D8EE692E151
:103870000F94D0128EE692E10F94BA12F8012081D3
:103880003181FCE0F81508F416C1E82DF0E0882736
:10389000E35BF34E8F4F0D94E5375A1C971C181DB0
:1038A0002F1D3B1D181DF11C181D3E1D491D051D1A
:1038B0004C1D581DD8011496CD90DC90F6018181E5
:1038C0008F70853009F4F7C050F48230C1F066EF94
:1038D00075E0C9010E9441F93C01912C4BC0873031
:1038E000D1F08A30A1F76FEE75E0C9010E9441F96D
:1038F0003C01D6019C9092FA992490F83BC069EE65
:1039000075E0C9010E9441F93C01D6019C9090FAF2
:10391000992490F82FC068EE75E0C9010E9441F922
:103920003C01F601908091FA992490F823C06BEF46
:1039300075E0C9010E9441F93C01D8011496ED914E
:10394000FC91808180FB992490F8982F9E7F80FFC6
:10395000916090836114710469F461E0CE0149962D
:103960000E944A1B298B3A8B4B8B5C8B6D8B7E8B19
:103970008F8B988FF801A080B18061E376E0C5015C
:103980000E9441F96C0166E376E0C5010E9441F9AD
:103990005C01892B81F4C114D10469F460E0CE018B
:1039A00049960E944A1B29833A834B835C836D832B
:1039B0007E838F839887D8011496ED91FC916114D2
:1039C000710409F07CC0898D811179C0B82DBF7058
:1039D0008B2E8181807F882A818280818F7E808367
:1039E000A7CE60E076E0C9010E9441F93C01D80110
:1039F0001496ED91FC91808181FB992490F8982F89
:103A00009D7F81FF92609083B5CF66E076E0C9012B
:103A10000E9441F93C01D8011496ED91FC918081FE
:103A200082FB992490F8982F9B7F82FF9460EBCFC4
:103A300066EF75E0C9010E9441F93C01892B09F04C
:103A40004CCF62E0CE0149960E944A1B29873A87F3
:103A50004B875C876D877E878F87988B3ECF6CE026
:103A600076E0C9010E9441F93C01D8011496ED911C
:103A7000FC9190804CCF61E176E0F3CF67E176E096
:103A8000C9010E9441F93C01D8011496ED91FC91C5
:103A900049CF6DE176E0F4CF64E276E0C9010E949F
:103AA00041F93C01D8011496ED91FC91908023CF0F
:103AB0006AE276E0F3CF912C712C612C5BCF83E02E
:103AC000E816F104B9F0982D9F70892E8181807FCE
:103AD000882A818280818F7E8083E98CFA8C0B8D8D
:103AE0001C8D2D8D3E8D4F8D58A1692DC3010E94D7
:103AF00028E11ECE81818F70881509F419CE829439
:103B000090EF8922882A81828081806168CFCF935B
:103B1000DF9300D000D01F921F92CDB7DEB7FC011B
:103B200091819F70906B91834483558366837783E3
:103B300088E0DE01119601900D928A95E1F72981C6
:103B40003A814B815C816D817E818F819885289639
:103B50000FB6F894DEBF0FBECDBFDF91CF910895B1
:103B6000CF93DF9300D000D01F921F92CDB7DEB766
:103B7000FC016F3F710519F014F06FEF70E077FDF5
:103B800060E09181892F82958F7081508230C8F4D6
:103B9000648388E0DE01119601900D928A95E1F729
:103BA00029813A814B815C816D817E818F819885ED
:103BB00028960FB6F894DEBF0FBECDBFDF91CF9130
:103BC00008959F7090619183E3CFCF93DF93CDB73A
:103BD000DEB760970FB6F894DEBF0FBECDBF198277
:103BE0001A821B821C821D821E821F8218868A8175
:103BF0008F708A836FEF70E0CE0101960E94B01D36
:103C000060960FB6F894DEBF0FBECDBFDF91CF91A7
:103C10000895CF92DF92EF92FF92DC01362F11963A
:103C2000EC911197E295EF70EC3008F0B6C0F0E03F
:103C30008827E25EF14E8F4F0D94E537D01E561E59
:103C4000561ECD1ECD1ECD1E9B1E5D1ECD1ECD1E35
:103C50002A1E2A1E14968D919D910D90BC91A02D27
:103C6000662399F0B7FD9FC08F3F9105A105B1056F
:103C700029F024F08FEF90E0A0E0B0E02FEF30E0EB
:103C8000A901481B590BCA010CC0B7FD89C08F3F61
:103C90009105A105B10529F024F08FEF90E0A0E097
:103CA000B0E0FF90EF90DF90CF90089514962C91A4
:103CB000822F90E06623A9F3E1CF1496CD90DD909A
:103CC000ED90FC901797662301F120E030E0A90108
:103CD000C701B6010F94243687FD65C020E030E0AF
:103CE0004FE753E4C701B6010F942C3918160CF4B2
:103CF00057C0A701960160E070E08FE793E40F944E
:103D000017380F94F638CB01CCCF20E030E0A90172
:103D1000C701B6010F94243687FD42C020E030E091
:103D20004FE753E4C701B6010F942C391816DCF1A4
:103D3000C701B601E6CF14966D917D918D919C914E
:103D400017973323B1F06D395FEF75078507950736
:103D500054F1611524E67207810591050CF52CE9F3
:103D60003FEF4FEF5FEF0F949037C90181509F4FA6
:103D700098CF6D394FEF7407840794078CF0611565
:103D800054E675078105910574F424E630E040E0BF
:103D900050E00F949037C90184CF8FEF9FEF81CF10
:103DA00090E080E07ECF8FEF90E07BCFCF93DF93EA
:103DB000EC01DB01898182958F708630E1F128F476
:103DC00081508230C8F080E014C0873009F18A50F9
:103DD0008230C8F72FEF30E00F94FC3724E630E054
:103DE00040E050E00F9490372C833D834E835F83F7
:103DF00081E0DF91CF9108952FEF30E00F94FC37F1
:103E000024E630E040E050E00F9490372C83F0CF70
:103E10002FEF30E00F94FC3724E630E040E050E034
:103E20000F949037CA01B9010F942B366C837D83B0
:103E30008E839F83DDCF2CE933E60F94FC3724E695
:103E400030E040E050E00F9490372C833D834E8368
:103E50005F83B9CFDC011196EC911197E295EF7079
:103E6000E150EB3008F039C0F0E08827E55CF04E17
:103E70008F4F0D94E5375E1F5E1F6D1F461F461F57
:103E80004F1F661F661F661F461F461F14966D91C3
:103E90007D918D919C9117970F942B3608951496D0
:103EA0006D917D918D919C91179724E630E040E0D3
:103EB00050E00F949037CA01B901EECF14966C917F
:103EC00070E090E080E00F942936089514966D918B
:103ED0007D918D919C911797089560E070E0CB01E2
:103EE0000895DC011196EC911197E295EF70E15085
:103EF000EB3008F037C0F0E08827EE57F04E8F4FD8
:103F00000D94E537941F941FB21F8D1F8D1FA31FA3
:103F10009A1F9A1F9A1F8D1F8D1F14966D917D9168
:103F20008D919C911797089514966C9170E090E094
:103F300080E0089514966D917D918D919C911797D5
:103F40000F94F638089514966D917D918D919C9102
:103F5000179724E630E040E050E00F949037CA0114
:103F6000B901089560E070E0CB010895CF92DF922F
:103F7000EF92FF920F931F93CF93DF9300D000D067
:103F80001F921F92CDB7DEB709831A832B833C8320
:103F90004D835E836F837887FC01208131812115F9
:103FA000310589F490E080E028960FB6F894DEBFE2
:103FB0000FBECDBFDF91CF911F910F91FF90EF907A
:103FC000DF90CF9008958C01C9010E9485FAE82EF8
:103FD000F12CF6E0EF16F10494F40E94F5BE009780
:103FE00021F0FC012085207F2087BC01F801808121
:103FF00091810E94F2FCFFEFEF1AFF0AEACF65E021
:10400000F801808191810E94F3F98C01892B51F292
:104010008981803138F6CE0101960E94711F1616F3
:1040200017061806190624F4F80180858D7089F0AA
:10403000F80180858F7080876FE37AE08EE692E1E9
:104040000F9406158EE692E10F94BA1281E090E08B
:10405000ABCF0F94B4066B017C01CE0101960E9498
:10406000711FC60ED71EE81EF91EF801C186D28642
:10407000E386F48689818295807F8260808764E30D
:104080007AE08EE692E10F940615CE0101960E9429
:10409000711FAB01BC012AE030E08EE692E10F9483
:1040A000AF136EE27AE08EE692E10F940615F80106
:1040B00041855285638574852AE030E08EE692E181
:1040C0000F94AF13BFCFEF92FF920F931F93CF9335
:1040D000DF93CDB7DEB7C056D1090FB6F894DEBF77
:1040E0000FBECDBF7C016A960FAF6A976B961FAF6C
:1040F0006B976C962FAF6C976D963FAF6D976E96E2
:104100004FAF6E976F965FAF6F97A0966FAFA09708
:10411000A1967FAFA19798E0FE01E75AFF4FDE011D
:10412000AF5ABF4F01900D929A95E1F76A96EFADA5
:104130006A97E150ED3008F07DC0F0E08827EC553B
:10414000FF4D8F4F0D94E5370A210C2118211A21BC
:104150001621B12008211A211A210E211021142123
:10416000122167E0CE018F5A9F4F0E944A1B6AE1DD
:104170007AE08EE692E10F9406154AE050E06296EE
:104180006FAD62978EE692E10F94D0126FE07AE005
:104190008EE692E10F940615CE018F5A9F4F0E9432
:1041A000711FAB01BC012AE030E08EE692E10F9472
:1041B000AF138EE692E10F94BA1262960FAD62973A
:1041C00063961FAD639764962FAD649765963FAD78
:1041D000659766964FAD669767965FAD67976896E9
:1041E0006FAD689769967FAD6997C7010E94B61F4A
:1041F00081E090E0C05ADF4F0FB6F894DEBF0FBEEB
:10420000CDBFDF91CF911F910F91FF90EF90089557
:1042100066E0A8CF62E0A6CF61E0A4CF6BE0A2CFBA
:104220006AE0A0CF6CE09ECF6DE09CCF63E09ACFB8
:1042300065E098CF90E080E0DDCFDC011196EC9155
:104240001197E295EF70E150EB3008F03EC0F0E0DE
:104250008827E25DFE4D8F4F0D94E53744214421C0
:104260006521392139215E214F214F214F213921EB
:10427000392114962D913D914D915C911797A4E6AB
:10428000B0E00F94AF37089514966C9184E6689F60
:10429000B0011124072E000C880B990B089520E023
:1042A00030E048EC52E414966D917D918D919C9193
:1042B00017970F948A360F94F638089514966D91D7
:1042C0007D918D919C911797089560E070E0CB01EE
:1042D0000895FC01A7812A2F2E7FD1F0818182953C
:1042E0008F7081508330A0F4A695A150BB0B2BE5B5
:1042F00031E00F94FC3724E630E040E050E00F94CA
:104300009037DA01C90187569F4FAF4FBF4F0895CD
:104310008FEF9FEF08952F923F924F925F926F928F
:104320007F928F929F92AF92BF92CF92DF92EF9245
:10433000FF920F93CF93DF9300D01F92CDB7DEB7DC
:104340007C017A8369835C834B83DB011C92FC01D3
:104350006081662309F44EC030FF4CC0F9E06F9FC6
:10436000B00111246F5B704FCD010F946630D701FF
:1043700011968C91807F41F04B815C8169E177E0FF
:1043800089819A810F94623CE981FA810190002031
:10439000E9F7319729813A81E21BF30B19012E0EBF
:1043A0003F1E4B815C814E1B5F0B415051095C836A
:1043B0004B83D7011196EC9111978E2F807F09F4D2
:1043C000F7C0E295EF70E150EC3008F0F1C0F0E09A
:1043D0008827E251FE4D8F4F0D94E537FD21A02235
:1043E0000D236C2387234B221D231D231D233922DC
:1043F0002122A32329803A80DCCFF7018481282F52
:1044000030E050E040E0002359F030E0A4E6B0E0B6
:104410000F94C2372FEF30E040E050E00F94903718
:104420005F934F933F932F938BE396E09F938F93EC
:10443000FC81FF932B812F933F922F920F949A3CF4
:10444000B2C017968C9117978F9316968C911697EA
:104450008F9315968C9115978F9314968C918F93BB
:104460008EE396E09F938F93BC81BF93EB81EF9394
:10447000E3CF17968C9117978F9316968C9116977A
:104480008F9315968C9115978F9314968C918F938B
:1044900082E496E0E7CF1496CD90DD90ED90FC900D
:1044A0001797F7FE34C084E6882E912CA12CB12CEE
:1044B000C701B601A50194010F9490379B01AC018F
:1044C00088279927DC01821B930BA40BB50BBF93A4
:1044D000AF939F938F9366277727CB016C197D0944
:1044E0008E099F09A50194010F9490375F934F9314
:1044F0003F932F9386E496E09F938F933C813F9365
:104500004B814F933F922F920F949A3C4CC0C7011E
:10451000B60124E630E040E050E00F9490379F93DE
:104520008F937F936F935F934F933F932F9387E482
:1045300096E09F938F939C819F93AB81AF93E2CF43
:10454000C7010E946921BC01D7011696CC9016972D
:104550001796DC901797D0FADD24D0F814969C912A
:1045600014971596FC90EB80BC80292F30E050E02A
:1045700040E077FD35C0011135C07F936F931F92E6
:104580001F921F929F931F92FF92DF92CF9280E51E
:1045900096E09F938F93FC81FF932B812F933F9203
:1045A0002F920F949A3C0FB6F894DEBF0FBECDBF8A
:1045B00089819A810F900F900F900F90DF91CF918A
:1045C0000F91FF90EF90DF90CF90BF90AF909F90B2
:1045D0008F907F906F905F904F903F902F900895B5
:1045E000002361F0292F30E0A4E6B0E00F94C23739
:1045F0002FEF30E040E050E00F9490375F934F93FF
:104600003F932F931F92FF92DF92CF9283E596E024
:104610009F938F93BF92EF9275CF15968C911597BC
:104620001F928F9316969C91169717968C91817076
:104630008F939F9386E596E015CF14968D909D906D
:10464000AD90BC90179720E030E0A901C501B401FE
:104650000F9424362401350187FF04C077FA709443
:1046600077F87094C301B2010F94F6386B01072EEE
:10467000000C880B990B0F942B369B01AC01C301E6
:10468000B2010F94173820E030E04AE754E40F9469
:104690008A360F9481390F94F638062F772E20E052
:1046A00030E0A901C501B4010F94243687FF07C08B
:1046B0007F920F93DF92CF928CE596E0D3CE7F92DC
:1046C0000F93DF92CF928DE596E09F938F933C817D
:1046D0003F934B814F93B0CE14968C9114971F92B9
:1046E0008F9315968C9115971F928F9316968C9198
:1046F0001F928F9383E596E09F938F93BC81BF9326
:10470000EB81EF933F922F920F949A3C4CCF1796E8
:104710008C9117971F928F9314968C9114971F92D8
:104720008F9315968C9115971F928F9316968C9157
:104730001F928F9380E596E09F938F93BC81BF93E8
:10474000EB81EF93DFCE14966D917C914B815C8170
:10475000C1010F94803C2CCFEF92FF920F93CF9327
:10476000DF93CDB7DEB7A0970FB6F894DEBF0FBECC
:10477000CDBF7C0100E020E033E040E250E0BE012C
:104780006F5F7F4F0E948B21BE016F5F7F4F8EE670
:1047900092E10F94101469E270E18EE692E10F94B9
:1047A0000615F701618162956F704AE050E08EE670
:1047B00092E10F94D01262E270E18EE692E10F94E2
:1047C0000615F70161816F704AE050E08EE692E1D4
:1047D0000F94D0128EE692E10F94BA12A0960FB603
:1047E000F894DEBF0FBECDBFDF91CF910F91FF9048
:1047F000EF900895CF93DF93EC016115710539F4C3
:104800008F8181708F8381E0DF91CF9108958981BD
:10481000982F92959F7029F180E09430A8F79B0122
:10482000770F440B550B2959310941095109A4E669
:10483000B0E00F94AF372BE531E040E050E00F944B
:10484000903737FF02C030E020E02536310514F004
:1048500024E630E02F5F220F8F818170282B2F8379
:10486000D2CF8F7080628983DACFFC019181892F4A
:1048700082958F7021F0823029F080E008959F703A
:10488000906291839B0177FF02C030E020E02E36DA
:1048900081E0380714F02DE631E02683878130FB74
:1048A00080F9878381E00895EF92FF920F931F9321
:1048B000CF93DF93FC01892B69F19081992351F10A
:1048C0009D3291F180ED890F8A3070F1C8E0D0E01F
:1048D000953211F1CEEFDFEF9B37F1F0C7E1D0E079
:1048E0009332D1F08F018AE4E82E8FE0F82EC1E0F8
:1048F000D0E0C7010F943F30AC01B701C8010F945D
:104900005830892B49F0219689E0E80EF11CC93115
:10491000D10579F7CFEFDFEFCE01DF91CF911F9176
:104920000F91FF90EF900895D0E0C0E0F5CFEF92A7
:10493000FF920F931F93CF93DF93EC01892B51F1DB
:1049400088858F70843009F5E984FA84C7010E9454
:1049500054248C0118161906ECF4C7010E946ABC95
:10496000C801012E000CAA0BBB0B89879A87AB8765
:10497000BC878885807F82608887C801DF91CF915E
:104980001F910F91FF90EF900895823019F40985DF
:104990001A85F3CF10E000E0F0CF4F925F926F9254
:1049A0007F928F929F92AF92BF92CF92DF92EF92BF
:1049B000FF920F931F93CF93DF93CDB7DEB760972E
:1049C0000FB6F894DEBF0FBECDBF6115710539F586
:1049D00028E0FC01DE01119601900D922A95E1F785
:1049E00029813A814B815C816D817E818F8198859F
:1049F00060960FB6F894DEBF0FBECDBFDF91CF91AA
:104A00001F910F91FF90EF90DF90CF90BF90AF90EC
:104A10009F908F907F906F905F904F9008956B0163
:104A20008C016EE877E0C6010E9441F95C01F80153
:104A3000F080FF2009F453C0009709F450C0FC0136
:104A400080858295807F859585958595859584302F
:104A500009F4BFC0853009F042C065E676E08EE615
:104A600092E10F9410148EE692E10F94BA12F501C0
:104A7000E680F780E114F10491F1F70180858F70F1
:104A80005701823061F0B12CA12CE114F10409F43A
:104A90001DC1F70180858F70853021F0F701E2801C
:104AA000F380F3CFC7010E9485FA8230B9F760E046
:104AB000C7010E94F3F90E9497244C0161E0C701ED
:104AC0000E94F3F9F80120812815190439F7FC0137
:104AD00020852F70223011F7009709F001C163E79C
:104AE00076E0C6010E9441F97C01F8018181807F56
:104AF00009F407C1E114F10409F47DC0F7018085D0
:104B00008F70853009F001C1C7010E9485FA843099
:104B100009F0FBC0C8010E94711F4B015C0160E0FD
:104B2000C7010E94F3F9FC0181859285A385B485B4
:104B300019821A821B821C821D821E821F82188685
:104B400088169906AA06BB060CF499C08A818F7054
:104B50008A8363E0C7010E94F3F95C0162E0C70148
:104B60000E94F3F9FC01418452846384748461E0FF
:104B7000C7010E94F3F94C0160E0C7010E94F3F9FC
:104B8000FC01C184D284E384F484C8010E94711FB3
:104B9000F501218532854385548524193509460957
:104BA00057096C197D098E099F090F945E37F4012E
:104BB00021853285438554852C193D094E095F09AD
:104BC0000F949037BA01A901440D551D661D771D3C
:104BD00031C066E377E0818592850F94523C892B42
:104BE00009F07DCFF0E1FF1609F460C0FF1568F011
:104BF00082E0F816E1F1F801408151816281738110
:104C000084819581A681B78129C0E1E1FE16F1F189
:104C1000F2E1FF12F0CF19821A821B821C821D82E0
:104C20001E821F8218868A818F708A8344E150E039
:104C300060E070E0CE0101960E94871D29873A87C7
:104C40004B875C876D877E878F87988B49855A85D0
:104C50006B857C858D859E85AF85B88949835A8310
:104C60006B837C838D839E83AF83B887B9CE198293
:104C70001A821B821C821D821E821F8218868A81D4
:104C80008F708A8340E050E0BA01D4CF19821A8233
:104C90001B821C821D821E821F8218868A818F7051
:104CA0008A8340E850E060E070E0C4CF19821A8245
:104CB0001B821C821D821E821F8218868A818F7031
:104CC0008A834FEF50E060E070E0B4CFA114B104EC
:104CD00009F405CFF50180858F7009F400CFC50177
:104CE00019821A821B821C821D821E821F821886D4
:104CF0002A812F702A83FC01418552856385748542
:104D000099CFE114F10409F476CFF70180858F7013
:104D100009F071CF19821A821B821C828A818F70DE
:104D20008A8349815A816B817C8180E090E0DC013B
:104D300095CF0F931F93CF93DF938C01FC01C0811C
:104D4000D1816FE270E0CE010F948F3C0097E9F0C3
:104D5000FC011192CF010E940017EC0163E07AE0A0
:104D60008EE692E10F9406154AE050E0BE018EE611
:104D700092E10F94F7138EE692E10F94BA12CE01EE
:104D8000DF91CF911F910F910895CE010E940017DE
:104D9000EC01892BA1F3F80111821082F0CFDC0124
:104DA000ED91FC91309729F090859F7081E09530CE
:104DB00009F080E00895EF92FF920F931F93CF9335
:104DC000DF93EC017B018E819F81892BD9F488814F
:104DD00099810E9485FA082F10E00530110594F49E
:104DE0000E94F5BE009721F0FC012085207F2087DE
:104DF0009F838E83BC01888199810E94F2FC0F5FA2
:104E00001F4FEBCFEE81FF813097D9F08085982F2F
:104E10009F70A9F4807F82608087EE81FF81118678
:104E2000128613861486EE81FF81F782E682C7011F
:104E3000DF91CF911F910F91FF90EF9008959230E5
:104E400061F3F12CE12CF3CFCF92DF92EF92FF923E
:104E50000F931F93CF93DF93EC016A017B018E8147
:104E60009F81892BD9F4888199810E9485FA082F26
:104E700010E00530110594F40E94F5BE009721F072
:104E8000FC012085207F20879F838E83BC01888141
:104E900099810E94F2FC0F5F1F4FEBCFEE81FF81E3
:104EA000309749F18085982F9F7019F5807F826037
:104EB0008087EE81FF81C186D286E386F48667EF24
:104EC00079E08EE692E10F9406152AE030E0B70112
:104ED000A6018EE692E10F94AF138EE692E1DF9188
:104EE000CF911F910F91FF90EF90DF90CF900D9495
:104EF000BA129230F1F2DF91CF911F910F91FF9092
:104F0000EF90DF90CF900895FC0186819781009704
:104F100099F0FC0120852F70223029F4618572857B
:104F2000838594850895253039F460E00E94F3F973
:104F3000009711F0FC01F2CF60E070E0CB01089522
:104F40000F931F93CF93DF93FC01C281D3812097EE
:104F5000F9F088858F70823049F4672BC9F4898510
:104F60009A85DF91CF911F910F910895853081F43B
:104F70008B01CE010E9485FA8017110649F044F09A
:104F8000602FCE010E94F3F9FC0181859285E9CF63
:104F900090E080E0E6CF0F931F93CF93DF93EC0177
:104FA0008B017B836A8380E692E09983888370E03B
:104FB00060E0C8010E94A02797FD0CC09D838C83F0
:104FC000C8010E946B169F838E83DF91CF911F9142
:104FD0000F910895919581959109F0CFCF92DF922D
:104FE000EF92FF920F931F93CF93DF93EC01888191
:104FF00099810E9485FA082F10E0043011059CF475
:105000000E94F5BE009739F0DC0118962C91189794
:10501000207F18962C93BC01888199810E94F2FC14
:105020000F5F1F4FEACFC880D98060E0C6010E94A1
:10503000F3F9FC011185188761E0C6010E94F3F9BC
:105040007C019B838A8362E0C6010E94F3F99D8301
:105050008C8364E0C6010E94F3F99F838E8315312F
:1050600008F027C1E12FF0E08827E65CF74D8F4F6D
:105070000D94E5376428642864284F285929592954
:10508000592959295929592983287228B928E028EA
:10509000CB285929EB2864283F29592962298AE01D
:1050A00090E00F94F62D8C01BE010E94CB2784E581
:1050B00093E0D80111969C938E9319961C921E92A0
:1050C00018971A870987F5C088E090E00F94F62DAD
:1050D0008C01BE010E94CB278EE293E0F801918300
:1050E0008083EFCF8DE090E00F94F62D8C01BE0110
:1050F0000E94CB2788E093E0D8018D939C93C80150
:105100000E9407E0DECF89E090E00F94F62D8C013D
:10511000FC01D383C28384EE92E091838083CE012D
:105120000E941B15D80115969C938E93149785E7C2
:105130009EE018969C938E931797CE010E946B1653
:10514000892B09F4BECF70E060E0CE010E94A02759
:10515000F8018683882341F0823009F0B2CF82E1E2
:105160009FE090878783ADCF81ED91E19087878322
:10517000A8CF8EE090E00F94F62D8C01DC01139601
:10518000DC93CE93129786EE93E08D939C93C801A7
:105190000E947DE096CF86E090E00F94F62D8C0182
:1051A000FC01D383C28380EC92E091838083CE01A3
:1051B0000E941B15D80115969C938E93149781CF4E
:1051C00086E090E00F94F62D8C01FC01D383C2831E
:1051D0008CE992E0EACF8BE090E00F94F62D8C0101
:1051E000FC01D383C28382EC93E091838083168297
:1051F00070E060E0CE010E94A02797FD2DC0D8018D
:1052000015969C938E931497D80114968D919C912A
:10521000009719F0863491052CF080E290E0F801B7
:105220009583848361E070E0CE010E94991620E0AE
:1052300030E04AE754E40F948A360F94FD38611544
:1052400071058105910589F0D80117966D937D93BD
:105250008D939C931A9735CF919581959109F8017B
:105260009583848381E08683CFCF88E893E1A0E0B3
:10527000B0E0F80187839087A187B28722CF86E0CC
:1052800090E00F94F62DFC01D383C2838EE993E066
:105290009183808315821482E114F10441F0D701D7
:1052A00018968C918F70863011F4F582E482FA871B
:1052B000E987DF91CF911F910F91FF90EF90DF90E1
:1052C000CF9008958CE090E00F94F62D8C01FC01B6
:1052D000D383C2838AE793E09183808370E060E0A8
:1052E000CE010E94991620E030E048EC52E40F9481
:1052F0008A360F94FD38D80114966D937D938D9363
:105300009C93179761E070E0CE010E94991620E00F
:1053100030E04AE754E40F948A360F94FD38F801E0
:105320006087718782879387CCCECF92DF92EF928E
:10533000FF926A017B0163E0FC01808191810E9400
:10534000F3F9FC01892BA9F080858D7091F4C0944C
:10535000D094E094F094CC24CA9481859285A3855E
:10536000B4858C219D21AE21BF2181879287A3879F
:10537000B487FF90EF90DF90CF900895CF92DF92A7
:10538000EF92FF926A017B0163E0FC0180819181D1
:105390000E94F3F9FC01892BA9F09085892F8D706B
:1053A00089F4907F92609087CC24FF2441855285B8
:1053B000638574854C295D296E297F294187528731
:1053C00063877487FF90EF90DF90CF900895CF921E
:1053D000DF92EF92FF926A017B0163E0FC01808122
:1053E00091810E94F3F9009791F0FC0120852F70C4
:1053F000223069F461857285838594856C217D21D5
:105400008E219F21FF90EF90DF90CF90089560E074
:1054100070E0CB01F7CFAF92BF92CF92DF92EF92C5
:10542000FF920F931F93CF93DF93CDB7DEB7CD5687
:10543000D1090FB6F894DEBF0FBECDBF5C01A796B1
:105440000FAFA797A8961FAFA897A9962FAFA997B8
:10545000AA963FAFAA97AB964FAFAB97AC965FAF0C
:10546000AC97AD966FAFAD97AE967FAFAE972396E4
:105470001FAE1EAE2397FE01ED5BFF4F82E1DF0101
:105480001D928A95E9F772961192119287E0DF01D9
:105490001D928A95E9F7CE018A599F4F0E94AC234D
:1054A000F0FE2CC0A796EFADA797E83108F050C1E9
:1054B000F0E08827E15AF54D8F4F0D94E537AE2B7C
:1054C000772AA52BA82BA82BA52B772AA82BA82BAE
:1054D000A82BA82BA82BA82BA82B772A772AA82B98
:1054E000A82BA82B772A772A772AA82BAE2B6FE335
:1054F0007EE0CE018B5A9F4F0F9438300E945FF9A7
:10550000882309F407C18091870C811103C1C1145C
:10551000D10409F05EC030E020E043E050E060E4F8
:10552000CE0101960E942DD9D501ED91FC916081AB
:1055300071814FE350E0CE0101960F94623CF1FE81
:1055400010C1A7968FADA797823009F40AC18530A4
:1055500009F407C1A8968FADA89782958F709FE038
:10556000980F9F70923018F0883009F0FAC001E06F
:1055700020E032E044E150E0BE016F5B7F4FCE019E
:105580008A599F4F0E948B21BE016F5B7F4FCE01D6
:1055900001960F94510767E27EE08EE692E10F9448
:1055A0000615BE016F5F7F4F8EE692E10F941014D7
:1055B00064E27EE08EE692E10F940615BE016F5B19
:1055C0007F4F8EE692E10F9410148EE692E10F94D5
:1055D000BA12A8968FADA897807F87010027107216
:1055E000882311F0F1FC04C00115110509F4F5C080
:1055F00030E020E043E050E060E4CE0101960E94FC
:105600002DD9D501ED91FC91608171814FE350E07E
:10561000CE0101960F94623CC114D10469F063EF8E
:1056200079E0CE0101960F943C3C4FE350E0B60187
:10563000CE0101960F94623C63EF79E0CE010196B2
:105640000F943C3C4FE350E067E17EE0011511050B
:1056500011F463E17EE0CE0101960F944830A896E4
:105660008FADA89782958F708450823008F09FC0CC
:1056700067E1CE018A599F4F0E944A1B6F962FAF58
:105680006F97A0963FAFA097A1964FAFA197A29614
:105690005FAFA297A3966FAFA397A4967FAFA4978F
:1056A000A5968FAFA597A6969FAFA69700E020E09E
:1056B00033E044E150E0BE016F5B7F4FCE018A5979
:1056C0009F4F0E948B216DE07EE08EE692E10F9469
:1056D0000615BE016F5F7F4F8EE692E10F941014A6
:1056E0006AE07EE08EE692E10F940615BE016F5BE4
:1056F0007F4F8EE692E10F9410148EE692E10F94A4
:10570000BA120E945FF9882329F08091870C8823C0
:1057100009F455C0A701FF0C660B770BC5010E9469
:10572000BE2990E080E0C359DF4F0FB6F894DEBF8A
:105730000FBECDBFDF91CF911F910F91FF90EF90E2
:10574000DF90CF90BF90AF9008956BE37EE0D1CE15
:105750006DE27EE08EE692E10F940615E894F0F893
:10576000CDCEF0FE36CF66968FAD6697882309F4CE
:1057700030CFBE016B5A7F4FCE0101960F94510777
:105780006EE17EE08EE692E10F940615BE016F5F3A
:105790007F4F8EE692E10F9410146BE17EE08EE66F
:1057A00092E10F940615BE016B5A7F4F0ACF20E09D
:1057B00032E0012B11F020E033E000E07ACFBE01AF
:1057C0006F5B7F4FCE0101960F94510740E052E08E
:1057D00060E070E0C5010E949529F0FE90C0A79698
:1057E000EFADA797E150E53118F5F0E08827E450D8
:1057F000F44D8F4F0D94E537072D182C182C182CCD
:10580000182C072D182C182C182C182C182C182C88
:10581000182C0C2D042D182C182C182C112CFE2CA7
:10582000012D60E07EE0CE018B5A9F4F0F943830FF
:1058300030E020E043E050E060E4CE0101960E94B9
:105840002DD9D501ED91FC91608171814FE350E03C
:10585000CE0101960F94623CC114D10469F063EF4C
:1058600079E0CE0101960F943C3C4FE350E0B60145
:10587000CE0101960F94623C63EF79E0CE01019670
:105880000F943C3C4FE350E06AEE7DE0CE01019680
:105890000F94483064EE7DE08EE692E10F94061599
:1058A000BE016F5F7F4F8EE692E10F94101461EEA0
:1058B0007DE08EE692E10F940615BE016B5A7F4F94
:1058C0008EE692E10F9410148EE692E10F94BA12D4
:1058D0000E945FF9882309F41DCF8091870C811104
:1058E00019CFBE016B5A7F4FCE0101960F9451071D
:1058F00040E051E060E070E0C5010E949529F2FEB1
:105900007AC040E050E061E070E0C5010E94E72904
:10591000672B682B692B09F482C069ED7DE0CE010D
:105920008B5A9F4F0F94383030E020E043E050E036
:1059300060E4CE0101960E942DD9D501ED91FC9134
:10594000608171814FE350E0CE0101960F94623C7B
:10595000C114D10469F063EF79E0CE0101960F9490
:105960003C3C4FE350E0B601CE0101960F94623CFF
:1059700063EF79E0CE0101960F943C3C4FE350E099
:1059800066EC7DE0CE0101960F94483060EC7DE03E
:105990008EE692E10F940615BE016F5F7F4F8EE693
:1059A00092E10F9410146DEB7DE08EE692E10F947E
:1059B0000615BE016B5A7F4F8EE692E10F941014CC
:1059C0008EE692E10F94BA120E945FF9882309F4DF
:1059D000A1CE8091870C81119DCEBE016B5A7F4F65
:1059E000CE0101960F94510740E054E060E070E072
:1059F000C5010E94952981E090E095CE6BEF7DE096
:105A000012CF67EF7DE00FCF6EEE7DE00CCFF5019A
:105A10008085853009F00CCF65E07EE004CF40E062
:105A200050E062E070E0C5010E94E729672B682B17
:105A3000692B19F062ED7DE072CF6BEC7DE06FCFEA
:105A4000CF93C62F63E0FC01808191810E94F3F91E
:105A5000FC01892B21F19085892F8D7001F5907FB4
:105A60009260908781859285A385B4858827BB271E
:105A70008C2B81879287A387B4876FEE79E08EE6BF
:105A800092E10F9406154AE050E06C2F8EE692E109
:105A90000F94D0128EE692E1CF910D94BA12CF916D
:105AA0000895CF92DF92FF920F931F93CF93DF93CE
:105AB000F12C6115710509F499C06A01EB018C01A3
:105AC000CB010E94CF26F82E882309F48FC0D2FE86
:105AD00009C0D8018C918B3009F44BC0E8F58A30AD
:105AE00009F44CC0D0FE09C0F801608186EF860F32
:105AF000843018F0CE010E94202DD1FE6EC0D80156
:105B000014964D915D916D917C91179711968C91A2
:105B100082958F70873038F0893008F43EC08A5003
:105B2000823008F46CC0CE010E942B15EC81FD81FF
:105B3000309709F452C080858F709EEF980F923095
:105B400010F081114AC0D80111969C91907F8085F8
:105B50008F70892B808741C08C30B9F040E050E0D5
:105B600062E070E08D3009F0BDCFCE010E94BE2909
:105B7000B9CF40E050E061E070E0F7CF40E050E0A6
:105B800061E070E0CE010E94952940E050E062E0C3
:105B900070E0CE010E949529A5CFEC81FD81309760
:105BA000E1F080858F709EEF980F923010F0811198
:105BB00014C04187528763877487EC81FD8180859B
:105BC000807F83608087EC81FD818085982F907F26
:105BD0008F708067903609F4BDCF6AE37FE08EE670
:105BE00092E10F940615C8010E94AC238F2DDF911E
:105BF000CF911F910F91FF90DF90CF900895CE012C
:105C00000E942B15EACF63E0FC01808191810E9404
:105C1000F3F9009719F0FC01818508958FEF08953D
:105C2000CF92DF92EF92FF920F931F93CF93DF9368
:105C30006115710509F460C06A017B018C01CB011B
:105C40000E94CF26D82F882389F1D70114968D91F1
:105C50009C91009709F43FC0FC01C0852C2F2F7048
:105C60003EEF320F323010F021112AC0C595C59594
:105C7000C595C595D0FE5EC0C7010E94032EF801F0
:105C80008083CC2351F1C295C07F81818F70C82B56
:105C9000C183D7011496ED91FC9181859285A385EE
:105CA000B485F80184839583A683B7838D2FDF9114
:105CB000CF911F910F91FF90EF90DF90CF900895BB
:105CC000253049F460E00E94F3F9009721F0DC01EF
:105CD0001896CC91CBCFC0E0CDCFD7011496ED91E3
:105CE000FC9180858295807F8595859585958595A4
:105CF000823021F0833081F0D0E0D8CF41855285C9
:105D000063857485F80181818F70806A8183448303
:105D1000558366837783CACF4185528563857485B1
:105D2000F80181818F708067818344835583668306
:105D30007783BCCFCC2389F2C295C07FF801A5CF71
:105D4000AF92BF92CF92DF92EF92FF920F931F9389
:105D5000CF93DF9300D000D01F921F92CDB7DEB754
:105D60005C017B0160FF03C0E894E0F8F4F8F4FC08
:105D70000DC00E94AEDA663971058105910530F0DB
:105D80008091F70D9091F80D059719F5A70144271B
:105D90005770052E000C660B770BC5010E94BE29BB
:105DA0006CEA7DE08EE692E10F9406158FEF9FEF8F
:105DB00028960FB6F894DEBF0FBECDBFDF91CF910E
:105DC0001F910F91FF90EF90DF90CF90BF90AF9019
:105DD000089519821A821B821C821D821E821F82D4
:105DE00018868A818F708A8340E053E0B501CE0126
:105DF00001960E94102E40E057E060E070E0C5017F
:105E00000E94E729E62AF72AD12CC12C09811A81A0
:105E10002B813C814D815E816F817885C5010E9417
:105E20000B2AC6CFCF93DF93EC0140E053E060E054
:105E300070E00E94E729611571058105910599F0CF
:105E40002091F70D3091F80D2630310561F4CE0127
:105E50000E94A02E40E053E060E070E0CE01DF91B0
:105E6000CF910C949529DF91CF910895AF92BF9275
:105E7000CF92EF92FF920F931F93CF93DF9300D0B7
:105E800000D01F921F92CDB7DEB75C0109831A8341
:105E90002B833C834D835E836F83788766E179E053
:105EA0008EE692E10F940615CE0101960E94AC2376
:105EB000898181112FC00A810F70013081F138F181
:105EC000023019F010E00530E9F5D501ED91FC91B3
:105ED00000A0F1A1E02D09811A812B813C814D8127
:105EE0005E816F817885C501199581E090E02896E3
:105EF0000FB6F894DEBF0FBECDBFDF91CF911F91DB
:105F00000F91FF90EF90CF90BF90AF900895CC2469
:105F1000C394DBCF813071F1823009F451C069E064
:105F200079E08EE692E10F9406154AE050E069812F
:105F30008EE692E10F94D0128EE692E10F94BA129F
:105F400001E010E069EF78E08EE692E10F9406152B
:105F50004AE050E0B8018EE692E10F94F7138EE626
:105F600092E10F94BA12CE0101960E94AC2390E008
:105F700080E0BDCFCE0101960E9402FA4497BCF4A6
:105F80006EE170E0CE0101960E94D61EF50162819D
:105F9000738140E052E0CE0101960E94512D60E0F5
:105FA00072E1D50112968D919C910E94A02ED5018F
:105FB000ED91FC9100A0F1A1E02DCC24C3948BCFF6
:105FC0001D821E821F821886D501ED91FC9100A0D2
:105FD000F1A1E02DCC24C39402E01A812B813C81F5
:105FE00040E07ECF8F929F92AF92BF92CF92DF928E
:105FF000EF92FF920F931F93CF93DF93CDB7DEB74E
:1060000060970FB6F894DEBF0FBECDBF7C018B0149
:1060100062E070E00E94A0276C0119861A861B8638
:106020001C861D861E861F86188A8A858F708A8721
:1060300090E080E0D7FC43C040E052E0B701CE01E1
:1060400009960E94102E63E070E0C7010E94A0270D
:10605000AC011816190614F04FE350E081E0C816A1
:10606000D10429F4012F110F110B112704C082E074
:10607000C816D104D4F32FEF30E0D8010F94FC37C9
:106080009A01550F440B550B0F9490374901690144
:10609000C7010E94032E082F10E060E0CE01099690
:1060A0000E94091E88159905E9F4892B31F0023008
:1060B000110501F105301105E9F081E090E06096ED
:1060C0000FB6F894DEBF0FBECDBFDF91CF911F9109
:1060D0000F91FF90EF90DF90CF90BF90AF909F9087
:1060E0008F900895CD2839F10630110539F001302F
:1060F000110521F061E0C7010E94202DB401CE01FD
:1061000009960E94B01D40E052E0B701CE01099609
:106110000E94512D0230110519F00530110529F4A6
:1061200060E071E0C7010E94A02E60E072E0C7014C
:106130000E94A02EC2CF0530110509F4BECF023057
:10614000110509F4BACF62E0C7010E94202D60E07A
:1061500071E0EDCF81E090E008950F931F93CF930E
:10616000DF9300D000D01F921F92CDB7DEB7198207
:106170001A821B821C821D821E821F8218862A811F
:106180002F702A83FC0102811381C8010E94032E13
:10619000813041F020F0823011F0853081F490E0C0
:1061A00080E002C081E090E028960FB6F894DEBF50
:1061B0000FBECDBFDF91CF911F910F91089540E0A9
:1061C00052E0B801CE0101960E94102E60E0CE018F
:1061D00001960E94091EE8CF8F929F92AF92BF92C4
:1061E000CF92DF92EF92FF920F931F93CF93DF93A3
:1061F000CDB7DEB767970FB6F894DEBF0FBECDBF41
:106200008C017B014C018BE0880E911C9F8A8E8A49
:10621000F801128611861386148E138E672B09F4EB
:1062200063C0A090F90DB090FA0DA114B10409F467
:106230005BC06FE270E0C7010F94473C6C01892B93
:1062400009F44AC0F701DE01119690E080E0BD013B
:106250002191222341F02F3231F08431910519F040
:106260002D930196F5CF860F971FFC011082C50173
:106270000E9441F9F80191838083B6016F5F7F4FDF
:106280004FE050E0C4010F94803CCE0146960E943E
:106290009926F801948F838F8E899F89892B09F421
:1062A0001386C8010E94CF26882319F0C8010E94D6
:1062B000EE2767960FB6F894DEBF0FBECDBFDF9115
:1062C000CF911F910F91FF90EF90DF90CF90BF90F3
:1062D000AF909F908F900895B701C5010E9441F93A
:1062E000F80191838083DDCFF80111821082D9CF2C
:1062F000DC0119968D919C91009739F0DC01ED91AC
:10630000FC910280F381E02D199408958F929F9261
:10631000AF92BF92CF92DF92EF92FF920F931F93B3
:10632000CF93DF93CDB7DEB7CD55D1090FB6F89433
:10633000DEBF0FBECDBF8C016B016115710519F079
:1063400041155105D1F466E970E18EE692E10F94B2
:1063500006156DE870E18EE692E10F940615B8011E
:106360008EE692E10F9410146BE870E18EE692E1F4
:106370000F9406158EE692E132C0460F571FDA01E0
:106380001C920E94AEDA4B0169E870E18EE692E160
:106390000F9406154AE050E0B4018EE692E10F94A6
:1063A000F71366E870E18EE692E10F940615B801E6
:1063B0008EE692E10F94101463E870E18EE692E1AC
:1063C0000F940615BAE38B16B1E09B06F4F466E76A
:1063D00070E187EC91E10F94061587EC91E10F9441
:1063E000BA12C35ADF4F0FB6F894DEBF0FBECDBF4F
:1063F000DF91CF911F910F91FF90EF90DF90CF90A1
:10640000BF90AF909F908F90089564E770E18EE603
:1064100092E10F940615B6018EE692E10F941014E6
:1064200062E770E18EE692E10F9406158EE692E146
:106430000F94BA121A821982FE0133968EE3DF019D
:106440001D928A95E9F78091F70D9091F80D0597C7
:1064500091F563E070E0C8010E9498177C01892BD8
:10646000E9F5E091ED0FF091EE0F808180FFB9CF5B
:1064700061E070E0C8010E949817892B09F4B1CF40
:1064800064E270E0C8010F948F3C892B09F0A9CF1A
:106490006AE570E18EE692E10F940615B8018EE68A
:1064A00092E10F9410148EE692E10F94BA12C80193
:1064B0000F94200196CF61E070E0C8010E94981708
:1064C0007C01892B49F562E070E0C8010E949817B1
:1064D0007C016FE470E1892B09F448CFE00EF11ED6
:1064E00066E470E1C7010F942F30892BE9F4F601BF
:1064F00001900020E9F73197EC19FD093297A0F0DF
:10650000C8010F942001F6018081882309F469CF26
:10651000C6010E9465BB65CF4FE350E0B801CE01D4
:1065200001960F94803CDACF64E270E0C8010F94CA
:106530008F3C892B09F055CFB701CE018F5B9F4F60
:106540000E94EC30CE018F5B9F4F0E94CF268823A4
:1065500039F1B601CE018F5B9F4F0F945617181675
:106560001906F4F489818823D9F08091F70D909170
:10657000F80D0597A9F06EE270E18EE692E10F94B6
:106580000615BE016F5F7F4F8EE692E10F941014E7
:106590008EE692E10F94BA12CE0101960F9420017B
:1065A000CE018F5B9F4F0E9478311BCFCF93DF933B
:1065B000EC01798368831A8619861B861C8E1B8ED4
:1065C0000E94CF26882329F0CE01DF91CF910C9431
:1065D000EE27DF91CF910895CF93DF93EC01FB017C
:1065E0002481358140815181628173810F94AF1381
:1065F000CE01DF91CF910895CF92DF92EF92FF927B
:106600001F93CF93DF9300D000D0CDB7DEB76AE9F8
:1066100070E18DEB91E10F94061581EAE82E81E19E
:10662000F82E10E090E1C92ED12CF70181917F0165
:10663000803130F467E776E08DEB91E10F94101430
:10664000153041F1F7013197808190E0B0E0A0E092
:1066500089839A83AB83BC83DE82CD82BE016F5F68
:106660007F4F8DEB91E10E94EC3268E970E10F946D
:1066700006151F5F1630C9F626960FB6F894DEBFD2
:106680000FBECDBFDF91CF911F91FF90EF90DF90B4
:10669000CF9008958091A61190E0B0E0A0E08983AA
:1066A0009A83AB83BC83DE82CD82BE016F5F7F4F56
:1066B0008DEB91E10E94EC320F94BA12DACFEF9297
:1066C000FF920F931F93CF93DF9300D000D0CDB7ED
:1066D000DEB77C018B0162E47EE08EE692E10F94EE
:1066E0000615012E000C220B330B09831A832B8312
:1066F0003C8380E190E09E838D83BE016F5F7F4F7E
:106700008EE692E10E94EC320F94BA1240E058E01B
:1067100060E070E0C7010E94BE2981E08093D20B47
:1067200026960FB6F894DEBF0FBECDBFDF91CF9196
:106730001F910F91FF90EF9008956F927F928F922B
:106740009F92AF92BF92CF92DF92EF92FF920F9300
:106750001F93CF93DF93CDB7DEB72C970FB6F89486
:10676000DEBF0FBECDBF4C01762E672E6A015901E8
:1067700081E090E09093E00B8093DF0B26E040E80F
:1067800055E260E070E082E19FE00E9431B97092D2
:10679000121082E19FE090931110809310101092DC
:1067A0001D1110921F1110921E110130110509F4D4
:1067B00093C00CF086C0012B09F493C06DE97EE014
:1067C0008EE692E10F9406154AE050E0672D762D93
:1067D0008EE692E10F94F71365E97EE08EE692E192
:1067E0000F940615C601B0E0A0E089839A83AB83BD
:1067F000BC8380E1682E712C7E826D82BE016F5F4A
:106800007F4F8EE692E10E94EC328C0161E97EE0DE
:106810000F9406154AE050E0B501C8010F94F71334
:1068200069E87EE0C8010F940615C701B0E0A0E05A
:106830008F839887A987BA877C866B86BE01695F3C
:106840007F4FC8010E94EC320F94BA12A114B10418
:1068500009F454C082E0A816B10409F05FC0D092D8
:106860009810C092971010929A1010929910F0926E
:106870009C10E0929B1086E00F94DE081092E00BD3
:106880001092DF0B882309F453C0682F70E0C40115
:106890000E945F3390E080E02C960FB6F894DEBF44
:1068A0000FBECDBFDF91CF911F910F91FF90EF9061
:1068B000DF90CF90BF90AF909F908F907F906F9020
:1068C00008950330110581F00430110509F076CFE9
:1068D000FE24EF24FE2472CFFE2CEE24EE24EA9454
:1068E0006DCFFF24FA946ACFEF2821F422E0E22E44
:1068F000F12CEECFEE24E394F12CEACFD092981055
:10690000C092971090E080E0EE2011F080E09FEFC1
:1069100090939A108093991085E0AECF61E77EE066
:106920008EE692E10F9406151092E00B1092DF0BA9
:1069300081E090E0B1CF8F929F92AF92BF92DF92B1
:10694000EF92FF920F931F93CF93DF93CDB7DEB7F4
:10695000A5970FB6F894DEBF0FBECDBF7C010E8F9A
:106960001F8F28A339A34AA35BA36CA37DA3CE01E9
:106970004E960E942A1F4B015C01D7011296ED91A1
:10698000FC9180858F70843009F0E0C0102F618504
:106990007285CE0101960E94EC30CE0101960E94D4
:1069A000CF26882309F44AC08985893009F046C07A
:1069B00070E060E0CE0101960E94A027082FD92E3A
:1069C00068E67EE08EE692E10F9406154AE050E01C
:1069D000602F7D2D8EE692E10F94F71366E67EE040
:1069E0008EE692E10F940615B501A4018EE692E1C0
:1069F0000F94DE1260E67EE08EE692E10F940615BB
:106A0000612F70E04AE050E08EE692E10F94F713B8
:106A10008EE692E10F94BA128091DF0B9091E00B19
:106A2000892B29F140E053E0B701CE014E960E9438
:106A3000512D70E060E0C7010E945F3310E000E07C
:106A4000CE0101960E947831C801A5960FB6F89440
:106A5000DEBF0FBECDBFDF91CF911F910F91FF9091
:106A6000EF90DF90BF90AF909F908F90089581E05E
:106A700090E09093E00B8093DF0B26E040E855E236
:106A800060E070E082E19FE00E9431B90093121053
:106A900082E19FE0909311108093101010921D11CD
:106AA00010921F1110921E11123009F44CC01530B3
:106AB00009F449C022E538EB42E152E4C501B401D2
:106AC0000F94183820E030E040E251E40F948A3609
:106AD0002DEE3EE94CE35EE30F9484384B015C01FC
:106AE00020E030E0A9010F942C3920E030E040E0B4
:106AF0005FE387FD23C0C501B4010F9418380F94DC
:106B0000F63883ED97E09093981080939710109249
:106B10009A101092991070939C1060939B1086E0CD
:106B20000F94DE081092E00B1092DF0B01E010E0F2
:106B3000882309F485CF682F70E07DCFC501B401AB
:106B40000F941738DCCF70E060E0DBCF10E000E09E
:106B50007BCFCF92DF92EF92FF920F931F93CF9351
:106B6000DF9300D000D01F921F92CDB7DEB77C011B
:106B700009831A832B833C834D835E836F837887DD
:106B8000CE0101960E9402FA8C018981882359F076
:106B90009A819F70923008F0BAC0823011F085302F
:106BA00011F410E000E070E060E0C7010E94A0274F
:106BB000D82EC92E6CE57EE08EE692E10F94061584
:106BC0004AE050E06D2D7C2D8EE692E10F94F71394
:106BD0006AE57EE08EE692E10F9406154AE050E009
:106BE000B8018EE692E10F94F7138EE692E10F94CE
:106BF000BA128091DF0B9091E00B892BE9F040E015
:106C000053E0B701CE0101960E94512D70E060E083
:106C1000C7010E945F3390E080E028960FB6F89499
:106C2000DEBF0FBECDBFDF91CF911F910F91FF90BF
:106C3000EF90DF90CF90089581E090E09093E00B8B
:106C40008093DF0B26E040E855E260E070E082E1EF
:106C50009FE00E9431B9D092121082E19FE09093A0
:106C600011108093101010921D1110921F1110928C
:106C70001E1180ED97E090939810809397101092DA
:106C80009A101092991001151105E1F185E090E03C
:106C900090939C1080939B1086E00F94DE08D82E72
:106CA00064E670E080E090E00F944304D1100AC0E5
:106CB00064E57EE08EE692E10F9406158EE692E1A1
:106CC0000F94BA1282ED97E09093981080939710EA
:106CD00010929A101092991024E6209FC001219FD3
:106CE000900D112490939C1080939B1086E00F943C
:106CF000DE081092E00B1092DF0B882359F0682F0A
:106D000070E086CF10929C1010929B10C5CF8FEF31
:106D10009FEF83CF81E090E080CF2F923F924F9200
:106D20005F926F927F928F929F92AF92BF92CF921B
:106D3000DF92EF92FF920F931F93CF93DF93CDB724
:106D4000DEB72E970FB6F894DEBF0FBECDBF6C0135
:106D500009831A832B833C834D835E836F837887FB
:106D6000CE0101960E9402FA1C01023011F005309A
:106D700011F4312C212CF60102811381F801808558
:106D80008F70853009F043C0C8010E9485FAE82E53
:106D9000F12CF2E0EF16F104D4F160E0C8010E949A
:106DA000F3F9FC01818592859C878B8761E0C8019E
:106DB0000E94F3F9FC0141845284638474848091BD
:106DC000DF0B9091E00B9E878D8788248A94982C06
:106DD00092E0E916F10459F062E0C8010E94F3F96B
:106DE000FC0181849284F3E0EF16F10499F492E0BF
:106DF000A92EB12C8FE390E09A878987ED85FE85D7
:106E0000EF2B49F170E060E0C6010E945F3390E033
:106E100080E035C063E0C8010E94F3F9FC01818580
:106E200092859A87898782E0A82EB12CF4E0EF162C
:106E3000F10439F064E0C8010E94F3F9FC01A18477
:106E4000B28489859A85892BC9F68D859E85892B83
:106E5000C9F671010CC029853A85D1010F94F43728
:106E600024E630E040E050E00F949037790184014F
:106E70009501A2016B857C85C6010E949D332E96EB
:106E80000FB6F894DEBF0FBECDBFDF91CF911F913B
:106E90000F91FF90EF90DF90CF90BF90AF909F90B9
:106EA0008F907F906F905F904F903F902F900895BC
:106EB0000895EF92FF920F931F93CF93DF93EC010E
:106EC0008B011D821C821A821B82E880F980E114EA
:106ED000F10409F45DC08091DA0B9091DB0B892BF2
:106EE00009F456C0672B09F48701F80180858F707B
:106EF0008630A9F46EE778E0C8010E9441F9009756
:106F000019F0FC0181858A836DEE79E0C8010E9449
:106F100041F9009709F443C0FC0181858B8369E73F
:106F200076E0C7010E9441F9009779F565E279E0C2
:106F30008EE692E10F9406154AE050E06B818EE6F2
:106F400092E10F94D01263E279E08EE692E10F9421
:106F500006154AE050E06A818EE692E10F94D01265
:106F60008EE692E10F94BA1220E030E0A90169E7C1
:106F700076E0888199810E9410FD69E776E088813A
:106F800099810E9441F9009719F009969D838C839D
:106F9000DF91CF911F910F91FF90EF900895F8012D
:106FA000808191810F94C32FB9CFAF92BF92CF92BE
:106FB000DF92EF92FF920F931F93CF93DF9364E0E2
:106FC00070E041E050E00091970B1091980B2091F8
:106FD000990B30919A0BCA01052E000CAA0BBB0B22
:106FE00080239123A223B323892B8A2B8B2BD9F0C7
:106FF000C090970BD090980BE090990BF0909A0B63
:10700000CA0180959095092E000CAA0BBB0B8C2110
:107010009D21AE21BF218093970B9093980BA09355
:10702000990BB0939A0B440F551F6150710959F693
:107030008091930B9091940BA091950BB091960B2E
:10704000892B8A2B8B2B09F47DC00F94B4069B01EE
:10705000AC016091930B7091940B8091950B909182
:10706000960BA12CB12C65011CE2E12EFF24F394B8
:1070700000E010E00E9452D3882309F463C010920C
:10708000930B1092940B1092950B1092960B80918B
:10709000D40B9091D50B892B09F183E0E82EF12CCC
:1070A000D0E0C0E0E091D40BF091D50BEE0DFF1DC8
:1070B000008110E0DF0111972C9130E011974C9185
:1070C00050E03397608170E0CE010E94621984E045
:1070D000E80EF11C2196C430D10521F7C1E0D0E0C3
:1070E00080912E0290912F028C179D0748F5809178
:1070F0002E0290912F02E0919A0CF0919B0CE80FD8
:10710000F91F4AE050E060818EE692E10F94D012C0
:107110006CE776E08EE692E10F9410142196C1316F
:10712000D105F1F68EE692E1DF91CF911F910F919B
:10713000FF90EF90DF90CF90BF90AF900D94BA1278
:10714000CE01D9CFDF91CF911F910F91FF90EF909A
:10715000DF90CF90BF90AF900895FC01611571054D
:1071600019F484819581089586819781681779073C
:107170002CF084819581860F971F089582819381D9
:107180000C94A027EF92FF920F931F93CF93DF935E
:10719000DC011296ED91FC91309709F17A018B0197
:1071A000EC0166E376E0808191810E9441F90097CD
:1071B000B1F0FC0120852F70243089F4618572853F
:1071C000E881F9810288F389E02D9701A801CE01B9
:1071D000DF91CF911F910F91FF90EF90199490E064
:1071E00080E0DF91CF911F910F91FF90EF90089574
:1071F000EF92FF920F931F93CF93DF93CDB7DEB73C
:1072000060970FB6F894DEBF0FBECDBF8C01790139
:10721000CE0101960E9455DAA701BE016F5F7F4F34
:10722000C8010E94C23860960FB6F894DEBF0FBE48
:10723000CDBFDF91CF911F910F91FF90EF900895F7
:107240002F923F924F925F926F927F928F929F9276
:10725000AF92BF92CF92DF92EF92FF920F931F9364
:10726000CF93DF93CDB7DEB7A6970FB6F894DEBF06
:107270000FBECDBF1C010F8B188F298F3A8F4B8FFC
:107280005C8F6D8F7E8F22E1E216F10408F035C02D
:10729000F701E65EFA4F30813F8FCE0147960E949C
:1072A000692197FD04C0BC01C1010E94FA23988D99
:1072B000892F8F70D1011196EC911197E07FE82B07
:1072C0001196EC9311978F898C93E295EF70EC30C7
:1072D00008F063C0F0E08827EF58F64C8F4F0D940C
:1072E000E537743B9A399A39123B7F39A03BDB3A38
:1072F0001C3B1C3B1C3BDB3ADB3A1F8ECECFB12C38
:1073000092959F709D3008F0CDC4E92FF0E088275A
:10731000E357F64C8F4F0D94E537CD39DA3BFA3B06
:10732000DA3BA33BA33BDA3BDA3B523E523EDA3B2D
:10733000DA3BA73A92959F709D3008F018C1E92F6B
:10734000F0E08827E955F64C8F4F0D94E537CD399D
:10735000853A783A3B3AB739B4395C3A873AB73A22
:10736000B73A463A463AA73A8E8DF10187838D8D1A
:10737000D10116968C9316978C8D15968C93159734
:107380008B8D14968C9314979295907F11968C9177
:1073900011978F70982B11969C93BF8DBB2309F486
:1073A00067C0F101818182958F702B2F30E08217A9
:1073B000130609F45DC068EA7EE08EE692E10F9460
:1073C0000615D10111966C9162956F704AE050E0FC
:1073D0008EE692E10F94D01265EA7EE08EE692E1AD
:1073E0000F9406154AE050E06F8D8EE692E10F94FF
:1073F000D01263EA7EE08EE692E10F940615F10169
:10740000008119821A821B821C821D821E821F82A9
:1074100018868F8D8295807F9A819F70892B8A83B1
:107420000983EE24EA94FE2C118122813381448168
:10743000558166817781CE0101960E942039D10164
:107440002C9311963C93119712964C931297139686
:107450005C93139714966C93149715967C931597D9
:1074600016968C93169717969C93C1010E94AC2395
:1074700088E0F10178C18D8D9E8DF1018683878131
:1074800090FB80F987838C8D858387CF8B8D9C8D36
:10749000AD8DBE8DB7FD0EC08F3F9105A105B10525
:1074A00029F024F08FEF90E0A0E0B0E0D101149635
:1074B0008C9373CF80E0FACF6B8D7C8D8D8D9E8DFC
:1074C00020E06D39BFEF7B078B079B076CF02FEF38
:1074D0006115E4E67E078105910534F424E630E089
:1074E00040E050E00F949037D10114962C9355CF83
:1074F0008D8D9E8DF1018683878190FB80F9878336
:107500008C8D85838B8D848348CF8B8DCFCFCB8C17
:10751000DC8CED8CFE8C20E030E0A901C701B601C7
:107520000F94243660E087FD0FC020E030E04FE785
:1075300053E4C701B6010F942C396FEF181624F0ED
:10754000C701B6010F94FD38F101648326CFD10144
:1075500011968C9111978F70806C11968C93119766
:107560008B8D9C8D15969C938E93149716CF68E205
:107570007FE08EE692E10F940615688D62956F703C
:107580004AE050E08EE692E10F94D01265E27FE08F
:107590008EE692E10F940615F101618162956F709C
:1075A0004AE050E08EE692E10F94D0128EE692E12E
:1075B0000F94BA12F2CE92959F70933091F09C3056
:1075C00031F24B8D5C8D6D8D7E8DF1014483558341
:1075D000668377839295907F81818F70982B9183BA
:1075E000DCCE60E0C1010E94091ED10114968C938B
:1075F00014978D8D9E8D16968C93169717968C9159
:10760000179790FB80F917968C9317978C8D15968A
:107610008C93159711968C9111978F7080621196AB
:107620008C93BBCE60E0CE0147960E94091ED1012B
:1076300014968C931497EECF92959F709D3008F01E
:1076400066C0E92FF0E08827E75DF44C8F4F0D947A
:10765000E537CD39443B733BF13A733B733B363BE3
:10766000633B633B633B523B5E3BA73A8B8D9C8DF8
:10767000AD8DBE8DF10184839583A683B78381810F
:107680008F708066818389CE6B8D70E090E080E0A2
:107690000F942936D10114966D937D938D939C930D
:1076A00017977BCE6B8D7C8D8D8D9E8D0F942B3699
:1076B000F10164837583868397836FCE6B8D7C8D98
:1076C0008D8D9E8DE5CF9295907FF10181818F7098
:1076D000982B91838B8D9C8DAD8DBE8D84839583EE
:1076E000A683B7835ACE9295907FD10111968C9143
:1076F00011978F70982B11969C938B8D9C8DAD8DCF
:10770000BE8DF10184839583A683B78346CE63E162
:107710007FE08EE692E10F940615688D62956F709A
:107720004AE050E08EE692E10F94D01260E17FE0F3
:107730008EE692E10F940615D10111966C912ECF31
:10774000BB24B394DDCD4B8D5C8D6D8D7E8DF101B1
:1077500044835583668377839295907F81818F7070
:10776000982B918388E0DE01119601900D928A9505
:10777000E1F729813A814B815C816D817E818F8126
:107780009885A6960FB6F894DEBF0FBECDBFDF91E9
:10779000CF911F910F91FF90EF90DF90CF90BF900E
:1077A000AF909F908F907F906F905F904F903F90A1
:1077B0002F900895963009F442C148F46B8D9130B2
:1077C00071F06FEF70E0933051F060E008C09730D7
:1077D00009F441C19A506B8D7C8D9230B0F784E6EC
:1077E0008D8F8E8D8E7F8E8F1C8E888D8F70806298
:1077F000888F6B8F2C8D30E0AFEFB0E00F94C237E5
:10780000C12CD12C7601CA946115F4E67F0781055D
:10781000910544F424E630E040E050E00F949037C6
:1078200069017A0186012B8D28A3622E712CBB2061
:1078300009F475C08E8D8695A82FA150BB0B2D0124
:10784000BFEF4B165B0609F027C1003811050CF09D
:1078500009C18FE790E08C199D09869DD001879D15
:10786000B00D969DB00D11242FEF30E00F94FC3732
:1078700021E83EE740E050E00F949037F101278384
:10788000ABE9B0E0A70196010F94AF37EFE78E2E7A
:10789000912CA12CB12CA50194010F949037890152
:1078A0009A010C591F4F2F4F3F4FAEEFB1E0A70188
:1078B00096010F94AF37A50194010F949037D3012F
:1078C0000F94AF372FEF30E040E050E00F94903747
:1078D00039012FEF6216710421F01CF066246A94BE
:1078E000712C63E07FE08EE692E10F9406154AE08A
:1078F00050E0B8018EE692E10F94F71365EF7EE059
:107900008EE692E10F9406154AE050E0B3018EE650
:1079100092E10F94F7138EE692E10F94BA1230E0E1
:1079200020E050E040E070E060E0CE0101960E946F
:1079300093B9F02E2D8D3E8D3170AFEFBFEF0F94C8
:10794000C2372DE631E040E050E00F9490374427F5
:107950005527AAEFB5E00F94AF37DC01CB01905863
:10796000AF4FBF4FCD01BB2797FDB095AB2F8E3FDB
:10797000E1E09E0708F06FC1382F8F3F910508F4B2
:107980008CC14EEF481B50E03FEFF30131961127B9
:107990000F5F1F4FF094EF2CF12C309FC001319FEF
:1079A000900D1124292F33272E0D3F1DDF010F9439
:1079B000FC374B015C018824AA24BB24509F900112
:1079C000519F300D1124232F33272E0D3F1D0F946F
:1079D000FC37BB27A92F982F872F882A992AAA2AF4
:1079E000409F9001419F300D1124232F33272E0DEE
:1079F0003F1DDF010F94FC37B82FA72F962F882744
:107A000088279927BB2788299929AA29F101A683C4
:107A10009583848369EC7EE08EE692E10F940615EF
:107A2000C1010E94AC238A859B850F94922E8F8181
:107A3000988597FDB2CC60E00F94FE01AECC6B8DC3
:107A40007C8D8D8D9E8D24E630E040E050E00F94DB
:107A50009037B901C4CE6B8D7C8D8D8D9E8D0F942A
:107A6000F638BDCEA70196012058310941095109C8
:107A7000ABE9B0E00F94AF372FE730E040E050E0E3
:107A80000F94903789019A010C591F4F2F4F3F4F88
:107A9000D10117961C9225CF9201AAEBBFEF0F944C
:107AA000F43744E6842E912CA12CB12CA50194012D
:107AB0000F949037DA01C9018C599F4FAF4FBF4FD8
:107AC00089A39AA3ABA3BCA326E430E0D2010F9410
:107AD000FC37A50194010F94903749015A019EE1AA
:107AE000890E911CA11CB11C003811050CF099C025
:107AF0008FE790E08C199D09869DD001879DB00D80
:107B0000969DB00D1124A50194010F94BA379B01E5
:107B1000AC01AFEFB0E00F94AF3724E63AE640E0B7
:107B200050E00F949037D10117962C9329A13AA1D8
:107B30004BA15CA12C0D3D1D4E1D5F1DAEEFB1E0B4
:107B40000F94AF3723EE30E040E050E00F949037D1
:107B500029013A013EA32DA3AFEFB0E0A7019601A2
:107B60000F94AF372FE730E040E050E00F949037AC
:107B70008901E8A1AE2FB0E0A30192010F94AF37C5
:107B80002FEF30E040E050E00F94903739012F3F65
:107B9000310521F01CF066246A94712C6FEE7EE0B2
:107BA0008EE692E10F9406152AE030E049A15AA131
:107BB0006BA17CA18EE692E10F94AF1369EE7EE09B
:107BC0008EE692E10F9406152AE030E0B501A4019B
:107BD0008EE692E10F94AF1361EE7EE08EE692E1C5
:107BE0000F9406154AE050E0B8018EE692E10F943A
:107BF000F71369ED7EE08EE692E10F9406154AE0F8
:107C000050E0B3018EE692E10F94F71360ED7EE051
:107C10008EE692E10F9406154AE050E06DA17EA138
:107C200076CEA70196012058310941095109ABE9E7
:107C3000B0E00F94AF372FE730E040E050E00F9412
:107C4000903789019A010C591F4F2F4F3F4FD10197
:107C500017961C92A3CF8C3FF3E09F0768F48D3FEB
:107C600022E0920728F452E0580F3FEF40E08DCE1B
:107C70003CEF381B5FEFFACF8A3F35E0930781F086
:107C80008B3FE4E09E0728F444E0480F5FEF30E0CC
:107C90007CCE5AEF581B30E001C050E04FEF75CE5C
:107CA00050E0F9CF67EB7EE08EE692E10F94061587
:107CB000688D62956F704AE050E08EE692E10F9415
:107CC000D01264EB7EE034CD2F923F924F925F92C0
:107CD0006F927F928F929F92AF92BF92CF92DF92DC
:107CE000EF92FF920F931F93CF93DF93CDB7DEB741
:107CF000C25CD1090FB6F894DEBF0FBECDBF1C0128
:107D0000C755DF4F0883C95AD040C655DF4F188387
:107D1000CA5AD040C555DF4F2883CB5AD040C455EE
:107D2000DF4F3883CC5AD040C355DF4F4883CD5AFC
:107D3000D040C255DF4F5883CE5AD040C155DF4F97
:107D40006883CF5AD040C055DF4F7883C05BD040A6
:107D5000CF54DF4FF982E882C15BD040CD54DF4F72
:107D6000C882C35BD0400E94AEDA6B01C954DF4FBA
:107D700079836883C75BD040683C7105B4F46BE8D5
:107D80007CE087EC91E10F9406154AE050E0B601E3
:107D900087EC91E10F94F71387EC91E10F94BA12FD
:107DA000CC24CA94DC2C0C9467480F94B406C154BC
:107DB000DF4F688379838A839B83CF5BD040C6552E
:107DC000DF4F8881CA5AD0408F70482E512C2091A5
:107DD000F70D3091F80DC354DF4F39832883CD5B05
:107DE000D040CF54DF4FE881F981C15BD04030975C
:107DF00021F0808181110C94A24FD1011B968C91AE
:107E0000882341F0C1010B96CF54DF4F99838883BB
:107E1000C15BD0404114510411F00C94EB4FCF548E
:107E2000DF4FE881F981C15BD040309711F00C94AD
:107E3000A64FF101438C548C4114510411F40C945D
:107E4000EB4FC655DF4F8881CA5AD0408F7011F072
:107E50000C94EB4F642DCE0187559F4F0E94231B3E
:107E6000C756DF4F2883C959D040C656DF4F3883E5
:107E7000CA59D040C556DF4F4883CB59D040C4566D
:107E8000DF4F5883CC59D040C356DF4F6883CD595C
:107E9000D040C256DF4F7883CE59D040C156DF4F15
:107EA0008883CF59D040C056DF4F9883C05AD04006
:107EB0000C94EB4FD1018D919C91892B09F470CFDB
:107EC000B4E04B16510471F5C755DF4F0881C95A0C
:107ED000D040C655DF4F1881CA5AD040C555DF4F34
:107EE0002881CB5AD040C455DF4F3881CC5AD0407E
:107EF000C355DF4F4881CD5AD040C255DF4F58811E
:107F0000CE5AD040C155DF4F6881CF5AD040C055BE
:107F1000DF4F7881C05BD040C1010E94B61F6C0169
:107F20000C946748C755DF4F1881C95AD0401430A8
:107F300009F412C330F4112309F49AC0B12CA12C16
:107F4000C8C288EF810F8230C8F788E0FE01E7558C
:107F5000FF4FDE01119601900D928A95E1F7C6550B
:107F6000DF4F8881CA5AD040807F09F448C3CE01D0
:107F700087559F4F0E941D216B017C01C114D104C4
:107F8000E104F10409F43BC3193041F4F094E094A6
:107F9000D094C094C11CD11CE11CF11CB101CE01D4
:107FA00087559F4F0F94BF1660E0CE0187559F4FB6
:107FB0000E944A1B6A962FAF6A976B963FAF6B97EA
:107FC0006C964FAF6C976D965FAF6D976E966FAF77
:107FD0006E976F967FAF6F97A0968FAFA097A19681
:107FE0009FAFA19712E04116510409F45FC30CF052
:107FF0000CC3662463944114510409F09FCFD1014E
:1080000019968D919C911A97009709F051C3189673
:108010008C9190E0F0E58F2E912CA12CB12C853025
:10802000910549F0812C912C5401449721F0812C29
:10803000912C54018A94C655DF4FE881CA5AD0402A
:10804000E295EF70E150EB3008F063C4F0E0882770
:10805000E35DFF4B8F4F0D94E537604360438944E8
:108060008944894456441444144414448E438E4332
:1080700019821A821B821C821D821E821F82188610
:108080008A818F708A83C655DF4F8881CA5AD04053
:10809000807F09F453CF0AE04016510409F41BC253
:1080A0000CF0F3C04114510409F413C122E042164C
:1080B000510409F043CFB12CA12C612C77247A9480
:1080C000B101CE0101960F94BF168A81982F929527
:1080D0009F70945F9F70923060F4C655DF4F988117
:1080E000CA5AD04092959F70923019F48F70806276
:1080F0008A83D10118969C91973071F4C655DF4F51
:108100008881CA5AD040807E803211F0803421F4B8
:108110008A818F7080628A83F101A185B285892F5F
:1081200090E0109741F0ED91FC911197048CF58D42
:10813000E02DCD0119957C01C755DF4F0881C95A43
:10814000D040C655DF4F1881CA5AD040C555DF4FC1
:108150002881CB5AD040C455DF4F3881CC5AD0400B
:10816000C355DF4F4881CD5AD040C255DF4F5881AB
:10817000CE5AD040C155DF4F6881CF5AD040C0554C
:10818000DF4F7881C05BD040CE0101960E9420393C
:10819000CF57DF4F2883C158D040CE57DF4F3883A9
:1081A000C258D040CD57DF4F4883C358D040CC573A
:1081B000DF4F5883C458D040CB57DF4F6883C55832
:1081C000D040CA57DF4F7883C658D040C957DF4FD9
:1081D0008883C758D040C857DF4F9883C858D040CD
:1081E000CE0101960E94AC23662051F1C655DF4FA7
:1081F0008881CA5AD04082958F709FE0980F9F70F7
:10820000923020F08A5F8F708230D0F48A8182951C
:108210008F7081508230A0F42D8130E0AFEFB0E05C
:108220000F94C2372FEF6115F4E67F0781059105A2
:1082300034F424E630E040E050E00F9490372D8392
:1082400088E0FE013196DE01A755BF4F01900D92E7
:108250008A95E1F702E1B02A812CD10118968C9120
:108260001897873009F065C6C954DF4FE881F98156
:10827000C75BD040EE35F1400CF0C0C36CE17CE050
:1082800087EC91E10F94061587CD3BE0431651042E
:1082900009F4CFC08CE04816510409F04FCEB1016B
:1082A000CE0101960F94BF16CE0187559F4F0E94B5
:1082B0006921BC01CE0101960E94FA2388E0FE01EB
:1082C0003196DE01A755BF4F01900D928A95E1F7D7
:1082D000FDC0EF2B59F068E47CE08EE692E10F944C
:1082E00006158EE692E10F94BA1228CEC1010E94C3
:1082F00001518C0161E070E01816190614F070E06D
:1083000060E04AE050E08EE692E10F94F71369E1F5
:1083100077E08EE692E10F941014CE0187559F4FBF
:108320000E94711FAB01BC012AE030E08EE692E1B1
:108330000F94AF138EE692E10F94BA12CE018755D7
:108340009F4F1016110614F00C94964F0E94711F47
:10835000B12CA12C672B682B692B89F562E0CE012B
:1083600087559F4F0E944A1BCF56DF4F2883C15924
:10837000D040CE56DF4F3883C259D040CD56DF4F64
:108380004883C359D040CC56DF4F5883C459D0409E
:10839000CB56DF4F6883C559D040CA56DF4F78832C
:1083A000C659D040C956DF4F8883C759D040C856F8
:1083B000DF4F9883C859D040AA24A394BA2C6624CE
:1083C0006394772473947CCE61E0CE0187559F4FF0
:1083D0000E944A1BC757DF4F2883C958D040C65751
:1083E000DF4F3883CA58D040C557DF4F4883CB583A
:1083F000D040C457DF4F5883CC58D040C357DF4FCD
:108400006883CD58D040C257DF4F7883CE58D040D4
:10841000C157DF4F8883CF58D040C057DF4F988374
:10842000C059D040AA24A394BA2C66246394712C1A
:1084300047CEB101CE0101960F94BF16C255DF4F52
:108440008881CE5AD0409A8192959F7041F09230A7
:1084500051F0B12CA12C88248394612C5CC19A81A9
:108460009F7090629A8390E08536910514F084E6BF
:1084700090E08E8388E0FE013196DE01A755BF4F64
:1084800001900D928A95E1F762E0CE0187559F4FEA
:108490000E94231BEA962FAFEA97EB963FAFEB972C
:1084A000EC964FAFEC97ED965FAFED97EE966FAF12
:1084B000EE97EF967FAFEF97C158DF4F8883CF5786
:1084C000D040C058DF4F9883C058D040A12C82E1E3
:1084D000B82E812CC2CFB101CE0101960F94BF16E8
:1084E000C155DF4F6881CF5AD040C055DF4F7881EA
:1084F000C05BD0407170CE0101960E943524682E79
:10850000882309F410C288E0FE013196DE01A755E8
:10851000BF4F01900D928A95E1F762E0CE01875539
:108520009F4F0E94231BE2962FAFE297E3963FAF47
:10853000E397E4964FAFE497E5965FAFE597E6964D
:108540006FAFE697E7967FAFE797E8968FAFE8972C
:10855000E9969FAFE997BACFC1010E940151181661
:1085600019063CF562E0CE0187559F4F0E944A1BD9
:10857000AA962FAFAA97AB963FAFAB97AC964FAFEB
:10858000AC97AD965FAFAD97AE966FAFAE97AF9627
:108590007FAFAF97E0968FAFE097E1969FAFE197FF
:1085A000AA24A394BA2C812C662463947724739410
:1085B00054CE61E0CE0187559F4F0E944A1BA29680
:1085C0002FAFA297A3963FAFA397A4964FAFA497C0
:1085D000A5965FAFA597A6966FAFA697A7967FAF14
:1085E000A797A8968FAFA897A9969FAFA997AA24F7
:1085F000A394BA2C812C66246394712C2ECEB5E002
:10860000CB2ED12CE12CF12CBFCC3AE043165104F7
:1086100009F48EC18BE04816510409F08FCCC65581
:10862000DF4F8881CA5AD04082958F70823009F01E
:10863000DAC1C701B60124E630E040E050E00F9413
:108640009037C255DF4F8881CE5AD04090E0280F36
:10865000391F37FF02C030E020E02536310514F025
:1086600024E630E0C255DF4F2883CE5AD04062E086
:10867000CE0187559F4F0E94231B2A962FAF2A9722
:108680002B963FAF2B972C964FAF2C972D965FAF25
:108690002D972E966FAF2E972F967FAF2F976096C0
:1086A0008FAF609761969FAF619710CF612CA7CC79
:1086B000DC01ED91FC91048CF58DE02D1995AACC8F
:1086C000C355DF4F1881CD5AD040C701B60124E60B
:1086D00030E040E050E00F949037DA01C901810F9B
:1086E000911DA11DB11DB7FF03C080E090E0DC012A
:1086F0008F3F9105A105B10529F024F08FEF90E09F
:10870000A0E0B0E0C355DF4F8883CD5AD040A12C04
:10871000E2E1BE2E812C77247A949FCDC355DF4FA2
:10872000088119812A813B81CD5AD040C754DF4F3F
:10873000088319832A833B83C95BD04014E6C116A2
:10874000D104E104F1040CF041C0A4E6B0E0C75448
:10875000DF4F288139814A815B81C95BD0400F940A
:10876000AF37C60ED71EE81EF91E81149104A1046E
:10877000B104B9F0A50194010F94AF37362F272F1C
:10878000B701A60177FF03C040E050E0BA01C32E55
:10879000D22E7C014C155D056E057F0514F46A012F
:1087A0007B01C355DF4FC882D982EA82FB82CD5A52
:1087B000D040C655DF4F8881CA5AD0408F7080663E
:1087C000C655DF4F8883CA5AD040A1CFC701B60132
:1087D00024E630E040E050E00F949037C754DF4F7C
:1087E00088819981AA81BB81C95BD040280F391F3C
:1087F0004A1F5B1F81149104A104B10461F057FF6B
:1088000003C020E030E0A90182169306A406B50655
:1088100014F4A5019401C355DF4F288339834A839B
:108820005B83CD5AD04073CFC355DF4F68817981C8
:108830008A819B81CD5AD0400F94F638C754DF4FC0
:10884000688379838A839B83C95BD040C701B60163
:1088500024E630E040E050E00F949037C754DF4FFB
:10886000688179818A819B81C95BD040620F731FC7
:10887000841F951F81149104A104B10461F097FF36
:1088800003C060E070E0CB0186169706A806B90623
:1088900014F4C501B4010F942B36C355DF4F688320
:1088A00079838A839B83CD5AD04031CFC355DF4F24
:1088B00088819981AA81BB81CD5AD040C80ED91E2A
:1088C000EA1EFB1E81149104A104B104C9F0A4E6C0
:1088D000B0E0A50194010F94AF37362F272FB701D1
:1088E000A60177FF03C040E050E0BA01C32ED22EAC
:1088F0007C014C155D056E057F0514F46A017B0152
:10890000C355DF4FC882D982EA82FB82CD5AD0405C
:10891000FECE88E0FE013196DE01A755BF4F0190E3
:108920000D928A95E1F7B12CA12C88248394F3CE83
:10893000C655DF4F8881CA5AD04082958F708230E9
:1089400009F051C0C701B60124E630E040E050E034
:108950000F949037C155DF4F8881CF5AD040C05512
:10896000DF4F6881C05BD040962F9170280F391F70
:108970002E3691E039072CF437FF05C02DE631E0A3
:1089800002C030E020E0C155DF4F2883CF5AD040ED
:10899000C055DF4F8881C05BD04030FB80F9C055A7
:1089A000DF4F8883C05BD04062E0CE0187559F4F88
:1089B0000E94231B62962FAF629763963FAF639727
:1089C00064964FAF649765965FAF659766966FAF95
:1089D000669767967FAF679768968FAF6897699637
:1089E0009FAF699773CD88E0FE013196DE01A755F0
:1089F000BF4F01900D928A95E1F72BCDCD54DF4FFB
:108A00001881C35BD040112339F11296ED91FC918E
:108A100080858F70853001F5C354DF4FE881F9817F
:108A2000CD5BD0403597C1F0C1010E940151772440
:108A30007394181619060CF0712CCF54DF4F48812F
:108A40005981C15BD040BE0167557F4FD10112965D
:108A50008D919C910E944150C755DF4F8881C95A22
:108A6000D040853009F4F7C128F4833009F46EC092
:108A7000C501EBC0863009F4FDC08730C9F7C101DC
:108A80000E94032E182F863009F0E1C0E1E04E1657
:108A90005104C9F5C655DF4F8881CA5AD040807F3E
:108AA00091F1711005C0C1010E948216892B59F104
:108AB000C755DF4F0881C95AD040C655DF4F1881CE
:108AC000CA5AD040C555DF4F2881CB5AD040C45533
:108AD000DF4F3881CC5AD040C355DF4F4881CD5A43
:108AE000D040C255DF4F5881CE5AD040C155DF4FDC
:108AF0006881CF5AD040C055DF4F7881C05BD040ED
:108B0000C1010E94632060EF7BE08EE692E10F944A
:108B100006154AE050E066E070E08EE692E10F94C0
:108B2000F7138EE692E10F94BA1262E0CE018755F8
:108B30009F4F0E944A1B29AF3AAF4BAF5CAF6DAF5E
:108B40007EAF8FAF21969FAF21977CC0C1010E945D
:108B5000032E853021F093E0C92ED12CB8C2B1E0AC
:108B60004B165104C9F5C655DF4F8881CA5AD0400B
:108B7000807F91F1772029F0C1010E948216892B14
:108B800059F1C755DF4F0881C95AD040C655DF4F4C
:108B90001881CA5AD040C555DF4F2881CB5AD040E2
:108BA000C455DF4F3881CC5AD040C355DF4F488180
:108BB000CD5AD040C255DF4F5881CE5AD040C15512
:108BC000DF4F6881CF5AD040C055DF4F7881C05BFE
:108BD000D040C1010E94632067E07CE08EE692E114
:108BE0000F9406154AE050E065E070E08EE692E1F1
:108BF0000F94F7138EE692E10F94BA12B101CE01F1
:108C000087559F4F0F94BF1661E0CE0187559F4F48
:108C10000E944A1B22962FAF229723963FAF23979D
:108C200024964FAF249725965FAF259726966FAF72
:108C3000269727967FAF279728968FAF2897299654
:108C40009FAF2997C50181609160912C84C062ED2E
:108C50007BE08EE692E10F940615612F70E04AE00A
:108C600050E08EE692E10F94F7138EE692E10F94B6
:108C7000BA1271CF40E050E061E070E0C1010E94A3
:108C8000E729672B682B692B09F0E2C0FFEF7F1201
:108C900009C0C1010E940151772473941816190666
:108CA0000CF0712C01E040165104D1F5C655DF4F90
:108CB0008881CA5AD040807F99F1772031F0C10174
:108CC0000E948216892B09F4BCC0C755DF4F08816A
:108CD000C95AD040C655DF4F1881CA5AD040C55531
:108CE000DF4F2881CB5AD040C455DF4F3881CC5A52
:108CF000D040C355DF4F4881CD5AD040C255DF4FD9
:108D00005881CE5AD040C155DF4F6881CF5AD040EC
:108D1000C055DF4F7881C05BD040C1010E94632005
:108D200071108FC0B101CE0187559F4F0F94BF16B0
:108D300061E0CE0187559F4F0E944A1B29AB3AAB99
:108D40004BAB5CAB6DAB7EAB8FAB98AFC5018160BD
:108D5000916076E0972E5C016894A0F8C655DF4FCD
:108D60002881CA5AD040322F3F70323058F4C7554C
:108D7000DF4F3881C95AD040332321F05C01689419
:108D8000A0F8B0F8207F09F4C9C06894B1F8CD54B8
:108D9000DF4F6882C35BD040CC24C394D12C8110B8
:108DA0000C943B50D10119968D919C91009709F03C
:108DB00037C640E050E062E070E0C1010E94E72960
:108DC000672B682B692B09F45DC664E77AE087ECB2
:108DD00091E10F94061587EC91E10F94BA12B2FE5F
:108DE00002C00C94804F69E57AE08EE692E10F9420
:108DF00006154AE050E0B6018EE692E10F94F713B3
:108E000062E57AE08EE692E10F9406150F94B406BF
:108E1000AB01BC01C154DF4F088119812A813B811C
:108E2000CF5BD040401B510B620B730B2AE030E04C
:108E30008EE692E10F94B8128EE692E10F94BA1288
:108E400046C168EB7BE08EE692E10F94061583CE77
:108E500063EA7BE0F8CF1FEF711209C0C1010E94E5
:108E6000015177247394181619060CF0712C21E027
:108E700042165104D1F5C655DF4F8881CA5AD040F9
:108E8000807F99F1711006C0C1010E948216892B62
:108E900009F441C0C755DF4F0881C95AD040C655B3
:108EA000DF4F1881CA5AD040C555DF4F2881CB5AB1
:108EB000D040C455DF4F3881CC5AD040C355DF4F26
:108EC0004881CD5AD040C255DF4F5881CE5AD0404C
:108ED000C155DF4F6881CF5AD040C055DF4F7881F0
:108EE000C05BD040C1010E9463207720A1F062E006
:108EF000CE0187559F4F0E944A1B29A73AA74BA72F
:108F00005CA76DA77EA78FA798ABC5018160916014
:108F100065E0962E20CF66E87BE095CF40E052E0FA
:108F2000B101CE0187559F4F0E94102E81112DCF88
:108F30002ECF3FEF731298C0C1010E9401517724D8
:108F40007394181619060CF492C0712C68E77BE034
:108F50008EE692E10F940615072D072C000C110BDD
:108F6000C954DF4F19830883C75BD0404AE050E003
:108F7000B8018EE692E10F94F71361E77BE08EE68D
:108F800092E10F940615662D70E04AE050E08EE6FF
:108F900092E10F94F7138EE692E10F94BA12CF5438
:108FA000DF4FE880F980C15BD040E114F10409F49F
:108FB000B3C06FE37EE0C7010F942F30CC24C3947D
:108FC000D12C892B09F459C06BE37EE0C7010F94C3
:108FD0002F3032E0C32ED12C892B09F44EC06DE422
:108FE0007AE0C7010F942F3025E0C22ED12C892BB7
:108FF00009F443C069E47AE0C7010F942F30892B4C
:10900000C9F160E07EE0C7010F942F30892B09F48D
:1090100079C06BEF7DE0C7010F942F3004E1C02EC3
:10902000D12C892B51F165E07EE0C7010F942F30E0
:109030001EE0C12ED12C892B01F16EEE7DE0C7011F
:109040000F942F30BFE0CB2ED12C892BB1F067EFDE
:109050007DE0C7010F942F30D12CC12C892B69F4EE
:10906000A5E1CA2ED12C09C0772009F46FCF662460
:1090700063946CCF96E0C92ED12CC1010E94032EBF
:10908000082F10E00115110531F4C954DF4F088194
:109090001981C75BD040C114D10409F462C00C151A
:1090A0001D05A1F165E57BE08EE692E10F940615C2
:1090B0004AE050E0B8018EE692E10F94F7138EE695
:1090C00092E10F94BA12FDEFCF2EDD24DA94C6019F
:1090D000CE53DF4F0FB6F894DEBF0FBECDBFDF918A
:1090E000CF911F910F91FF90EF90DF90CF90BF90A5
:1090F000AF909F908F907F906F905F904F903F9038
:109100002F90089583E1C82ED12CB7CFCF54DF4FD5
:1091100019821882C15BD040C755DF4FE881C95A18
:10912000D040E63108F033C4F0E08827E556F74B2D
:109130008F4F0D94E537DE4C4B4BED4AEA48DE4C41
:10914000854A014A7D49DE4CDE4CD44BFA4B474CF4
:10915000744CB44BB44BC74CC74CC74CB44BB44B1A
:10916000B44BD10119968D919C91009709F4AFCF22
:10917000DC01ED91FC910488F589E02DC62CC755E2
:10918000DF4F0881C95AD040C655DF4F1881CA5AEF
:10919000D040C555DF4F2881CB5AD040C455DF4F52
:1091A0003881CC5AD040C355DF4F4881CD5AD0408A
:1091B000C255DF4F5881CE5AD040C155DF4F68812C
:1091C000CF5AD040C055DF4F7881C05BD040199551
:1091D0000C948F3FC1010E94032E853009F0BBCC57
:1091E000B1E04B16510409F040C0CD54DF4FE88187
:1091F000C35BD040EE23C9F1C655DF4F8881CA5A00
:10920000D040807F91F1711005C0C1010E9482168B
:10921000892B59F1C755DF4F0881C95AD040C6552F
:10922000DF4F1881CA5AD040C555DF4F2881CB5A2D
:10923000D040C455DF4F3881CC5AD040C355DF4FA2
:109240004881CD5AD040C255DF4F5881CE5AD040C8
:10925000C155DF4F6881CF5AD040C055DF4F78816C
:10926000C05BD040C1010E94632060E47BE08EE6D9
:1092700092E10F9406154AE050E065E070E08EE65A
:1092800092E10F94F7138EE692E10F94BA12B101B6
:10929000CE0187559F4F0F94BF16D10118968C9120
:1092A0008530E1F46EE0CE0187559F4F0E944A1B46
:1092B00029A33AA34BA35CA36DA37EA38FA398A776
:1092C0006894A0F8B0F8912CCC24CA94DC2CB1E0BE
:1092D000CD54DF4FB883C35BD04061CD61E0CE0198
:1092E00087559F4F0E944A1B298F3A8F4B8F5C8F67
:1092F0006D8F7E8F8F8F98A3E3CFC1010E94032EC5
:10930000182F863009F07AC0E1E04E16510409F0BA
:1093100040C0CD54DF4FF881C35BD040FF23C9F17B
:10932000C655DF4F8881CA5AD040807F91F17110B5
:1093300005C0C1010E948216892B59F1C755DF4F24
:109340000881C95AD040C655DF4F1881CA5AD0404B
:10935000C555DF4F2881CB5AD040C455DF4F3881E7
:10936000CC5AD040C355DF4F4881CD5AD040C2556A
:10937000DF4F5881CE5AD040C155DF4F6881CF5A58
:10938000D040C055DF4F7881C05BD040C1010E9402
:10939000632069E27BE08EE692E10F9406154AE0D5
:1093A00050E066E070E08EE692E10F94F7138EE6EF
:1093B00092E10F94BA1262E0CE0187559F4F0E944E
:1093C0004A1B298B3A8B4B8B5C8B6D8B7E8B8F8BE7
:1093D000988F40E050E068E070E0C1010E9495295C
:1093E0006894A0F8B0F8912CCC24CA94DC2C01E04D
:1093F000CD54DF4F0883C35BD040D1CC6BE07BE022
:1094000028CC40E050E061E070E0C1010E94E72913
:10941000672B682B692B09F075C011E041165104C8
:1094200009F041C0CD54DF4F2881C35BD0402223D7
:10943000D1F1C655DF4F8881CA5AD040807F99F15B
:10944000772031F0C1010E948216892B09F457C0A0
:10945000C755DF4F0881C95AD040C655DF4F188124
:10946000CA5AD040C555DF4F2881CB5AD040C45589
:10947000DF4F3881CC5AD040C355DF4F4881CD5A99
:10948000D040C255DF4F5881CE5AD040C155DF4F32
:109490006881CF5AD040C055DF4F7881C05BD04043
:1094A000C1010E94632071102AC0B101CE0187550D
:1094B0009F4F0F94BF1661E0CE0187559F4F0E94CA
:1094C0004A1B29873A874B875C876D877E878F8702
:1094D000988B40E050E068E070E0C1010E94BE2936
:1094E0006894A0F8B0F8E6E09E2ECC24CA94DC2C58
:1094F00031E0CD54DF4F3883C35BD04050CC61EFB7
:109500007AE0A1CC6CED7AE09ECC81E04816510463
:1095100009F041C0CD54DF4F9881C35BD0409923FF
:10952000D1F1C655DF4F8881CA5AD040807F99F16A
:10953000711006C0C1010E948216892B09F44AC02D
:10954000C755DF4F0881C95AD040C655DF4F188133
:10955000CA5AD040C555DF4F2881CB5AD040C45598
:10956000DF4F3881CC5AD040C355DF4F4881CD5AA8
:10957000D040C255DF4F5881CE5AD040C155DF4F41
:109580006881CF5AD040C055DF4F7881C05BD04052
:10959000C1010E9463207720E9F062E0CE01875587
:1095A0009F4F0E944A1B29833A834B835C836D83C0
:1095B0007E838F8398876894A0F8B0F875E0972E23
:1095C000CC24CA94DC2CA1E0CD54DF4FA883C35B2C
:1095D000D040E5CB6FEB7AE036CCC655DF4F188133
:1095E000CA5AD040812F8F70912C823008F004C26B
:1095F000C1010E94032E853009F4ADCAB1E04B16BB
:109600005104D9F5CD54DF4FE881C35BD040EE2340
:10961000A1F1107F91F1711005C0C1010E94821665
:10962000892B59F1C755DF4F0881C95AD040C6551B
:10963000DF4F1881CA5AD040C555DF4F2881CB5A19
:10964000D040C455DF4F3881CC5AD040C355DF4F8E
:109650004881CD5AD040C255DF4F5881CE5AD040B4
:10966000C155DF4F6881CF5AD040C055DF4F788158
:10967000C05BD040C1010E9463206894A0F8B0F89C
:10968000912CCC24CA94DC2CF1E0CD54DF4FF8832C
:10969000C35BD04084CB01E04016510409F040C0C8
:1096A000CD54DF4F1881C35BD0401123C9F1C6559B
:1096B000DF4F8881CA5AD040807F91F1772029F00E
:1096C000C1010E948216892B59F1C755DF4F0881CD
:1096D000C95AD040C655DF4F1881CA5AD040C55527
:1096E000DF4F2881CB5AD040C455DF4F3881CC5A48
:1096F000D040C355DF4F4881CD5AD040C255DF4FCF
:109700005881CE5AD040C155DF4F6881CF5AD040E2
:10971000C055DF4F7881C05BD040C1010E946320FB
:10972000C655DF4F8881CA5AD0408F70912C823045
:1097300008F06CC1C755DF4F9880C95AD0409920B6
:1097400009F43ECF772081F066EA7AE08EE692E176
:109750000F94061561E0C1010E94202D60E071E1C7
:10976000C1010E94A02EF7C9C655DF4F8881CA5A91
:10977000D040982F9F70923008F0A5CDC755DF4F8D
:109780009880C95AD040992009F41EC1807F31F4D5
:10979000B101CE0187559F4F0F94BF166894A0F872
:1097A00023E0B22A912CA1CE6894B2F8CD54DF4FB9
:1097B0008881C35BD040882309F462CFC655DF4F50
:1097C0008881CA5AD040807F81F040E050E061E05B
:1097D00070E0C1010E94E729672B682B692B59F5BE
:1097E000C1010E948216892B31F5912CCC24CA9498
:1097F000DC2CD5CA6894B2F891E04916510409F0FE
:10980000F2CDCD54DF4FA881C35BD040AA2309F429
:10981000C7C0C655DF4F8881CA5AD040807F29F320
:1098200040E050E061E070E0C1010E94E729672B51
:10983000682B692BA9F6C755DF4F0881C95AD0405C
:10984000C655DF4F1881CA5AD040C555DF4F288111
:10985000CB5AD040C455DF4F3881CC5AD040C35585
:10986000DF4F4881CD5AD040C255DF4F5881CE5A84
:10987000D040C155DF4F6881CF5AD040C055DF4F2F
:109880007881C05BD040C1010E946320AECFB1E0BF
:109890004B16510409F0A2C0CD54DF4FE881C35BE1
:1098A000D040912CA12C14E0B12EEE2309F41DCE52
:1098B000C655DF4F8881CA5AD040807F81F040E092
:1098C00050E062E070E0C1010E94E729672B682B3D
:1098D000692B89F5C1010E948216892B61F5912CB3
:1098E000A12C64E0B62E82CF912CA12CA4E0BA2E3C
:1098F000F1E04F16510409F07FC0CD54DF4F0881CD
:10990000C35BD040912CA12CE4E0BE2E002309F4CF
:109910007DC0C655DF4F8881CA5AD040807FF9F29A
:1099200040E050E062E070E0C1010E94E729672B4F
:10993000682B692B79F6C755DF4F0881C95AD0408B
:10994000C655DF4F1881CA5AD040C555DF4F288110
:10995000CB5AD040C455DF4F3881CC5AD040C35584
:10996000DF4F4881CD5AD040C255DF4F5881CE5A83
:10997000D040C155DF4F6881CF5AD040C055DF4F2E
:109980007881C05BD040C1010E946320A8CFC6553A
:10999000DF4F8881CA5AD040807F69F46894B0F85C
:1099A000912CCC24CA94DC2C11E0CD54DF4F1883C9
:1099B000C35BD040F4C923E0B22AF4CECD54DF4FCC
:1099C0006882C35BD04011CFCC24CA94DC2CE1E088
:1099D000CD54DF4FE883C35BD040E1C9912CA12C6B
:1099E00004E0B02ECC24CA94DC2C21E0CD54DF4F0F
:1099F0002883C35BD040D3C9CC24CA94DC2C81E03B
:109A0000CD54DF4F8883C35BD040C9C9CC24CA94EE
:109A1000DC2C91E0CD54DF4F9883C35BD040BFC9AD
:109A2000DC01ED91FC91008CF18DE02DC755DF4FED
:109A30000881C95AD040C655DF4F1881CA5AD04054
:109A4000C555DF4F2881CB5AD040C455DF4F3881F0
:109A5000CC5AD040C355DF4F4881CD5AD040C25573
:109A6000DF4F5881CE5AD040C155DF4F6881CF5A61
:109A7000D040C055DF4F7881C05BD040199581112F
:109A800098C9A3C9A114B10439F0A501B101CE014F
:109A900087559F4F0E94512DF10181859285009736
:109AA00009F460C0CF54DF4FE880F980C15BD0403B
:109AB000DC01ED91FC910488F589E02DCD54DF4F58
:109AC000C880C35BD040C755DF4F0881C95AD0401A
:109AD000C655DF4F1881CA5AD040C555DF4F28817F
:109AE000CB5AD040C455DF4F3881CC5AD040C355F3
:109AF000DF4F4881CD5AD040C255DF4F5881CE5AF2
:109B0000D040C155DF4F6881CF5AD040C055DF4F9C
:109B10007881C05BD04019956C01F10181859285F7
:109B2000DC01ED91FC91048CF58DE02D19950597E4
:109B300011F46894A0F8B2FC3CC1992021F0692D81
:109B4000C1010E94202DC354DF4F08811981CD5BD4
:109B5000D040B5010530110509F445C9C1010E9485
:109B6000A02E41C98085863009F45DC098F4843008
:109B700009F427C1853009F702E04016510409F4C1
:109B80001CC113E04116510409F4BBC04A94452896
:109B9000A1F6B3C0883009F46EC1893071F6CD5496
:109BA000DF4FE881C35BD040EE2339F2772079F0B4
:109BB000C755DF4F8881C95AD040813041F4C6551E
:109BC000DF4F8881CA5AD040807F09F4B6CFC7558D
:109BD000DF4F0881C95AD040C655DF4F1881CA5A95
:109BE000D040C555DF4F2881CB5AD040C455DF4FF8
:109BF0003881CC5AD040C355DF4F4881CD5AD04030
:109C0000C255DF4F5881CE5AD040C155DF4F6881D1
:109C1000CF5AD040C055DF4F7881C05BD040C101E2
:109C20000E94A93512C1C755DF4F8880C95AD0405C
:109C3000882009F4A1CF70E060E0C1010E94A02754
:109C40008C01009709F479CFF12CE12C97FF06C025
:109C5000119501951109EE24E394F12CC8010197A7
:109C60008634910508F069CFD02E61E0802F0F94E3
:109C7000FE01EFEFE80DE53110F5F0E08827EC5B31
:109C8000F14B8F4F0D94E537594E5B4E5F4E5F4E53
:109C90005B4E594E5B4E5F4E5F4E5F4E5F4E5F4E6A
:109CA0005F4E594E594E5F4E5F4E5F4E5F4E594E5E
:109CB000594EF1E0EF266E2D8D2D0F94D0016FE6F9
:109CC0007AE08EE692E10F9406154AE050E0B80182
:109CD0008EE692E10F94F7136DE67AE08EE692E15C
:109CE0000F9406154AE050E0B7018EE692E10F941A
:109CF000F7138EE692E10F94BA126894A0F8B0F8C8
:109D000058C0C1010E948427892B49F4D101ED91EB
:109D1000FC91608171818EE796E00F946C07CE0113
:109D200087559F4F0E942A1F20E030E048EC52E404
:109D30000F948A360F94F638CD54DF4F68837983B9
:109D40008A839B83C35BD040CD54DF4FC880D980CA
:109D5000C35BD04088E00E94B4D32B013C0169E68C
:109D60007AE08EE692E10F9406154AE050E0CD5479
:109D7000DF4F68817981C35BD0408EE692E10F941A
:109D8000F71364E67AE08EE692E10F940615B301CC
:109D9000A201662777272AE08EE692E10F946C12E3
:109DA0008EE692E10F94BA12B201A601C1010E949F
:109DB0002427CC24C394D12CC0CE6894A0F8B1F849
:109DC000F8CFCD54DF4FB881C35BD040BB2309F43B
:109DD000B4CEC755DF4F8881C95AD0407720B9F13A
:109DE000813041F4C655DF4F8881CA5AD040807F08
:109DF00009F4A3CEC755DF4F0881C95AD040C655D4
:109E0000DF4F1881CA5AD040C555DF4F2881CB5A41
:109E1000D040C455DF4F3881CC5AD040C355DF4FB6
:109E20004881CD5AD040C255DF4F5881CE5AD040DC
:109E3000C155DF4F6881CF5AD040C055DF4F788180
:109E4000C05BD040C1010E948D366C0176CE81305E
:109E500089F6CE0187559F4F0E9402FA449750F62B
:109E60006EE170E0CE0187559F4F0E94D61E689428
:109E7000A0F8B1F8BFCFCD54DF4FF881C35BD0401D
:109E8000FF2309F45ACE772079F0C755DF4F888138
:109E9000C95AD040813041F4C655DF4F8881CA5A33
:109EA000D040807F09F449CEC755DF4F0881C95A99
:109EB000D040C655DF4F1881CA5AD040C555DF4F34
:109EC0002881CB5AD040C455DF4F3881CC5AD0407E
:109ED000C355DF4F4881CD5AD040C255DF4F58811E
:109EE000CE5AD040C155DF4F6881CF5AD040C055BF
:109EF000DF4F7881C05BD040C1010E949B34A5CF69
:109F0000C354DF4F28813981CD5BD04025303105E6
:109F100011F40C94F34640E054E0B101CE018755B2
:109F20009F4F0E94512D60E074E018CE0E94711F77
:109F3000672B682B692B11F00C94E441B12CA12CF8
:109F40000C9415424114510409F045C080818823C6
:109F500011F40C94193FCE018F549F4F0E94992603
:109F60002C01C655DF4F8881CA5AD0408F7071F5D9
:109F7000642DCE0187559F4F0E94231BCF55DF4F85
:109F80002883C15AD040CE55DF4F3883C25AD040C3
:109F9000CD55DF4F4883C35AD040CC55DF4F58834F
:109FA000C45AD040CB55DF4F6883C55AD040CA55FC
:109FB000DF4F7883C65AD040C955DF4F8883C75AD0
:109FC000D040C855DF4F9883C85AD040411451043F
:109FD00011F40C94193F60E87CE08EE692E10F9456
:109FE00006154AE050E0B6018EE692E10F94F713B1
:109FF00069E77CE08EE692E10F940615D101ED91C0
:10A00000FC91608171818EE692E10F94101463E7F8
:10A010007CE08EE692E10F940615CF54DF4F688105
:10A020007981C15BD0408EE692E10F94101461E714
:10A030007CE08EE692E10F940615CE0187559F4F86
:10A040000E94AC23CF54DF4FE881F981C15BD0403F
:10A05000309711F40C945A3F8081843211F00C94A3
:10A060005A3F6DE57CE08EE692E10F9406158EE690
:10A0700092E10F94BA128CEFC82EDD24DA940C947E
:10A0800067484F925F926F927F928F929F92AF92AA
:10A09000BF92CF92EF92FF920F931F93CF93DF93D4
:10A0A000CDB7DEB76D970FB6F894DEBF0FBECDBF4C
:10A0B000009709F4A4C0FC0120852F70253009F019
:10A0C0009EC02A015B01868097808091880C8F5FFB
:10A0D0008093880C8114910409F48CC0F40180856C
:10A0E0008F70843009F082C0618572858091F90D8E
:10A0F0009091FA0D0E9441F93C01009709F476C055
:10A10000FC0180858F70853009F070C0B301CE01ED
:10A1100001960E94D632A114B104A9F0CE01019695
:10A120000E94CF26882379F0C12C7201F5010081AD
:10A130001181228133814481558166817781CE01ED
:10A1400001960E94643E60E0C3010E94F3F900970B
:10A15000D1F1FC0120852F702230A9F581859285EF
:10A16000A385B4850797A105B10569F561E0C30131
:10A170000E94F3F9A201B5010E944150A114B1045B
:10A1800089F5882379F18091880C81508093880C1F
:10A19000CE0101960E94783181E06D960FB6F89459
:10A1A000DEBF0FBECDBFDF91CF911F910F91FF900A
:10A1B000EF90CF90BF90AF909F908F907F906F90D7
:10A1C0005F904F900895A114B10461F4CE010196FF
:10A1D0000E94CF26882331F0CE0101960E940151C2
:10A1E000892B89F6CE0101960E947831F401828094
:10A1F000938070CF8091880C81508093880C80E090
:10A20000CCCFDF92EF92FF920F931F93CF93DF9308
:10A2100000D000D01F921F92CDB7DEB77C0119820B
:10A220001A821B821C821D821E821F8218868A81CE
:10A230008F708A83D701ED91FC91608171818EE6E8
:10A2400092E10F9410146CEC7CE08EE692E10F9496
:10A250000615C7010E94CF2681111BC063EC7CE06C
:10A260008EE692E10F9406158EE692E10F94BA12F3
:10A270000FEF1FEFC80128960FB6F894DEBF0FBE90
:10A28000CDBFDF91CF911F910F91FF90EF90DF90A5
:10A290000895C7010E94032ED82EF701818592856B
:10A2A000009791F0DC01ED91FC910688F789E02D93
:10A2B00019958C0197FD08C081E00115110509F47D
:10A2C00080E00E94DF16D6CFF7018085873009F441
:10A2D0002EC0EFEFED0DE43150F5F0E08827EC589B
:10A2E000FE4A8F4F0D94E537885191519751975100
:10A2F0009151885197519751975197519751975133
:10A30000975188519751975197519751885188513A
:10A3100064EA7CE08EE692E10F94061501E010E01D
:10A32000A9CF80E00E94DF1610E000E0A3CF40E05C
:10A3300052E0B701CE0101960E94102ED701189667
:10A340008C911897873089F160F4833009F456C0F6
:10A35000843061F064EB7CE08EE692E10F940615A8
:10A36000E3CF883009F44AC08930A1F760E0CE011C
:10A3700001960E94091E8C0169EA7CE08EE692E15A
:10A380000F9406154AE050E0B8018EE692E10F9472
:10A39000F7138EE692E10F94BA1291E080E0012B60
:10A3A00009F490E0092F182F65CF1296ED91FC91DA
:10A3B00080858F7010E000E08530F1F661EC7CE084
:10A3C0008EE692E10F94061550E040E070E060E008
:10A3D000F701828193810E944150F82E082F10E0EE
:10A3E0006EEB7CE08EE692E10F9406158F2D0E94B5
:10A3F000DF168EE692E10F94BA123CCFCE010196A1
:10A400000E94711F8B01B8CFCF92EF92FF920F93F2
:10A410001F93CF93DF9300D000D01F921F92CDB730
:10A42000DEB719821A821B821C821D821E821F8245
:10A4300018861A811F70CC24C394F12CE12C02E001
:10A440002B813C8140E05E816F8178850E94643E73
:10A4500028960FB6F894DEBF0FBECDBFDF91CF9127
:10A460001F910F91FF90EF90CF9008952F923F9200
:10A470004F925F926F927F928F929F92AF92BF9214
:10A48000CF92DF92EF92FF920F931F93CF93DF93C0
:10A49000CDB7DEB7C155D1090FB6F894DEBF0FBEF8
:10A4A000CDBF5C014B01D090D20BDD2009F4FCC084
:10A4B0008091DF0B9091E00B892B09F0F5C0809122
:10A4C000880C8F5F8093880CE091F90DF091FA0D64
:10A4D000309709F4E1C0668077800091F90D109102
:10A4E000FA0D0115110509F4D3C06114710409F4C2
:10A4F000CFC0D30118968C918F70853091F7C3012E
:10A500000E9485FA823068F3B301CE0101960E9461
:10A51000D632CE0101960E94CF26882309F4B0C01E
:10A520008091DF0B9091E00B892B09F065C040E032
:10A5300058E060E070E0CE0101960E94E729672BA9
:10A54000682B692B09F49CC019A21AA21BA21CA299
:10A550001DA21EA21FA218A68AA18F708AA340E086
:10A5600053E0BE016F5F7F4FCE0181960E94102E97
:10A570006EED7CE08EE692E10F94061540E058E027
:10A5800060E070E0CE0101960E9495298A859B8546
:10A590000097A1F1DC01ED91FC910488F589E02D93
:10A5A000CC24C394F12CE12C09A11AA12BA13CA12C
:10A5B0004DA15EA16FA178A519958F3F980709F469
:10A5C0005FC0E981FA8160817181892B09F044C003
:10A5D0008EE692E10F9410146CED7CE08EE692E131
:10A5E0000F94061564ED7CE08EE692E10F9406155B
:10A5F0008EE692E10F94BA12D12C42C08985883040
:10A60000F1F0893079F08430D9F509A11AA12BA194
:10A610003CA14DA15EA16FA178A5CE0101960E943B
:10A620008D36CBCF09A11AA12BA13CA14DA15EA1D2
:10A630006FA178A5CE0101960E94A935BECF09A1D0
:10A640001AA12BA13CA14DA15EA16FA178A5CE01BD
:10A6500001960E949B34B1CF8EE692E10F941014C4
:10A6600062ED7CE08EE692E10F9406156EEC7CE0E4
:10A670008EE692E10F9406158EE692E10F94BA12DF
:10A68000F30162807380CE0101960E94783125CF5C
:10A690008EE692E10F94BA128091880C81508093DB
:10A6A000880CD1101092D20B65E0D5018D919C9150
:10A6B0000E94F3F91C01009709F4CBC0FC018085CE
:10A6C00085958595859585952F968FAF2F97418494
:10A6D0005284638474840F94B4062F96FFAD2F9731
:10A6E000FF2309F4B6C0461A570A680A790A19A264
:10A6F0001AA21BA21CA2F9A31AA11F70106A1AA306
:10A700004DA25EA26FA278A624E08216910449F5BC
:10A71000D12CC12CE12C50E2F52E0F2F2BA13CA106
:10A720004DA15EA16FA178A5C5010E940B2AC301AE
:10A73000B20128EE33E040E050E00F949037BA01C8
:10A74000A9012AE030E08EE692E10F94AF136DE9A3
:10A750007DE08EE692E10F9406158EE692E10F946D
:10A76000BA1277FE76C082E048165104610480E890
:10A7700078060CF46EC00E94AEDA2B0162967FAFB1
:10A780006EAF6297D12CC12CE12C40E2F42E09A1CE
:10A790001AA12BA13CA14DA15EA16FA178A5C50175
:10A7A0000E940B2A6296AEADBFAD6297A83CB10580
:10A7B0007CF564E87DE087EC91E10F9406154AE0B2
:10A7C00050E0B20187EC91E10F94F71387EC91E12F
:10A7D0000F94BA1288248A94982CC401CF5ADF4F60
:10A7E0000FB6F894DEBF0FBECDBFDF91CF911F91A2
:10A7F0000F91FF90EF90DF90CF90BF90AF909F9020
:10A800008F907F906F905F904F903F902F90089522
:10A8100019821A821B821C821D821E821F82188648
:10A820001A811F701A832F96BFAD2F97B983CC243E
:10A83000C394F12CE12C0B2F2B813C8140E05E81F5
:10A840006F817885C5010E94643EF10180858F701B
:10A850008087F1E08F16910459F4D50118968C91F8
:10A86000843079F0893009F44DC1C5010E94122F5E
:10A87000F50181859285009709F013C4912C812CF4
:10A88000ACCF8091DF0B9091E00B892BB9F4F501EF
:10A8900042805380D20118968C918F70853041F49C
:10A8A000C2010E9485FA082F10E00230110554F40D
:10A8B0006DE27DE08EE692E10F940615C5010E94DF
:10A8C000122F8BCF9092E00B8092DF0B70E060E054
:10A8D000C5010E94A0271C0161E070E0C5010E9433
:10A8E000A0273C01053011056CF164E0C2010E9413
:10A8F000F3F9FC010185128526E040E855E260E0AD
:10A9000070E082E19FE00E9431B92092121082E152
:10A910009FE0909311108093101010921D111092CF
:10A920001F1110921E110130110509F4C2C06CF400
:10A93000012B09F4B3C065E17DE08EE692E10F944E
:10A94000061525C002E010E0D7CF0230110579F0DE
:10A950000330110581F7709214106092131081E09A
:10A9600090E0909316108093151084E00BC07092C5
:10A9700014106092131081E090E090931610809371
:10A98000151083E00F94DE0860968FAF6097609695
:10A99000FFAD6097F11197C000911710109118103A
:10A9A00060E17DE08EE692E10F940615D501ED9110
:10A9B000FC91608171818EE692E10F94101469E040
:10A9C0007DE08EE692E10F940615C801012E000C81
:10A9D000AA0BBB0B89839A83AB83BC8380E190E095
:10A9E0009E838D83BE016F5F7F4F8EE692E10E9452
:10A9F000EC320F94BA12B801C5010E94F22FE09117
:10AA0000DC0BF091DD0B62817381CE0101960E9417
:10AA1000D6328091DC0B9091DD0B892BB1F1CE0108
:10AA200001960E94CF26882381F18985843069F5BB
:10AA300070E060E0CE0101960E94A027281639063A
:10AA400021F561E070E0CE0101960E94A027681612
:10AA50007906D9F4B801CE0101960E94F22FE09157
:10AA6000DC0BF091DD0B828193819093DD0B809361
:10AA7000DC0B892B51F4E091F90DF091FA0D8681F0
:10AA800097819093DD0B8093DC0BCE0101960E94A1
:10AA900078311092E00B1092DF0B10CF70921410EF
:10AAA0006092131081E090E090931610809315103F
:10AAB00069CF7092141060921310109316100093C7
:10AAC000151082E05FCF63EF7CE08EE692E10F9499
:10AAD00006156096EFAD60978E2F90E0B0E0A0E095
:10AAE00089839A83AB83BC8380E190E09E838D83CE
:10AAF000BE016F5F7F4F8EE692E10E94EC320F94B1
:10AB0000BA12C7CF8091DF0B9091E00B892B09F02F
:10AB1000D5CE9092E00B8092DF0B0E94F5BE3C01F7
:10AB2000009741F0DC0118968C911897807F866021
:10AB300018968C9330E020E043E050E060E2CE01D4
:10AB400001960E942DD9D501ED91FC916081718112
:10AB50004FE150E0CE0101960F94623C6DE876E043
:10AB6000CE0101960F943C3C26E040E855E260E0BF
:10AB700070E082E19FE00E9431B970E060E0C501C1
:10AB80000E94A0278093121082E19FE09093111001
:10AB90008093101010921D1110921F1110921E110F
:10ABA00084E398E090931410809313108AE090E06F
:10ABB000909316108093151083E00F94DE08182FE1
:10ABC000811127C26AE77DE08EE692E10F940615B7
:10ABD00007E110E19BE2292E90E1392E20E1422E7F
:10ABE000512CF801819191918F01092E000CAA0B33
:10ABF000BB0B89A39AA3ABA3BCA35EA24DA2BE01CB
:10AC00006F5D7F4F8EE692E10E94EC3268E77DE057
:10AC10000F9406152016310621F78EE692E10F9467
:10AC2000BA1260911B1070911C1090E080E00F949C
:10AC30002B3620E030E048EC52E40F9484389B013E
:10AC4000AC0168E279E0C3010E94D6FEC0901F10FB
:10AC5000D0902010F12CE12CA701960163E976E059
:10AC6000C3010E9410FD609121107091221090E0AC
:10AC700080E00F942B3620E030E048EC52E40F9453
:10AC800084389B01AC0167E976E0C3010E94D6FEDF
:10AC9000609123107091241090E080E00F942B3687
:10ACA00020E030E040E251E40F9484389B01AC0195
:10ACB00065E976E0C3010E94D6FE2091171030911D
:10ACC000181050E040E069E976E0C3010E9410FDF1
:10ACD000CD28CE28CF2809F479C0D5011296ED9160
:10ACE000FC9190859F70953009F070C061E0CF01B4
:10ACF0000E94F3F9009709F469C0FC0120852F70C8
:10AD0000243009F063C061857285CE0181960E946E
:10AD1000EC30CE0181960E94CF26882309F452C0E0
:10AD200022961CAE1DAE1EAE1FAE229726961CAEFE
:10AD30001DAE1EAE1FAE26978FAD8F7080618FAF98
:10AD40008FEF23968FAF239724965FAD2497259698
:10AD50003FAD259726962FAD26979EAD7FAD2196C8
:10AD60006FAD219722964FAD2297092F27969FAF5F
:10AD7000279728967FAF289729966FAF29972A960D
:10AD80004FAF2A97482F2B968FAF2B972C965FAFFC
:10AD90002C972D963FAF2D972E962FAF2E97CC2424
:10ADA000C394F12CE12C172F262F2A963FAD2A971A
:10ADB0002D966FAD2D972E967FAD2E97CE01819655
:10ADC0000E94643ECE0181960E94783180911710D6
:10ADD00083FF3BC18EE398E090931410809313108F
:10ADE00081E090E0909316108093151083E00F940B
:10ADF000DE0881110BC0209117103091181050E01F
:10AE000040E06CE976E0C3010E9410FD1092E00B77
:10AE10001092DF0BC5010E940151181619061CF48F
:10AE2000C5010E94045281E090E09093E00B809372
:10AE3000DF0B62E370E080E090E00F94430483E175
:10AE400090E0909314108093131084E090E090931E
:10AE500016108093151083E00F94DE08182F8111CF
:10AE600006C168E57DE08EE692E10F94061507E1E4
:10AE700010E18FE1E82E80E1F82ED8016D917D91EF
:10AE80008D014AE050E08EE692E10F94F71366E5FB
:10AE90007DE08EE692E10F940615E016F10669F763
:10AEA0008EE692E10F94BA120091171010911810CB
:10AEB00001151105D1F0B801012E000C880B990B7A
:10AEC0000F942B362DEE3EE94CE35EE30F948A3669
:10AED00022E538EB42E152E40F9417389B01AC01B4
:10AEE00061E377E0C3010E94D6FE60911910709172
:10AEF0001A10072E000C880B990B0F942B362DEE91
:10AF00003EE94CE35EE30F948A3622E538EB42E1FA
:10AF100052E40F9417386B017C01AC019B0161E98D
:10AF200076E0C3010E94D6FE60911D1070911E1044
:10AF3000161617060CF092C0072E000C880B990B02
:10AF40000F942B3620E030E040E251E40F94843837
:10AF50009B01AC0160EA76E0C3010E94D6FE20E0CE
:10AF600030E040E252E4C701B6010F942C391816C4
:10AF7000B4F4012BA1F00E945FF9882369F080915D
:10AF8000870C811109C0D501ED91FC91608171811F
:10AF900084EA96E00F946C07C5010E94045280E099
:10AFA00091E00F94F62D8C01892BD9F01CA21BA2E5
:10AFB0001EA21DA28FEF9FEF98A78FA386E892E0B5
:10AFC0009AA389A31AA619A61CA70BA780E091E053
:10AFD00098AB8FA71EA61DA6B301CE0181960E9435
:10AFE000DCBC0E945FF9882349F08091870C8111B5
:10AFF00005C0B801CE0101960F946C07C8010F94EB
:10B00000922E6114710409F444CDC3010E94A4FE80
:10B0100040CD62E67DE08EE692E10F940615812F29
:10B0200090E0B0E0A0E089A39AA3ABA3BCA380E129
:10B0300090E09EA38DA3BE016F5D7F4F8EE692E1EF
:10B040000E94EC320F94BA12C1CE20E030E0A90188
:10B050006CE976E0C3010E9410FDEBCE20E030E009
:10B06000A90160EA76E0C3010E9410FD78CF60E498
:10B070007DE08EE692E10F940615812F90E0B0E01E
:10B08000A0E089A39AA3ABA3BCA380E190E09EA318
:10B090008DA3BE016F5D7F4F8EE692E10E94EC3280
:10B0A0007ECFDC01ED91FC910484F585E02D1995AE
:10B0B000892B09F4E3CBF50181859285DC01ED91C3
:10B0C000FC910480F581E02DB40119954C0185CBEC
:10B0D0002F923F924F925F926F927F928F929F92A8
:10B0E000AF92BF92CF92DF92EF92FF920F931F9396
:10B0F000CF93DF93CDB7DEB7C457D1090FB6F8941D
:10B10000DEBF0FBECDBFDC0114962D913C9115978B
:10B11000232B11F40C9492623B014C01AA969FAF31
:10B120008EAFAA9786EB94E0A8969FAF8EAFA897B4
:10B13000AE96BFAFAEAFAE978EE994E0AC969FAF40
:10B140008EAFAC97FD0182819B01225031092230E4
:10B15000310508F003C6803409F4F7C208F04AC08C
:10B16000843008F085C280919B0B8F5F80939B0B8E
:10B17000A3016FEFC4010E946C1BD40112960C91C5
:10B1800012970695017013961C9113978AEC810F04
:10B19000803108F043C061EB76E08D919C910E9474
:10B1A00041F97C010097D1F1FC0180858F708530D9
:10B1B000A9F58091AD12181324C08091AE1280348D
:10B1C00001F58091AF129091B0125C01990FCC08FB
:10B1D000DD0860E0C7010E94F3F9FC0181859285DA
:10B1E000A385B485A816B906CA06DB060CF065C0AF
:10B1F000512C3EC0823409F4A8C208F439C28058E8
:10B20000AFCF1093AD1280E48093AE12812F0F94D4
:10B2100011039093B0128093AF12D7CF212F30E05B
:10B22000F901E459F74D8491F901E453F74D149174
:10B23000F901EE5EF64DF490FF2009F43BC0811158
:10B240000F946901EF2DF0E0EE0FFF1FE751F84D6D
:10B25000A591B491EC911E2331E020E009F430E097
:10B26000832F922F552453940817190609F0C0CF45
:10B27000F3E06F16710409F488C0D4011496ED91BF
:10B28000FC91E181EF70E150EC3008F07EC0F0E01D
:10B290008827E25BF64A8F4F0D94E5376F59EB5ADA
:10B2A000A559DB59EB5AF459EB5A285A555A6E5A9C
:10B2B000B05AD25A90E080E0D5CF61E0C7010E9439
:10B2C000F3F955245394FC0181859285A385B485B7
:10B2D0008A159B05AC05BD050CF0CACF89CF0F942C
:10B2E000B4069B01AC0144275527D4011496ED9177
:10B2F000FC916281738190E080E0AA24AA94BA2C28
:10B30000C12CD12C18EEE12E13E0F12E00E010E05C
:10B310000E9452D38823C9F1F401008111816CE0AD
:10B3200076E0C8010E9441F9892B41F461E176E0A1
:10B33000C8010E9441F9892B09F40EC142E050E096
:10B3400063E0C4010E946C1B20C00F94B4069B01F3
:10B35000AC0144275527D4011496ED91FC916281EC
:10B36000738190E080E0AA24AA94BA2CC12CD12C3D
:10B370001CE2E12EFF24F39400E010E00E9452D37F
:10B3800042E050E064E0811184C0D4011496ED9154
:10B39000FC91808183FB992790F9951509F4D2C11E
:10B3A000982F907E09F439C1982F907E90528F711A
:10B3B000892B808358C10F94B4069B01AC014427AC
:10B3C0005527D4011496ED91FC916281738190E030
:10B3D00080E0AA24AA94BA2CC12CD12C16E9E12E23
:10B3E000F12C00E010E0CACF0F94B4069B01AC0131
:10B3F00044275527D4011496ED91FC916281738105
:10B4000090E080E0AA24AA94BA2CC12CD12C18EE8A
:10B41000E12E13E0F12E00E010E00E9452D38823C9
:10B4200009F4B3CFF4010081118167E176E0C8012E
:10B430000E9441F9892B41F46DE176E0C8010E9438
:10B4400041F9892B09F488C042E050E068E079CFE7
:10B450000F94B4069B01AC0144275527D4011496E0
:10B46000ED91FC916281738190E080E0AA24AA941E
:10B47000BA2CC12CD12C1CE2E12EFF24F39400E065
:10B4800010E00E9452D342E050E069E0882309F4C2
:10B490007CCFC4010E946C1B0F94B406D401149697
:10B4A000ED91FC917383628370CF0F94B4069B017E
:10B4B000AC0144275527D4011496ED91FC9162818B
:10B4C000738190E080E0AA24AA94BA2CC12CD12CDC
:10B4D00016E9E12EF12C00E010E0D3CF0F94B40672
:10B4E0009B01AC0144275527D4011496ED91FC91A2
:10B4F0006281738190E080E0AA24AA94BA2CC12CC6
:10B50000D12C18EEE12E13E0F12E00E010E00E94A5
:10B5100052D3882309F439CFF4010081118164E208
:10B5200076E0C8010E9441F9892B39F46AE276E09D
:10B53000C8010E9441F9892B21F042E050E06BE004
:10B5400000CF66E076E0C8010E9441F942E050E099
:10B5500066E0892B09F4F5CE42E050E06DE0F1CED3
:10B560000F94B4069B01AC0144275527D4011496CF
:10B57000ED91FC916281738190E080E0AA24AA940D
:10B58000BA2CC12CD12C1CE2E12EFF24F39400E054
:10B5900010E00E9452D3882309F4F7CE42E050E035
:10B5A0006CE077CF0F94B4069B01AC01442755277C
:10B5B000D4011496ED91FC916281738190E080E05A
:10B5C000AA24AA94BA2CC12CD12C16E9E12EF12C74
:10B5D00000E010E0DECF0F94B4069B01AC014427DD
:10B5E0005527D4011496ED91FC916281738190E00E
:10B5F00080E0AA24AA94BA2CC12CD12C18E5E12E03
:10B6000012E0F12E00E010E00E9452D3882309F4EA
:10B61000BCCE42E050E060E094CE0F94B406D4017A
:10B620001496ED91FC91159773836283E181EF701D
:10B63000552009F445C0E230F1F050F4EE23E9F171
:10B64000D4011496ED91FC91808150FA83F9B1CE2A
:10B65000E53089F0A3016AE0E73091F7C4010E9468
:10B660006C1B8111EDCF80919B0B815080939B0BC4
:10B6700090E080E059C7F4010081118160E076E03C
:10B68000C8010E9441F9892BA9F467E176E0C8015D
:10B690000E9441F9892B71F46DE176E0C8010E94A6
:10B6A00041F9892B39F468EE75E0C8010E9441F92F
:10B6B000892B19F0A30166E0D1CFA30161E0CECFC1
:10B6C000E150ED3008F0BCCFF0E08827E559F44AAE
:10B6D0008F4F0D94E537785B205B7B5B7B5B205B5A
:10B6E0007E5B205B9F5B9F5B9F5B9F5B9F5B7B5B4E
:10B6F000A30162E0B3CFA30165E0B0CF0D911C912F
:10B7000060E076E0C8010E9441F9892BA9F467E165
:10B7100076E0C8010E9441F9892B71F46DE176E071
:10B72000C8010E9441F9892B39F468EE75E0C8011F
:10B730000E9441F9892B19F0A30167E08FCFA30183
:10B7400060E08CCF8F71806434CEB3E06B167104EF
:10B7500009F48ECF61EB76E0F401808191810E9443
:10B7600041F98C01D40113968C919091AD128913FB
:10B77000CEC09091AE12903409F0C9C08091AF1242
:10B780009091B0123C010115110509F4F0C0F801C7
:10B7900020852F70253009F0EAC0C8010E9485FA83
:10B7A000E1968FAFE197843008F4BDC063E0C80133
:10B7B0000E94F3F9DC0119968D919C91BAE0FB2E61
:10B7C000F89EF001F99EF00D1124E096FFAFEEAF68
:10B7D000E09762E0C8010E94F3F9DC0119968D91AF
:10B7E0009C91F89E5001F99EB00C112465010B2C20
:10B7F000000CEE08FF0861E0C8010E94F3F9E3962F
:10B800009FAF8EAFE39760E0C8010E94F3F9FC019F
:10B8100021843284438454849301072C000C440B0C
:10B82000550B2219330944095509E096AEADBFAD59
:10B83000E097BD01BB0F880B990B6C197D098E0930
:10B840009F090F945E37E396EEADFFADE397218538
:10B8500032854385548522193309440955090F94CB
:10B860009037C20ED31EE41EF51EE196FFADE197A0
:10B87000F53009F46BC081E090E0E096EEADFFADED
:10B88000E097AF01FF0F660B770B4C155D056E055A
:10B890007F050CF464C0B701A60165010B2C000CF8
:10B8A000EE08FF084C155D056E057F050CF45CC0C5
:10B8B0006A017B01E196FFADE197F23009F06BC0C0
:10B8C0006301770CEE08FF0860E0C8010E94F3F9FD
:10B8D000FC0181859285A385B485C816D906EA0640
:10B8E000FB060CF43BC661E0C8010E94F3F9FC01C1
:10B8F00081859285A385B4858C159D05AE05BF0510
:10B900000CF0B6CE81E090E0A0E0B0E02AC68093D3
:10B91000AD1290E49093AE120F9411039093B01275
:10B920008093AF122FCF8AE0869D6001879DD00C57
:10B9300011240D2C000CEE08FF08B12CA12C20E0E6
:10B9400038E2E0963FAF2EAFE09795CF64E0C801B4
:10B950000E94F3F9DC0119968D919C918ECF66249B
:10B960006A94A3E07A2E99CF712C612CA3CF2AE0A0
:10B97000289F6001299FD00C11240D2C000CEE088B
:10B98000FF08B12CA12C20E038E2E0963FAF2EAFAB
:10B99000E09781E090E0D4011496ED91FC916281F2
:10B9A0007381A301461B570B57FF03C05195419567
:10B9B0005109841795070CF4BEC08081982F929589
:10B9C00096959770963008F0B9C09F5F9295990F41
:10B9D000907E8F71892BB1C0F20161857285DB0188
:10B9E0008C9181114FC60115110509F456C0D8017B
:10B9F00018968C9118978F70843009F04EC0199664
:10BA00006D917C91CE0101960E94EC30CE010196A1
:10BA10000E94CF268823E9F1A114B10409F45FC084
:10BA20004114510431F0F20180858F70843009F4A3
:10BA30004BC025961CAE1DAE1EAE1FAE2597299697
:10BA40001CAE1DAE1EAE1FAE299723961FAD2397C9
:10BA50001F7023961FAF239781E022968FAF229706
:10BA6000CC24C394F12CE12C01E024962FAD249733
:10BA700025963FAD259740E027965FAD27972896FE
:10BA80006FAD289729967FAD2997CE0101960E9428
:10BA9000643ECE0101960E947831D4011496ED9156
:10BAA000FC91B382A282E4CD6114710429F0F30108
:10BAB00080858F70843019F062EE7AE0E3C561858D
:10BAC0007285FB0180818DCF61857285FB0180814C
:10BAD0008823F9F2CE0101960F945617DACF61143C
:10BAE000710431F0D30118968C918F708430E9F095
:10BAF00025961CAE1DAE1EAE1FAE259729961CAE18
:10BB00001DAE1EAE1FAE299723961FAD23971F7043
:10BB100023961FAF239782E022968FAF2297CC24E3
:10BB2000C394F12CE12C02E0A0CFF3016185728572
:10BB3000DB018C91CDCF80818F7180838081803AB1
:10BB4000B8F0C501BB0CAA0BBB0B8C159D05AE054F
:10BB5000BF0571F0E096EEADFFADE097CF01FF0FAE
:10BB6000AA0BBB0B8C159D05AE05BF0509F080CD5A
:10BB70006615770509F47CCDA2961CAE1DAE1EAEEF
:10BB80001FAEA297A0968FADA0978F708066A096EB
:10BB90008FAFA097A2968CAD9DADAEADBFADA29775
:10BBA00068968CAF9DAFAEAFBFAF6897AAE0B0E02C
:10BBB000A70196010F94AF376C966CAF7DAF8EAF37
:10BBC0009FAF6C976CE279E08EE692E10F940615D8
:10BBD0004AE050E0D40113966C918EE692E10F9406
:10BBE000D0126AE279E08EE692E10F940615CE015A
:10BBF0008C5A9F4F0E94AC2365EB76E0F401808164
:10BC000091810E9441F9B12CA12CD12CC12C6596B7
:10BC1000EFAC65976696FFAC669767960FAD679732
:10BC200068961FAD689769962FAD69976A963FAD84
:10BC30006A976B964FAD6B976C965FAD6C976FEF95
:10BC40000E9428E1D4010D911C9161E376E0C801C6
:10BC50000E9441F97C0166E376E0C8010E9441F947
:10BC60008C010097E1F1FC0180858F708430B9F57B
:10BC70006185728540E450E0CE0101960F94803CCE
:10BC80006FE270E0CE0101960F94473C892B59F486
:10BC9000D80119962D913C9143E050E060E4CE012B
:10BCA00001960E942DD900E020E032E040E150E012
:10BCB000BE016F5B7F4FCE018C5A9F4F0E948B213C
:10BCC0000E945FF9882359F08091870C811107C089
:10BCD000BE016F5B7F4FCE0101960F945107E114B7
:10BCE000F104A9F1F70180858F70843081F56185B9
:10BCF0007285CE0101960E94EC30CE0101960E9421
:10BD0000CF26882301F1CC24C394F12CE12C659635
:10BD10000FAD659766961FAD669767962FAD6797CF
:10BD200068963FAD689769964FAD69976A965FAD23
:10BD30006A976B966FAD6B976C967FAD6C97CE01E3
:10BD400001960E94643ECE0101960E947831D40192
:10BD50001496ED91FC91738262828ACC863009F44C
:10BD600056C070F4843009F45AC0853009F080CC94
:10BD700061E070E0CE018A599F4F0E944A7078CCF2
:10BD8000883009F4E1C2803109F072CC0F94B40616
:10BD90002B013C01C4010E948815A12CB12C650126
:10BDA00010E3E12E15E7F12E00E010E0A30192016F
:10BDB0000E9452D3882309F45BCC66E376E0D40179
:10BDC0008D919C910E9441F98C01009709F497C2D2
:10BDD000FC0180858F70843009F091C20F94B40605
:10BDE0002AE0AE014F5F5F4F0F94D3300E945FF99E
:10BDF000882309F484C28091870C811180C2BE011E
:10BE00006F5F7F4FD80119968D919C9176C261E04A
:10BE100070E0CE0186599F4F0E94F47129CC0F9497
:10BE2000B4062B013C01C4010E948815A12CB12C41
:10BE3000650118E9E12E1AE3F12E00E010E0A301FC
:10BE400092010E9452D3882309F412CCF401838119
:10BE500027968FAF279796E128969FAF2897282F90
:10BE600030E0F901E453F74DE4912996EFAF2997BB
:10BE7000F901EE5EF64DE4912A96EFAF2A9740E87D
:10BE80005EE360E070E062964CAF5DAF6EAF7FAF97
:10BE9000629762E00F94FE010F94B406605D7740F4
:10BEA000810991092E966CAF7DAF8EAF9FAF2E9713
:10BEB00087E364968FAF6497CE018F5B9F4F0F949B
:10BEC000DA07882349F028968FAD28978C3009F43B
:10BED0006FC048F48B3011F1412C512C50EC652E81
:10BEE0005FE7752E47C085518230B0F724961FADAD
:10BEF0002497612F70E0762F662766277F77259637
:10BF00008FAD2597682B90E080E00F9429362DECBB
:10BF10003CEC4CEC5DE30F948A3668C024966FAD20
:10BF2000249770E090E080E00F9429366B017C014B
:10BF300025961FAD259717FF0AC0AC019B0160E055
:10BF400070E080E89FEB0F9417386B017C011F7045
:10BF5000612F70E090E080E00F942B362DEC3CECEC
:10BF60004CEC5DE30F948A36A70196010F941838C4
:10BF70002B013C01CE018F5B9F4F0F94DA07882382
:10BF800009F4D7C128968FAD28978B3030F08D30CB
:10BF9000B0F18551823008F4BAC1312C212C30EC3B
:10BFA000AF963FAFAF978FE7E1968FAFE1974DC068
:10BFB00024961FAD2497612F70E090E080E00F94ED
:10BFC00029366B017C0125966FAD25976F7070E067
:10BFD00090E080E00F942B362DEC3CEC4CEC5DE3D4
:10BFE0000F948A36A70196010F9418382B013C0153
:10BFF00017FFC0CF77FA709477F87094BBCF239671
:10C000006FAD239770E090E080E00F942B362DEC1D
:10C010003CEC4CEC5DE30F948A366B017C0122967C
:10C020006FAD229770E090E080E00F942B369B017B
:10C03000AC01C701B6010F941838362E272EAF96E3
:10C040008FAFAF97E1969FAFE19766E579E08EE617
:10C0500092E10F9406154AE050E0D40113966C91DA
:10C060008EE692E10F94D01266E479E08EE692E1DA
:10C070000F940615B301A2018EE692E10F94DE1231
:10C080006FE379E08EE692E10F940615432D522D71
:10C09000AF966FADAF97E1967FADE1978EE692E1F7
:10C0A0000F94DE126DE379E08EE692E10F940615AF
:10C0B0008EE692E10F94BA12F4010081118162E8D8
:10C0C00077E0C8010E9441F9E3969FAF8EAFE397F6
:10C0D00069EB76E0C8010E9441F9E5969FAF8EAF0B
:10C0E000E597A3019201C301B2010F948C3981112C
:10C0F0001FC019821A821B821C828A818F708067FE
:10C10000F82E8A83242D4D825E826F827886B12C30
:10C11000A12CD12CC12CE9800B811C813E814F8147
:10C1200058856FEFE3968EAD9FADE3970E9428E1AF
:10C13000232D322DAF964FADAF97E1965FADE197CE
:10C14000632D722DAF968FADAF97E1969FADE197BE
:10C150000F948C39811127C019821A821B821C828C
:10C160008A818F708067F82E8A83232D832D922DEC
:10C17000AF96AFADAF97E196BFADE1978D839E834C
:10C18000AF83B887B12CA12CD12CC12CE9800B81B5
:10C190001C813E814F8158856FEFE5968EAD9FAD36
:10C1A000E5970E9428E166E376E0D4018D919C91A9
:10C1B0000E9441F97C01009709F4A1C0FC0180852F
:10C1C0008F70843009F09BC020E030E0A901C301EA
:10C1D000B2010F942436882309F491C020E030E0A6
:10C1E000A901632D722DAF968FADAF97E1969FADEC
:10C1F000E1970F942436882309F481C0A3019201AA
:10C20000C301B2010F942436811179C0232D322D40
:10C21000AF964FADAF97E1965FADE197632D722D6D
:10C22000AF968FADAF97E1969FADE1970F9424360F
:10C23000811165C01A821982FE0133968EE3DF01F7
:10C240001D928A95E9F7F7016185728540E450E017
:10C250008E010F5F1F4FC8010F94803C6FE270E0AA
:10C26000C8010F94473C892B51F4D70119962D91A1
:10C270003C9143E050E060E4C8010E942DD96EE794
:10C2800078E0C8010F943C3CB301A201CE018C5A66
:10C290009F4F0E9455DA0E945FF9882351F08091E8
:10C2A000870C811106C0BE016C5A7F4FC8010F94E4
:10C2B0006C07F80101900020E9F73197E01BF10BC2
:10C2C000EC0FFD1F88E48083432D522DAF966FAD98
:10C2D000AF97E1967FADE197CE018C5A9F4F0E94B8
:10C2E00055DA0E945FF9882351F08091870C811103
:10C2F00006C0BE016C5A7F4FC8010F946C070F94A3
:10C30000B406AB01BC01C4010E946115B1C92396FA
:10C310006EAD7FAD239776276727762790E080E084
:10C320000F9429362DEC3CEC4CEC5DE30F948A36EF
:10C3300084CE312C212CF0ECAF96FFAFAF972FE7D6
:10C34000E1962FAFE19781CE0F94B4062B013C010B
:10C35000C4010E948815A12CB12C650118E9E12EB9
:10C360001AE3F12E00E010E0A30192010E9452D3E3
:10C37000882309F47DC9D4011496ED91FC91159799
:10C38000818113961C91811155C01630F0F58CE017
:10C39000E0E5F2E0DE01119601900D928A95E1F759
:10C3A000E12FF0E0EE0FFF1F21E030E02C0F3D1FEA
:10C3B000E20FF31F60E080810F94FE0168ED75E1EC
:10C3C00083E01330C9F070F460EE75E181E0113064
:10C3D00099F06CED75E182E0123071F064EE75E178
:10C3E00080E00AC064ED75E184E0143029F060ED6E
:10C3F00075E185E0153091F70E944FFDD401149648
:10C40000ED91FC9181E0818333C96EEA79E08EE69B
:10C4100092E10F9406154AE050E0F40163818EE644
:10C4200092E10F94D01261E879E08EE692E10F94E8
:10C4300006151EC924E0129FF0011124E456F44FA2
:10C44000C080D180E280F3806DE779E08EE692E1F2
:10C450000F9406154AE050E0D40113966C918EE6D5
:10C4600092E10F94D01269E679E08EE692E10F94A2
:10C4700006152AE030E0B701A6018EE692E10F949E
:10C48000AF1366E376E0F401808191810E9441F967
:10C490008C01009709F443C0DC0118968C91189721
:10C4A0008F708430E1F519966D917C9140E450E0F5
:10C4B000CE0101960F94803C6FE270E0CE010196B0
:10C4C0000F94473C892B51F4F8012185328543E0D4
:10C4D00050E060E4CE0101960E942DD9FF92EF92C8
:10C4E000DF92CF9282E496E09F938F938E010F5B51
:10C4F0001F4F1F930F930F94D73C0E945FF90FB605
:10C50000F894DEBF0FBECDBF882309F4F8CE80912A
:10C51000870C8111F4CEB801CE010196EECE6AE50A
:10C5200079E083CF8FEF9FEFCC58DF4F0FB6F894B1
:10C53000DEBF0FBECDBFDF91CF911F910F91FF9056
:10C54000EF90DF90CF90BF90AF909F908F907F90B3
:10C550006F905F904F903F902F90089580E090E013
:10C56000DC01F40124813581F90142815381052EDA
:10C57000000C660B770B481759076A077B0709F40D
:10C5800077C85C01D4016D907C9061E376E0C301D3
:10C590000E9441F98C0166E376E0C3010E9441F9F3
:10C5A0001C010115110519F4892B09F476CA6BEFEA
:10C5B00075E0C3010E9441F92C0166EF75E0C301EB
:10C5C0000E9441F93C0162E379E08EE692E10F942A
:10C5D00006154AE050E0F40163818EE692E10F9483
:10C5E000D01260E379E08EE692E10F9406154AE0FE
:10C5F00050E0B5018EE692E10F94F7138EE692E1DA
:10C600000F94BA122114310409F4EDC9D10118961E
:10C610008C9118978F70843009F0E5C919966D9147
:10C620007C9140E450E0CE0101960F94803C0E9442
:10C630005FF9882309F4D7C98091870C8111D3C988
:10C640006FE270E0CE0101960F94473C892B51F4C4
:10C65000F1012185328543E050E060E4CE0101968E
:10C660000E942DD9A114B10409F41ECA4114510429
:10C6700039F0D20118968C918F70843009F4ACC9CE
:10C6800067ED7AE0CE0101960F945107ACC9AF92E5
:10C69000BF92DF92EF92FF920F931F93CF93DF939E
:10C6A00000D000D0CDB7DEB78C017B01D42EFB01CA
:10C6B00084819581892BF9F0A080B1806FE370E0CF
:10C6C000C5010F94473C0097B1F09C012A193B0922
:10C6D00037FD11C050E040E0B701CE0101960F9444
:10C6E000E60FBE016F5F7F4FC7010F941C0FCE0195
:10C6F00001960F94C40FF70184819581892BD9F19C
:10C70000E080F1806DEB76E0C7010F94523C892BFD
:10C7100001F5F801128A118A80E090E195878487FB
:10C7200084E890E0948B838B81E08687D58A81E0D2
:10C7300090E026960FB6F894DEBF0FBECDBFDF9116
:10C74000CF911F910F91FF90EF90DF90BF90AF902E
:10C7500008956AEC76E0C7010F94523C892B59F496
:10C76000F801128A118A148A138A84E890E0958766
:10C7700084871686DBCF90E080E0DBCFDC01149667
:10C78000ED91FC91309729F08081082E000C990BD7
:10C79000089590E080E00895DC011296ED91FC91FF
:10C7A00013973097B9F016968D919C91843091052E
:10C7B00041F08530910541F0039749F482E090E023
:10C7C000089581E090E0089581E190E008958085EA
:10C7D00090E0089590E080E008958091720C90912F
:10C7E000730C089584E190E008958091700C90910D
:10C7F000710C08951092710C1092700C81E090E011
:10C800000895DC011496ED91FC9180E0309711F0D1
:10C8100085A1817090E00895DC011296ED91FC9164
:10C82000309761F00190F081E02D808585958595A8
:10C830008595859519F081E090E0089590E080E07D
:10C8400008956AE87AE1811102C06CE87AE18DEB23
:10C8500091E10D9406156BE477E18DEB91E10F9476
:10C860000615F0E0E0E0199584EF91E00895CF938C
:10C87000DF93EC0160E670E28EE692E10F9406151C
:10C88000EA81FB810190F081E02D608171818EE66B
:10C8900092E10F9410148EE692E10F94BA12109266
:10C8A000730C1092720C81E090E0DF91CF910895AB
:10C8B000CF93DF93EC01EC81FD8141815281052E04
:10C8C000000C660B770B238182E19FE00E9431B957
:10C8D00070E060E08A819B810E94A027E0E1F0E1A6
:10C8E000828382E19FE09183808310921D111092D8
:10C8F0001F1110921E11DF91CF9108951F93CF93B6
:10C90000DF9300D000D0CDB7DEB7909314108093A2
:10C91000131063307105E9F1509316104093151010
:10C9200083E00F94DE08182F80E00E94B4D3609358
:10C93000760C7093770C8093780C9093790C11237C
:10C94000D9F06EEA71E287EC91E10F940615812F20
:10C9500090E0B0E0A0E089839A83AB83BC8380E160
:10C9600090E09E838D83BE016F5F7F4F87EC91E1E6
:10C970000E94EC320F94BA1281E0111180E02696E9
:10C980000FB6F894DEBF0FBECDBFDF91CF911F91E0
:10C9900008955527509316104093151084E0C1CF89
:10C9A000CF93DF93EC0166ED76E08EE692E10F9493
:10C9B000BE128C819D810F94922E70E060E08A817E
:10C9C0009B810E94DB261D821C8281E090E0DF912A
:10C9D000CF9108950D94922E0D94922E0D94922E37
:10C9E000CF93DF93EC0161E570E28EE692E10F9464
:10C9F0000615EA81FB810190F081E02D6081718153
:10CA00008EE692E10F9410148EE692E10F94BA1222
:10CA100081E090E09093730C8093720CDF91CF9142
:10CA2000089581E090E09093710C8093700C0895CC
:10CA3000AF92BF92CF92DF92EF92FF920F931F932C
:10CA4000CF93DF93EC018C819D81892B61F40A8166
:10CA50001B8181E190E00F94F62DBC01C8010E947A
:10CA6000DB269D838C830C811D810115110569F4E2
:10CA70006AE971E287EC91E10F94061587EC91E188
:10CA80000F94BA1290E080E086C180E00E94B4D397
:10CA9000D80117966D937D938D939C931A97CC80B4
:10CAA000DD80C114D104D9F0EA81FB813097B9F05F
:10CAB000028113810115110591F0F80180858F70B5
:10CAC000853069F4C8010E9485FA823040F0E09018
:10CAD000740CF090750CE114F10409F082C06DE55E
:10CAE00071E287EC91E10F94061561E070E08C81B2
:10CAF0009D81892B11F470E060E04AE050E087EC02
:10CB000091E10F94F7136BE571E287EC91E10F94DB
:10CB1000061561E070E08A819B81892B11F470E039
:10CB200060E04AE050E087EC91E10F94F71369E58B
:10CB300071E287EC91E10F940615EA81FB8161E0D7
:10CB400070E082819381892B11F470E060E04AE00B
:10CB500050E087EC91E10F94F71367E571E287EC01
:10CB600091E10F940615EA81FB810280F381E02DAB
:10CB700080858F7061E070E0853011F470E060E0D6
:10CB80004AE050E087EC91E10F94F71365E571E21C
:10CB900087EC91E10F940615EA81FB8182819381F4
:10CBA0000E9485FA61E070E0823010F070E060E091
:10CBB0004AE050E087EC91E10F94F71387EC91E1A4
:10CBC0000F94BA1262E771E287EC91E10F940615B7
:10CBD00087EC91E10F94BA12EC81FD818FEF808395
:10CBE00051CF61E0C8010E94F3F98C01DC01189675
:10CBF0008C9118978F70843031F419966D917C91D7
:10CC00006115710539F46DE371E287EC91E10F94E0
:10CC10000615D4CFC7010E9441F97C01009771F439
:10CC20006BE171E287EC91E10F940615F8016185E3
:10CC3000728587EC91E10F941014C0CF64EE76E01A
:10CC40000E9441F9009709F4C4C0DC0118962C91A8
:10CC500018972F70243009F0BCC01996AD90BC9085
:10CC600010E000E0A114B10409F4A6C0B8016D52AF
:10CC70007F4DC5010F942F30892B09F097C0F80123
:10CC8000E952FF4D25913491922F832FF601938322
:10CC900084836BEE76E0C7010E9441F9EC81FD814F
:10CCA000009709F49EC0DC0118962C9118972F70FC
:10CCB000223009F096C019964D915D916D917C914D
:10CCC0001C97411551056105710509F48AC052830D
:10CCD000418341815281052E000C660B770B238125
:10CCE00082E19FE00E9431B960EF76E0C7010E94C7
:10CCF00041F96C010C811D81009709F47FC0FC0192
:10CD000080858F70863009F079C065EF76E0C601C6
:10CD10000E9441F9D8011C969C938E931B976AEF51
:10CD200076E0C6010E9441F9F801968785876EEF8B
:10CD300076E0C6010E9441F9009709F457C0DC0172
:10CD400019968D919C91F8019683858364E077E034
:10CD5000C7010E9441F9D80150969C938E931F976A
:10CD600065E871E28DEB91E10F940615EA81FB8194
:10CD70000190F081E02D608171818DEB91E10F9444
:10CD800010148DEB91E10F94BA12EC81FD8181E0DA
:10CD9000808381E090E0DF91CF911F910F91FF9010
:10CDA000EF90DF90CF90BF90AF9008950A5F1F4F34
:10CDB0000834110509F056CF66EB70E28EE692E179
:10CDC0000F9406158EE692E10F94BA1296E080E079
:10CDD0005DCF86E090E0D60114969C938E931397D6
:10CDE00058CF80E895E29283818373CF88EE93E0F9
:10CDF000D80116969C938E931597A8CFF8011486A8
:10CE0000138688EE93E096838583168615869ECFDB
:10CE10004F925F926F927F928F929F92AF92BF924A
:10CE2000CF92DF92EF92FF920F931F93CF93DF93F6
:10CE3000CDB7DEB768970FB6F894DEBF0FBECDBF93
:10CE4000098B1A8B2B8B3C8B4D8B5E8B6F8B788F6A
:10CE5000DC0112962D913C911397232B09F4E0C02D
:10CE6000CC2009F4DDC06C01ED91FC91048CF58DB2
:10CE7000E02D19955C0169E770E28EE692E10F946E
:10CE80000615CE0141960E94AC23A114B10471F4A1
:10CE900060E0CE0141960E94091E682FF601848150
:10CEA00095810E9460CE81E090E0BCC0CE014196A9
:10CEB0000E9469214C0184E0F2E0AF16B10459F000
:10CEC00081E1A816B10409F447C081E0A1E0AA16E7
:10CED000B10409F485E019861A861B861C861D8616
:10CEE0001E861F86188A8295807F9A859F70892B5F
:10CEF0008A87EE24EA94FE2C09891A892B893C89B9
:10CF00004D895E896F89788DCE0109960E942039FE
:10CF10006FE670E28EE692E10F940615CE01099657
:10CF20000E94AC23B2E0AB16B10489F0E1E1AE1689
:10CF3000B104B1F0AA94AB2809F0B5CF188963E029
:10CF400070E0C6010E94AD38612F0E9460CE6F85EF
:10CF5000F6018481958151C0888D8170888FBACF08
:10CF60000FE710E08FEF88169806A9F0092C000C47
:10CF7000AA08BB08A50194012959310941095109A1
:10CF8000AFEFB0E00F94AF372BE531E040E050E079
:10CF90000F949037890163E070E0C6010E94AD38BC
:10CFA0005C01288930E0D8010F94FC37412C512CCA
:10CFB00032014A94A30192010F949037622FC50168
:10CFC0000E9460CE64E070E0C6010E94AD385C0152
:10CFD000AFEFB0E0A01BB10B288930E00F94FC3715
:10CFE000A30192010F949037622FC5010E9460CE79
:10CFF0006F85D60114968D919C910E9460CE1E85FE
:10D0000061E070E0C6010E94AD38612F0E9460CEE1
:10D010001D8562E070E0C6010E94AD38612F41CFEE
:10D0200090E080E068960FB6F894DEBF0FBECDBFEB
:10D03000DF91CF911F910F91FF90EF90DF90CF90F4
:10D04000BF90AF909F908F907F906F905F904F9028
:10D050000895CF93DF93FC0122813381232B59F173
:10D06000EC016AEB7FE18EE692E10F9406154AE04F
:10D0700050E06E818EE692E10F94D0128EE692E13E
:10D080000F94BA128C819D810F94922E70E060E013
:10D090008A819B810E94DB261D821C82EA81FB81A2
:10D0A0000190F081E02D80858F70808781E090E095
:10D0B000DF91CF91089590E080E0FACF6F927F9258
:10D0C0008F929F92AF92BF92CF92DF92EF92FF9298
:10D0D0000F931F93CF93DF93EC018C819D81892B5C
:10D0E00009F499C0EA81FB81309709F494C03A01B0
:10D0F0004B010190F081E02D8085807F803201F529
:10D10000EC81FD8180A591A5A2A5B3A5892B8A2BD1
:10D110008B2BB1F00F94B4069B01AC01EC81FD8127
:10D1200060A571A582A593A5A12CB12C650116E976
:10D13000E12EF12C00E010E00E9452D3882301F38D
:10D140008F81988521E0621A7108DC01ED91FC91D4
:10D150000280F381E02DA301B40119958F81988598
:10D16000DC01ED91FC910190F081E02DD40112964B
:10D1700060E09D01281939092615370518F42D910D
:10D18000620FF7CF19950C811D8180E00E94B4D306
:10D19000F80160A771A782A793A76FE57FE18EE6EC
:10D1A00092E10F9406154AE050E06E818EE692E11E
:10D1B0000F94D0126BE57FE18EE692E10F94061595
:10D1C0008401C8018819990986159705B8F4D80112
:10D1D0006C9140E150E06A3050F467E776E08EE60B
:10D1E00092E10F94101440E150E0F80160818EE666
:10D1F00092E10F94D0120F5F1F4FE3CF8EE692E1C2
:10D200000F94BA12EA81FB810190F081E02D8085B4
:10D210008F7080628087DF91CF911F910F91FF9077
:10D22000EF90DF90CF90BF90AF909F908F907F90C6
:10D230006F900895CF92EF92FF920F931F93CF9329
:10D24000DF9300D000D01F921F92CDB7DEB77C01D4
:10D2500009831A832B833C834D835E836F83788796
:10D2600067E470E28EE692E10F940615CE01019616
:10D270000E94AC23898181112AC00A810F7001307C
:10D2800071F128F010E00230E9F5CC20E9F060E01F
:10D29000CE0101960E94091EF70102811381892B9C
:10D2A00069F0C8010E948427672B682B692B61F401
:10D2B00080E00E94B4D3AB01BC0103C040E050E069
:10D2C000BA01C8010E94242781E090E02EC080317D
:10D2D000D0F58E30D8F58130C9F18230D9F16AE3CA
:10D2E00070E28EE692E10F9406154AE050E0698103
:10D2F0008EE692E10F94D0128EE692E10F94BA126C
:10D3000001E010E06AE270E28EE692E10F94061509
:10D310004AE050E0B8018EE692E10F94F7138EE6F2
:10D3200092E10F94BA1290E080E028960FB6F8943C
:10D33000DEBF0FBECDBFDF91CF911F910F91FF9048
:10D34000EF90CF9008958351833048F6F701028122
:10D350001381A7CF40E050E0BA01F70182819381A9
:10D36000B1CF4F925F926F927F928F929F92AF92C6
:10D37000BF92CF92DF92EF92FF920F931F93CF93C2
:10D38000DF93CDB7DEB72C970FB6F894DEBF0FBE94
:10D39000CDBF6D7F6130710509F4B2C0DC0112961A
:10D3A0002D913C912115310509F4AAC04C01C90108
:10D3B0000E9484272B013C01411451046104710433
:10D3C00009F49EC0D40118968D919D910D90BC9149
:10D3D000A02D89879A87AB87BC87892B8A2B8B2BBB
:10D3E00009F48EC00F94B4069B01AC01A12CB12CA2
:10D3F0006501E984FA840B851C85C301B2010E9492
:10D4000052D3882309F47CC0F401E280F38080E0E9
:10D410000E94B4D3AB01BC01C7010E94242719822A
:10D420001A821B821C821D821E821F8218868A819C
:10D430008F708A83D40112966D917C9140E053E005
:10D44000CE0101960E94102ECE0101960E941D2150
:10D450006B017C0168E077E08EE692E10F94101496
:10D460002AE030E0B701A6018EE692E10F94B812EF
:10D4700067E177E08EE692E10F941014F4014481A5
:10D480005581668177812AE030E08EE692E10F9443
:10D49000B8128EE692E10F94BA12F401848195815C
:10D4A000A681B781C80ED91EEA1EFB1E8A818F7025
:10D4B00080668A83CD82DE82EF82F8866281738104
:10D4C00040E052E0CE0101960E94512D6BE177E0E1
:10D4D0008EE692E10F9410142AE030E0B701A60125
:10D4E0008EE692E10F94B8128EE692E10F94BA1292
:10D4F00060E072E0D40112968D919C910E94A02E62
:10D5000090E080E02C960FB6F894DEBF0FBECDBF42
:10D51000DF91CF911F910F91FF90EF90DF90CF900F
:10D52000BF90AF909F908F907F906F905F904F9043
:10D530000895CF92DF92EF92FF920F931F93CF93B4
:10D54000DF93CDB7DEB762970FB6F894DEBF0FBE9C
:10D55000CDBF6C010B871C872D873E874F87588B6B
:10D56000698B7A8B65E270E2C7010F942F30EEE091
:10D57000F0E0892BF1F06FE170E2C7010F942F30DA
:10D58000E0E1F0E0892BA9F069E170E2C7010F94B6
:10D590002F30EFE0F0E0892B61F01F7065E170E261
:10D5A000C7010F942F30E12FF0E0892B11F4EDE04B
:10D5B000F0E09B85992341F0309731F4EF2809F48E
:10D5C00061C08FEF9FEF96C0E131F10508F03CC0DC
:10D5D0008827E251F5498F4F0D94E537E16A426B98
:10D5E000FF6A246B246B246B246BCD6B156C246B4E
:10D5F000246B246B246B246B1F6C686C2D6CCE0128
:10D600000B960E94711F20EF260F2931D0F6D6010C
:10D610001496ED91FC91159723A39B01AC01332740
:10D62000442755271296ED91FC9113970190F081B4
:10D63000E02D60817181ED91FC910684F785E02DEC
:10D6400000E317E0C6011995D6011496ED91FC91FF
:10D650001597118A1496ED91FC91159781E08187B9
:10D660001496ED91FC9115978DE482871496ED91B7
:10D67000FC9115978FE5838714966D917C9145E217
:10D6800050E033C0F601A481B58191509531E0F6A8
:10D69000E92FF0E08827E05BF4498F4F0D94E537E0
:10D6A000656B896B246B246B896B656B246B246BB6
:10D6B000246B246B246B246B246B9A6BB26B246BEE
:10D6C000246B246BAE6BAA6BB06B95968C9195977F
:10D6D0005D968C93D6011496ED91FC91858D8160B9
:10D6E000858F4DE050E06AE172E0C6010E945E68FD
:10D6F00081E090E062960FB6F894DEBF0FBECDBF1A
:10D70000DF91CF911F910F91FF90EF90DF90CF901D
:10D71000089595968C9195975D968C93D601149665
:10D72000ED91FC91858D8E7F858F4DE050E06DE011
:10D7300072E0DBCF57961C92D6011496ED91FC91C6
:10D74000159785A1858F1496ED91FC91858D81604B
:10D75000858F7ACF81E057968C93EECF82E0FBCF16
:10D7600084E0F9CF83E057968C93D6011496ED911F
:10D77000FC91159785A1858F1496ED91FC911597D5
:10D78000858D8160858F1496ED91FC91818D83301C
:10D7900009F05ACF82E0818F57CF1982F6010481B8
:10D7A00015819031B1F150F49E3091F0CE010B967D
:10D7B0000E94711FD80159966C9314C0913171F178
:10D7C0009231A1F782E0F801818F60E070E206C03B
:10D7D00083E0D80159968C9360E170E2CE01019606
:10D7E0000F943830D6011296ED91FC911397019069
:10D7F000F081E02D60817181ED91FC910288F389C7
:10D80000E02D25E337E0AE014F5F5F4FC60119956C
:10D810001BCFF801118E6BE070E2E0CF81E0D80100
:10D8200059968C9364E070E2D9CFCE010B960E949A
:10D83000711FD6011496ED91FC91678B05CFD6012F
:10D840001496ED91FC91913029F0923009F0FCCEC4
:10D85000148EFACE80E5848FF7CEF601048115810F
:10D86000913049F09230F1F0CE010B960E94711F79
:10D87000F801638FE9CE83E0D8015B968C93D601E3
:10D880000280F381E02D0190F081E02D60817181B3
:10D89000ED91FC910288F389E02D2AE337E047ED12
:10D8A0005AE0B4CFF801138ED6011296ED91FC9197
:10D8B00013970190F081E02D60817181ED91FC91D1
:10D8C0000288F389E02D2AE337E042EE5AE09ECF4A
:10D8D000D6011496ED91FC91913031F0923009F01F
:10D8E000B3CE858D877F34CF858D886031CFCF9340
:10D8F000C1E068EE73E080E090E00F9443044AE0FA
:10D9000050E06C2F8DEB91E10F94D012CF5FC431BA
:10D9100081F784EF91E0CF9108954F925F926F92DB
:10D920007F928F929F92AF92BF92CF92DF92EF92AF
:10D93000FF920F931F93CF93DF9300D000D000D0BE
:10D940001F92CDB7DEB7FC01248135812115310549
:10D9500009F4BDC282819381DC018D919C91DC012F
:10D9600018969C91959595959595959509F4AFC2C6
:10D970003B014F019230A9F5F90180A591A5A2A51F
:10D98000B3A5892B8A2B8B2B61F10F94B4069B01D5
:10D99000AC01D40114964D905C90F20160A571A584
:10D9A00082A593A5A12CB12C650116E9E12EF12CDD
:10D9B00000E010E00E9452D3882399F0D40112961F
:10D9C000ED91FC910190F081E02D80858F70806158
:10D9D000808780E00E94B4D3F20160A771A782A77C
:10D9E00093A790E080E06A94672809F072C2D4019E
:10D9F0001296ED91FC910190F081E02D8085807F61
:10DA0000803131F50F94B4069B01AC01D40114961A
:10DA1000ED91FC9160A571A582A593A5A12CB12CD7
:10DA2000650118E8E12E13E1F12E00E010E00E94FC
:10DA300052D3882369F064EF7FE18EE692E10F9480
:10DA4000DA194DE050E060E072E0C4010E945E68C7
:10DA5000F40187819085DC01ED91FC910084F185D2
:10DA6000E02D199585970CF4F2C1F401648175815C
:10DA700045E250E0878190850F94C111D40117963B
:10DA80008D919C91DC01ED91FC910084F185E02D5C
:10DA900019957C01892B89F062E070E080E090E0CC
:10DAA0000F944304F40187819085DC01ED91FC9192
:10DAB0000284F385E02D1995E1CF6FEE7FE18EE6CC
:10DAC00092E10F9406154AE050E0F40166818EE67B
:10DAD00092E10F94D0126AEE7FE18EE692E10F940C
:10DAE0000615D4011496ED91FC91EE0DFF1D608199
:10DAF00040E150E06A3078F467E776E08EE692E144
:10DB00000F941014D4011496ED91FC91EE0DFF1DAD
:10DB100040E150E060818EE692E10F94D012BFEFB9
:10DB2000EB1AFB0AE4E2EE16F104D9F6D4011496DE
:10DB3000ED91FC91159784A197A1891709F483C1F0
:10DB400087A31496ED91FC9183A190E02C01B0E1A4
:10DB50004B0E511C499708F070C17584878986A3C4
:10DB6000E18CF12C638CD40114962D913C91858D20
:10DB7000D90195968C93048D10E0878DF401A281D4
:10DB8000B381208131810D90BC91A02D6D917C914C
:10DB9000D9015296ED91FC9121E437E047ED5AE02E
:10DBA00080FD02C042EE5AE0C4011995003811050B
:10DBB00009F050C1D4011296ED91FC911397019098
:10DBC000F081E02D60817181ED91FC910288F389F3
:10DBD000E02D28E437E047ED5AE0C40119956EE4E2
:10DBE00077E08EE692E10F941014D4011496ED9133
:10DBF000FC914AE050E065A18EE692E10F94D012CC
:10DC00008EE692E10F94BA12D4011496ED91FC9134
:10DC1000159785A112960D90BC91A02DF40120813D
:10DC200031810D90BC91A02D6D917C91D9015296BE
:10DC3000ED91FC9129E537E047ED5AE083FD02C004
:10DC400042EE5AE0C4011995D401ED91FC9111976F
:10DC50000288F389E02D12968D919C91DC018D91C3
:10DC60009C91DC016D917C91D40114968D919C91D5
:10DC7000DC0195968C9120E637E047ED5AE081FD76
:10DC800002C042EE5AE0C4011995262D30E050E062
:10DC900040E0D4011296ED91FC9113970190F08130
:10DCA000E02D60817181ED91FC910684F785E02D76
:10DCB0000AE317E0C4011995F401228133818081C0
:10DCC0009181E114F10409F0DCC0F901A081B18176
:10DCD0006D917C91DC015296ED91FC9125E337E04A
:10DCE0004CE657E0C4011995D401ED91FC911197D0
:10DCF0000288F389E02D12968D919C91DC018D9123
:10DD00009C91DC016D917C912AE337E042EE5AE070
:10DD1000662011F047ED5AE0C40119959201550CA7
:10DD2000440B550BD4011296ED91FC911397019081
:10DD3000F081E02D60817181ED91FC910684F78581
:10DD4000E02D00E317E0C4011995BFEF7B16B9F091
:10DD5000272D30E050E040E0D4011296ED91FC9187
:10DD600013970190F081E02D60817181ED91FC911C
:10DD70000684F785E02D01E817E0C40119951982A2
:10DD8000D4011496ED91FC9186A160E170E28823A4
:10DD9000A1F06EED7FE1813081F069ED7FE18230AD
:10DDA00061F060ED7FE1833041F06CEC7FE1843025
:10DDB00021F08D3631F468EC7FE1CE0101960F94AD
:10DDC0003830D4011496ED91FC91159726A130E0DE
:10DDD00050E040E01296ED91FC9113970190F08194
:10DDE000E02D60817181ED91FC910684F785E02D35
:10DDF00007E817E0C4011995D4011496ED91FC9140
:10DE0000159785A112960D90BC91A02DF40120814B
:10DE100031810D90BC91A02D6D917C91D9015296CC
:10DE2000ED91FC912DE837E0AE014F5F5F4F80FD33
:10DE300002C042EE5AE0C401199563EE7FE18EE61E
:10DE400092E10F9406158EE692E10F94BA1281E0EA
:10DE500090E03FC0012B09F0C2CED4011296ED91A3
:10DE6000FC9113970190F081E02D60817181ED911B
:10DE7000FC910288F389E02D28E437E042EE5AE075
:10DE8000ACCEDC015296ED91FC91D9018D919C9123
:10DE9000DC016D917C9125E337E041E757E0B1E08B
:10DEA000EB16F10409F41ECF22E0E216F10429F486
:10DEB00025E337E048E757E015CF83E0E816F104A3
:10DEC00009F012CF25E337E04CE757E00BCF8FEF97
:10DED0009FEF2A960FB6F894DEBF0FBECDBFDF913D
:10DEE000CF911F910F91FF90EF90DF90CF90BF9057
:10DEF000AF909F908F907F906F905F904F9008951C
:10DF00000F931F93CF93DF93DC0112962D913C91D9
:10DF1000232B81F1EC016FEA7FE18EE692E10F9411
:10DF200006154AE050E06E818EE692E10F94D01221
:10DF30008EE692E10F94BA128C819D81892B61F457
:10DF40000A811B818CE290E00F94F62DBC01C80180
:10DF50000E94DB269D838C83EC81FD81309769F4E0
:10DF60006DE97FE187EC91E10F94061587EC91E173
:10DF70000F94BA1290E080E041C085E2DF011D926B
:10DF80008A95E9F7EC81FD8116A2EC81FD8115A24D
:10DF9000EC81FD8117A20C811D8180E00E94B4D329
:10DFA000F80160A771A782A793A78E81811112C083
:10DFB00062E00F94FE0164E67FE18DEB91E10F9446
:10DFC00006158DEB91E10F94BA121092310281E0A7
:10DFD00080938A0C26E040E855E260E070E08F8193
:10DFE00098850E9431B9EA81FB810190F081E02D92
:10DFF00080858F708061808781E090E0DF91CF9194
:10E000001F910F910895EF92FF921F93CF93DF938B
:10E01000192F7B01C82FD92FD7FF03C0D195C195E8
:10E02000D10961E08C2F0F94FE0182E0E816F10423
:10E0300099F460E08C2F0F94D00160EB7DE18EE6C7
:10E0400092E10F9406158EE692E1DF91CF911F9138
:10E05000FF90EF900D94BA12612FEF2851F4609564
:10E06000661F6627661F8C2F0F94D0016CEA7DE136
:10E07000E6CF661F6627661F8C2F0F94D00167EAD4
:10E080007DE1DDCF60E08DE00D94D00161E08DE0B9
:10E090000D94D0012F923F924F925F926F927F9298
:10E0A0008F929F92AF92BF92CF92DF92EF92FF92A8
:10E0B0000F931F93CF93DF93CDB7DEB766970FB65D
:10E0C000F894DEBF0FBECDBF4C0180916F0C64E4AD
:10E0D0007FE1882309F47DC160E083E00F94D001E3
:10E0E00061E070E080E090E00F944304BE016F5F58
:10E0F0007F4F80E00E943DFE892B09F068C1898135
:10E1000083FF65C144E0BE016F5F7F4F82E00E94E4
:10E11000E8FD009791F429813A813227232732279D
:10E120003093DD0F2093DC0F2B813C813227232796
:10E1300032273093DB0F2093DA0F0F94DA1462E961
:10E1400077E08EE692E10F9410146091DC0F7091ED
:10E15000DD0F90E080E00F942936362E272E898B34
:10E16000492E462F572F682F792F8EE692E10F9474
:10E17000DE1268E977E08EE692E10F941014609168
:10E18000DA0F7091DB0F90E080E00F942936562E65
:10E190007A8B8B8B9C8B462F572FBC018EE692E19E
:10E1A0000F94DE1260EA77E08EE692E10F9410148D
:10E1B00042E0BE016F5F7F4F81E10E94E8FD49812F
:10E1C0005A81542745275427892B11F050E040E00D
:10E1D00070E060E040936B0C50936C0C60936D0C9E
:10E1E00070936E0C2AE030E08EE692E10F94AF134C
:10E1F00020E030E44CE156E4632D722D8989942DA2
:10E200000F94243687FF78C0D4011296ED91FC91CB
:10E21000608071806CEA77E0C3010E9441F99E8BB7
:10E220008D8B60EB77E0C3010E9441F93C011982BC
:10E230001A821B821C828A818F708067F82E8A83E3
:10E24000232D832D922DA989B42D8D839E83AF8399
:10E25000B887B12CA12CD12CC12CE9800B811C8159
:10E260003E814F8158856FEF8D899E890E9428E1FC
:10E2700019821A821B821C828A818F708067F82E15
:10E280008A83252D852D9A89AB89BC898D839E83B0
:10E29000AF83B887E9800B811C813E814F8158850F
:10E2A0006FEFC3010E9428E125EB37E0432D522D8B
:10E2B0006989742DC4010E94F8382AEB37E0452D96
:10E2C0005A896B897C89C4010E94F83860916B0C73
:10E2D00070916C0C80916D0C90916E0C2AE0AE01E7
:10E2E0004F5F5F4F0F94D33040EC57E0BE016F5F3C
:10E2F0007F4FC4010E94C23866EC77E08EE692E15F
:10E300000F94BE12BE016F5F7F4F80EE0E943DFEF4
:10E31000892B19F419811F3F29F568EC77E08EE607
:10E3200092E10F94BE1261E083E00F94D00181E08E
:10E3300090E066960FB6F894DEBF0FBECDBFDF91BA
:10E34000CF911F910F91FF90EF90DF90CF90BF90F2
:10E35000AF909F908F907F906F905F904F903F9085
:10E360002F90089515FF06C069EE77E08EE692E1E2
:10E370000F94101414FF06C06DEF77E08EE692E163
:10E380000F94101413FF06C060E178E08EE692E16E
:10E390000F94101412FF06C065E278E08EE692E159
:10E3A0000F94101411FF06C06CE378E08EE692E142
:10E3B0000F94101410FF06C062E578E08EE692E13B
:10E3C0000F9410148EE692E10F94BA12ACCF69E26A
:10E3D0007FE18EE692E10F9406158EE692E10F94AE
:10E3E000BA1290E080E0A5CF2F923F924F925F92B9
:10E3F0006F927F928F929F92AF92BF92CF92DF9255
:10E40000EF92FF920F931F93CF93DF93CDB7DEB7B9
:10E410002E970FB6F894DEBF0FBECDBF61307105E9
:10E4200079F42C0180916A0C811125C061E17FE1B2
:10E430008EE692E10F9406158EE692E10F94BA12E1
:10E4400090E080E02E960FB6F894DEBF0FBECDBFF1
:10E45000DF91CF911F910F91FF90EF90DF90CF90C0
:10E46000BF90AF909F908F907F906F905F904F90F4
:10E470003F902F90089564E678E08EE692E10F9445
:10E48000101482E00F947604892E912C40E150E024
:10E49000B4018EE692E10F94FE138FEF881691047B
:10E4A00009F42CC160E778E08EE692E10F94101435
:10E4B00080E00F947604BC0190E080E00F94293650
:10E4C00020E030E040E857E30F948A3620E030E067
:10E4D00045E253E40F948A3620E030E040E252E413
:10E4E0000F941738962E672E782E892E462F572F89
:10E4F000682F792F8EE692E10F94DE1264E778E0C0
:10E500008EE692E10F94101481E00F947604BC0122
:10E5100090E080E00F94293620E030E040E857E3B7
:10E520000F948A3620E030E048EC52E40F948A36AB
:10E53000362E272E89879A87462F572FBC018EE6C5
:10E5400092E10F94DE126BE778E08EE692E10F9491
:10E55000BE12D2011296ED91FC91E080F18062E84A
:10E5600077E0C7010E9441F99C878B8769EB76E0D1
:10E57000C7010E9441F99E878D87292D362D472D91
:10E58000582D692D762D872D982D0F948C3981115A
:10E590003EC019821A821B821C828A818F7080671A
:10E5A000F82E8A83292D892D962DA72DB82D8D83A0
:10E5B0009E83AF83B887B12CA12CD12CC12CE980CC
:10E5C0000B811C813E814F8158856FEF8B859C8527
:10E5D0000E9428E119821A821B821C828A818F7014
:10E5E0008067F82E8A83232D832D922DA985BA85E5
:10E5F0008D839E83AF83B887E9800B811C813E8128
:10E600004F8158856FEF8D859E850E9428E12DE70B
:10E6100038E0492D562D672D782DC2010E94F8381B
:10E6200020E838E0432D522D69857A85C2010E9489
:10E63000F83880916F0C882309F45DC020E030E049
:10E6400048EC51EC692D762D872D982D0F942436AA
:10E6500087FD51C020E030E048E452E4692D762D7A
:10E66000872D982D0F942C3918160CF444C020E0F7
:10E6700030E048EC52E4632D722D89859A850F9421
:10E680002C391816C4F120E030E04AE754E4632D39
:10E69000722D89859A850F948A360F94FD386650BD
:10E6A0007F4F8F4F9F4F24EFC22EDD24D394E12C58
:10E6B000F12CA70196010F946E3729831A8220E06E
:10E6C00030E04AE754E4692D762D872D982D0F947C
:10E6D0008A360F94FD386E557D498F4F9F4FA701A5
:10E6E00096010F946E372B831C82BE016F5F7F4FA4
:10E6F00085E00E94AEFD88EE93E0A4CE63E878E06A
:10E700008EE692E10F94BE1281E00F945303F3CF93
:10E71000EF92FF920F931F93CF93DF93CDB7DEB7A6
:10E7200060970FB6F894DEBF0FBECDBF80916A0C24
:10E730008823C9F062EF7EE18EE692E10F94061520
:10E740008EE692E10F94BA1290E080E060960FB6E8
:10E75000F894DEBF0FBECDBFDF91CF911F910F9117
:10E76000FF90EF9008956DE878E08EE692E10F94C7
:10E77000BE120E948DFE80E48093E60F0E948DFE03
:10E7800010E01B7F8091E60F0E94A4FD62E083EC05
:10E790009FE00E940BAB612F83EC9FE00E940BABCC
:10E7A00060E083EC9FE00E940BAB83EC9FE00E9453
:10E7B0003ED06AE070E080E090E00F9443046BE9A3
:10E7C00078E08EE692E10F9410148EEF0F947604A9
:10E7D000AC0170E060E020E18EE692E10F946C12F3
:10E7E0008EE692E10F94BA126EEA78E08EE692E13C
:10E7F0000F9410148FEF0F947604AC0170E060E07A
:10E8000020E18EE692E10F946C128EE692E10F9475
:10E81000BA126BEB78E08EE692E10F9410148BEF56
:10E820000F947604182F092F8CEF0F947604F82E8E
:10E83000E92E8DEF0F9476049F938F93EF92FF92C2
:10E840000F931F9381ED98E09F938F938E010F5F3D
:10E850001F4F1F930F930F94D73CB8018EE692E1A0
:10E860000F94BE1281E080936A0C0FB6F894DEBF5D
:10E870000FBECDBF81E090E069CF0F931F93CF9380
:10E88000DF9300D000D01F92CDB7DEB780916F0C20
:10E89000882369F064ED7EE187EC91E10F94061521
:10E8A00087EC91E10F94BA1290E080E0BBC061E088
:10E8B00083E00F94FE0160E083E00F94D00160EEEE
:10E8C00078E08DEB91E10F94BE120E948DFE88ECF2
:10E8D0008093B8008091060490910704A0910804E9
:10E8E000B091090489839A83AB83BC8383EC9FE056
:10E8F0009093D00F8093CF0F1E8280E197E22E81FC
:10E900002F5F2E830197D9F71D82BE016B5F7F4F6A
:10E9100080E20E943DFE8C01892BF1F48D8101E0A3
:10E9200010E08138C9F4BE016F5F7F4F8FEF0E9406
:10E93000AEFD1F8280E89EE32F812F5F2F8301971A
:10E94000D9F7BE016B5F7F4F80E00E943DFE8D8155
:10E9500080FF0CC003E010E06CEE78E087EC91E102
:10E960000F941014C8010F94DA149ECFBE016B5F90
:10E970007F4F80E00E943DFE892B61F78D8184FFEF
:10E98000E9CF8091D10F0E94A4FD8091CF0F90918B
:10E99000D00FDC01ED91FC910190F081E02D64EF4E
:10E9A00019958091CF0F9091D00F0E943ED088236F
:10E9B00019F002E010E0D0CFBE016B5F7F4F81E025
:10E9C0000E943DFE8C01892B39F61D811F78106154
:10E9D0001D838091D10F0E94A4FD8091CF0F909153
:10E9E000D00FDC01ED91FC910190F081E02D61E010
:10E9F00019958091CF0F9091D00FDC01ED91FC9192
:10EA00000190F081E02D612F19958091CF0F9091A9
:10EA1000D00F0E943ED08111CCCF81E080936F0C4B
:10EA200081E090E027960FB6F894DEBF0FBECDBF11
:10EA3000DF91CF911F910F910895CF93DF9300D075
:10EA400000D01F921F92CDB7DEB7E7EAF1E1128A3C
:10EA5000118A80E090E19587848784E890E0948B28
:10EA6000838B81E0868787E7858B1C821B8284EEFF
:10EA700094E09A838983FE83ED838FEF9FEF9887DD
:10EA80008F8367E47EE18DEB91E10F940615609131
:10EA9000DA0B7091DB0BCE0101960E94DCBC87EA99
:10EAA00091E10E94E91667E37EE18DEB91E10F941D
:10EAB00006158DEB91E10F94BA120F943516289636
:10EAC0000FB6F894DEBF0FBECDBFDF91CF91089592
:10EAD000CF93DF93EB010297B4F167E87AE18A8183
:10EAE0009B810F941130892B29F40F94E4116F77D7
:10EAF0000E948EFC63E87AE18A819B810F94113039
:10EB0000892B29F40F94E41160680E948EFC6BE855
:10EB100079E18DEB91E10F9406150F94E411609566
:10EB2000661F6627661F70E04AE050E08DEB91E1BA
:10EB30000F94F7138DEB91E10F94BA1288EC90E0EB
:10EB4000DF91CF9108950E941D75F8CFEF92FF924B
:10EB50000F931F93CF93DF9300D000D01F92CDB7B8
:10EB6000DEB77B01CE0107969F938F9301979F930A
:10EB70008F9301979F938F9301979F938F93019703
:10EB80009F938F9301979F938F938E010F5F1F4FDA
:10EB90001F930F938FEF98E09F938F93DB01139652
:10EBA0008C9113978F9312968C918F930F94073DAE
:10EBB0000FB6F894DEBF0FBECDBF0697ECF469E147
:10EBC0007AE187EC91E10F940615D70112966D91C9
:10EBD0007C9187EC91E10F94101480E991E02796E5
:10EBE0000FB6F894DEBF0FBECDBFDF91CF911F915E
:10EBF0000F91FF90EF9008958091991190919A1143
:10EC0000892B09F449C00E9495FA882309F444C06D
:10EC1000A0919911B0919A1152961C921E925197FF
:10EC200054961C921E92539784E890E01D969C93F4
:10EC30008E931C971E961C921E9781E655968C9378
:10EC40005597ED91FC9111970088F189E02D64E0D2
:10EC500070E0CD0119958091991190919A11DC0184
:10EC6000ED91FC910280F381E02D46E050E0B80187
:10EC7000199586E0F801A1EAB1E101900D928A951B
:10EC8000E1F78091991190919A11DC01ED91FC913D
:10EC90000488F589E02D19950E94FC326BE27AE137
:10ECA0008DEB91E10F94061588EC90E098CF892BBD
:10ECB00071F0FB01828193810F94791463E07AE112
:10ECC0008DEB91E10F94061588EC90E0089590E0AB
:10ECD00080E0F2CF892B71F0FB01828193810F9448
:10ECE00018146CEE79E18DEB91E10F94061588EC28
:10ECF00090E0089590E080E0F2CF8091991190919A
:10ED00009A11892B51F00F94AB15882331F06CEDDB
:10ED100079E18DEB91E10F9406151092B9111092E3
:10ED2000B81180E090E19093B4118093B31184E81E
:10ED300090E09093BB118093BA1181E08093B5115C
:10ED400082E78093BC1187EA91E10E94241687EA4A
:10ED500091E10E94E91688EC90E00895EF92FF920D
:10ED60000F931F93CF93DF93CDB7DEB72C970FB6DA
:10ED7000F894DEBF0FBECDBF8C017B018DED95E019
:10ED80009A8389831B821C821D821E8298878F83AF
:10ED900019861A861B861C8605301105ECF0BE010B
:10EDA000695F7F4FF701808591850E9417DA892B73
:10EDB00099F0CE0107960E9453FBBE01695F7F4F19
:10EDC000F701868197810E9417DA892B61F0CE01C5
:10EDD00007960E9425FC0EC0CE0101960E9453FBAF
:10EDE0000430110554F7CE0101960E9425FC033032
:10EDF0001105A4F1BE01695F7F4FF7018481958100
:10EE00000E9417DA892B51F1CE0107960E94BCFBB4
:10EE1000BE01695F7F4FF701828193810E9417DAFB
:10EE2000892B19F1CE0107960E94EAFA65EC79E187
:10EE30008DEB91E10F94061580E00F943E1288EC63
:10EE400090E02C960FB6F894DEBF0FBECDBFDF91D9
:10EE5000CF911F910F91FF90EF900895CE010196F1
:10EE60000E94BCFB023011059CF6CE0101960E9467
:10EE7000EAFA01301105D1F6CE0101960E94EAFAB4
:10EE80006CEC79E18DEB91E10F940615CFCF0F93E8
:10EE90001F93CF93DF938C01EB010297C4F08A811B
:10EEA0009B810F94C32F8093310299270F944712AF
:10EEB0000230110549F08C819D810F94C32F8093FE
:10EEC000300299270F945112C8ECD0E002C0C0E97B
:10EED000D1E061EB79E18DEB91E10F9406154AE009
:10EEE00050E0609131028DEB91E10F94D0126CE90A
:10EEF00079E18DEB91E10F9406154AE050E06091C5
:10EF000030028DEB91E10F94D0128DEB91E10F94D3
:10EF1000BA12CE01DF91CF911F910F9108958F9278
:10EF20009F92AF92BF92CF92DF92EF92FF920F9398
:10EF30001F93CF93DF93CDB7DEB7E0970FB6F8946A
:10EF4000DEBF0FBECDBF4B0169017A0194E0EAE05C
:10EF5000F4E0DE01119601900D929A95E1F7FE0121
:10EF600035968CE1DF011D928A95E9F7AE014F5F7E
:10EF70005F4F68E0C4010E943ADC1A8A8091DA0B84
:10EF80009091DB0B892B09F46BC08EE692E10F9414
:10EF9000BA1261ED74E18EE692E10F940615B701A5
:10EFA000A6018EE692E10F94DE126FEC74E18EE61C
:10EFB00092E10F940615BE016F5F7F4F8EE692E1DE
:10EFC0000F9410146DEC74E18EE692E10F94061527
:10EFD0008EE692E10F94BA12BE016F5F7F4F80916F
:10EFE000FB0D9091FC0D0E9441F94C0120E030E0B6
:10EFF0004EEF52ECC701B6010F942436882381F1FD
:10F0000020E030E04AEA52E4C701B6010F9424360A
:10F01000882331F120E030E0A901C701B6010F9447
:10F0200024368823E9F019A61AA61BA61CA68AA5D1
:10F030008F7080678AA7CDA6DEA6EFA6F8AA63E048
:10F04000CE0189960E94231BB12CA12CD12CC12C5E
:10F0500079018A019B01AC016FEFC4010E9428E194
:10F06000E0960FB6F894DEBF0FBECDBFDF91CF9113
:10F070001F910F91FF90EF90DF90CF90BF90AF90D6
:10F080009F908F9008950F931F93CF93DF938C01E0
:10F09000D0E0C0E001151105B1F0BE016C577F4D05
:10F0A000C8010F942F30892B51F4FE01E857FF4D12
:10F0B000849190E0DF91CF911F910F910895259653
:10F0C000C233D10539F781E090E0F4CF2F923F921F
:10F0D0004F925F926F927F928F929F92AF92BF9268
:10F0E000CF92DF92EF92FF920F931F93CF93DF9314
:10F0F000CDB7DEB7CB56D1090FB6F894DEBF0FBE41
:10F10000CDBF6B969FAF8EAF6B9767965FAF4EAFDD
:10F110006797922EA2961FAF0EAFA297A896FFAE4A
:10F12000EEAEA8976C96CFAE6C976596BFAEAEAEBE
:10F130006597DC011496ED91FC910784F089E02D30
:10F1400066807780AB2839F4FE01EE5AFF4F659652
:10F15000FFAFEEAF659781E06596AEADBFAD659749
:10F160008C931B01512C412C6114710409F4CAC504
:10F17000B2E09B1641F0E3E09E1609F487C0F3016C
:10F1800062807380F1CF6CE179E0C3010E9441F9A4
:10F190000097A9F3FC0181859285A385B48582152A
:10F1A0009305A405B50559F763E179E0C3010E9411
:10F1B00041F97C0161EB76E0C3010E9441F94C0109
:10F1C00069E378E0C3010E9441F96E969FAF8EAF6C
:10F1D0006E976B96AEADBFAD6B971296ED91FC91AD
:10F1E00062E0828193810E94F3F9A0969FAF8EAF77
:10F1F000A0976696BFAD66970FEF1FEFB03458F437
:10F200006796EEADFFAD6797FF27EE0FFF1FE05F3C
:10F21000FF4E078110852D961CAE1DAE1EAE1FAE93
:10F220002D9761961CAE1DAE1EAE1FAE61972B963C
:10F230008FAD2B978F702B968FAF2B9762961FAE4B
:10F240006297E114F10429F1F70180858F70843011
:10F2500001F5818592850E944378F82EEFEFE80F43
:10F26000EA3008F050C10E2E000CFF0B8827E45C3A
:10F27000F6488F4F0D94E5374979F879D5790D7AAD
:10F28000837A837A397A257A4E7A657A64E279E0EC
:10F290007CCF1801512C412C2B968FAD2B978F7062
:10F2A000806A2B968FAF2B97012E000C220B330B0D
:10F2B00061960CAF1DAF2EAF3FAF6197FF24F39463
:10F2C00062E472E28EE692E10F94061500E020E01F
:10F2D00033E040E150E0BE016F5F7F4FCE01875BBE
:10F2E0009F4F0E948B21BC018EE692E10F94101477
:10F2F0006BE372E28EE692E10F9406156F2DFF0C20
:10F30000770B4AE050E08EE692E10F94F71369E341
:10F3100072E28EE692E10F940615D3016D917C9115
:10F320008EE692E10F9410148EE692E10F94BA12D9
:10F330008114910409F4BBC1F40180858F7085505C
:10F34000823008F0B4C16EE877E0C4010E9441F950
:10F35000FC01892B09F4FBC190859295907F9595CE
:10F36000959595959595943009F40FC1953009F0D0
:10F37000EEC1068117810115110509F4E8C1D80114
:10F3800018968C9118978F70823019F412960D91FF
:10F390001C910115110509F4DAC1F80180858F70FF
:10F3A000853009F4B4C0D801F1CF1801512C412C9B
:10F3B000B201A801CE01875B9F4F0E94871D229654
:10F3C0002FAF229723963FAF239724964FAF2497D2
:10F3D00025965FAF259726966FAF269727967FAF26
:10F3E000279728968FAF289729969FAF299768CFA0
:10F3F0001027012710271801512C412C2B968FAD77
:10F400002B978F70806A2B968FAF2B9761962CAEBF
:10F410003DAE4EAE5FAE619753CF10270127102748
:10F420001801512C412CB201A101CE01875B9F4FE5
:10F430000E94871D29AF3AAF4BAF5CAF6DAF7EAF77
:10F440008FAF21969FAF21973BCF11271801512CE9
:10F45000412CB201A801CE01875B9F4F0E94871DFE
:10F4600029AB3AAB4BAB5CAB6DAB7EAB8FAB98AF24
:10F4700027CF012F11271801512C412CB201A801CF
:10F48000CE01875B9F4F0E94871D29A73AA74BA7F4
:10F490005CA76DA77EA78FA798AB12CF1801512C40
:10F4A000412C2B968FAD2B978F7080662B968FAF4C
:10F4B0002B972AE030E0D8010F94FC3761966CAFAF
:10F4C0007DAF8EAF9FAF6197FBCE1801512C412CC1
:10F4D0002B968FAD2B978F7080672B968FAF2B97C6
:10F4E000B801110F880B990B0F942B3620E030E0F8
:10F4F00048EC52E40F94843861966CAF7DAF8EAFC8
:10F500009FAF6197DDCE212C312C2101D9CEC801CE
:10F510000E9485FA823009F046CF60E0C8010E945F
:10F52000F3F96C010E94972461E0C8010E94F3F98D
:10F530007C01FC0180858F70823009F034CFCE01D0
:10F54000875B9F4F0E94711FD70119962D913D91A6
:10F550004D915C911C97621773078407950709F01A
:10F5600022CFC114D10409F4F2C0198A1A8A1B8A65
:10F570001C8A1D8A1E8A1F8A188E8A898F708A8B20
:10F58000F6016185CE01419651C066E377E0818541
:10F5900092850F94523C892B09F0D9C0CE01875B2C
:10F5A0009F4F0E94711F611571058105910509F436
:10F5B000B4C0660F771F881F991F2FEF30E040E01F
:10F5C00050E00F94903757FD16C0233031054105A8
:10F5D00051050CF088C0DA01C9010196A11DB11DC9
:10F5E00082309105A105B10509F463C00397A10517
:10F5F000B10509F478C0198A1A8A1B8A1C8A1D8AE7
:10F600001E8A1F8A188E8A898F708A8B67E0CE01C6
:10F6100041960E94231B298F3A8F4B8F5C8F6D8FF1
:10F620007E8F8F8F98A362E1CE0149960E944A1B7C
:10F6300029A33AA34BA35CA36DA37EA38FA398A792
:10F640008DA19EA1AFA1B8A52A962FAF2A972B9680
:10F650003FAF2B972C964FAF2C972D965FAF2D97E2
:10F6600061968CAF9DAFAEAFBFAF6197211103C064
:10F67000307F09F47FC16AE272E28EE692E10F9474
:10F68000061500E020E033E040E150E0BE016F5F8E
:10F690007F4FCE01875B9F4F0E948B21BC018EE67E
:10F6A00092E10F9410148EE692E10F94BA1210E0DA
:10F6B000E4C1198A1A8A1B8A1C8A1D8A1E8A1F8A1B
:10F6C000188E8A898F708A8B67E0CE0141960E94DE
:10F6D000231B298F3A8F4B8F5C8F6D8F7E8F8F8F7F
:10F6E00098A361E1A1CF198A1A8A1B8A1C8A1D8AF4
:10F6F0001E8A1F8A188E8A898F708A8B67E0CE01D6
:10F7000041960E94231B298F3A8F4B8F5C8F6D8F00
:10F710007E8F8F8F98A360E187CF198A1A8A1B8A00
:10F720001C8A1D8A1E8A1F8A188E8A898F708A8B6E
:10F7300067E0CE0141960E94231B298F3A8F4B8FA1
:10F740005C8F6D8F7E8F8F8F98A362E06DCF63E7A4
:10F7500076E0C4010E9441F98C01009709F4F7C0DA
:10F76000DC0118968C918F70853009F0E0C0C801DB
:10F770000E9485FA843009F0EAC060E0C8010E9466
:10F78000F3F97C0161E0C8010E94F3F94C0162E0E9
:10F79000C8010E94F3F9DC0119962D913D914D911C
:10F7A0005C911C9769962CAF3DAF4EAF5FAF6997E8
:10F7B00063E0C8010E94F3F98C01CE01875B9F4F83
:10F7C0000E94711F69962CAD3DAD4EAD5FAD69973E
:10F7D00062177307840795079CF4198A1A8A1B8A93
:10F7E0001C8A1D8A1E8A1F8A188E8A898F708A8BAE
:10F7F00040E050E0BA01CE0141960E94871D18CF2B
:10F80000D7011996CD90DC90F4010184F285E02DAA
:10F81000AA96FFAFEEAFAA97D80119960D90BC91AA
:10F82000A02DAC96BFAFAEAFAC97198A1A8A1B8ACF
:10F830001C8A1D8A1E8A1F8A188E8A898F708A8B5D
:10F8400046010D2C000CAA08BB086796EEACFFAC75
:10F8500067970F2C000C000B110BA696ECAEFDAEBB
:10F860000EAF1FAFA697CE01875B9F4F0E94711FFF
:10F870009B01AC012E193F09400B510BAA960EAD0E
:10F880001FADAA97B801110F880B990B6819790958
:10F890008A099B090F945E37AC96EEACFFACAC972F
:10F8A0009701FF0C440B550BA696ECACFDAC0EADCE
:10F8B0001FADA6972E193F09400B510B0F9490379F
:10F8C000820E931EA41EB51EAA968EAD9FADAA975A
:10F8D0008C199D09AC966EAD7FADAC9767960EAD59
:10F8E0001FAD6797601B710B0F94D13777FF02C074
:10F8F0006F5F7F4F75956795CB01770FAA0BBB0B99
:10F90000880E991EAA1EBB1EB7FC0CC0A401B5012F
:10F910001FEF81169104A104B10409F00CF46BCF20
:10F920004FEF01C040E050E060E070E064CF811133
:10F930000EC0198A1A8A1B8A1C8A3A893F703A8B30
:10F9400029894B895C8980E090E0DC017DCE2A9694
:10F950002FAD2A972B963FAD2B972C964FAD2C971A
:10F960002D965FAD2D9761968CAD9DADAEADBFADC3
:10F9700061976ACE68E179E0C3010E9441F98C0188
:10F9800082E0982E01151105A1F460E279E0C3012F
:10F990000E9441F98C0193E0992E0115110549F45B
:10F9A00069EF71E287EC91E10F94061587EC91E124
:10F9B0007CCED80118968C9118978F70823081F781
:10F9C00019968D919D910D90BC91A02DA296EEADB2
:10F9D000FFADA297AF0170E060E084179507A6071E
:10F9E000B707F4F2A896EEACFFACA897A70170E0B9
:10F9F00060E0481759076A077B0794F26EE072E2ED
:10FA00008EE692E10F9406158EE692E10F94BA12FB
:10FA1000D80119966D917C91AB01A296EEADFFAD28
:10FA2000A2974E1B5F0B8E010F5A1F4F5801C12C1E
:10FA3000A896EEACFFACA8978F01292D6B968EADE2
:10FA40009FAD6B970E9466782A962FAF2A972B96C8
:10FA50003FAF2B972C964FAF2C972D965FAF2D97DE
:10FA60002E966FAF2E972F967FAF2F9760968FAF02
:10FA7000609761969FAF619711E06C962FAD6C9780
:10FA80002223E9F06E964EAD5FAD6E97411551059C
:10FA9000B1F0DA0118968C918F70823081F4FA01FE
:10FAA00081859285A385B48581309105A105B10535
:10FAB00009F47BC00297A105B10509F485C0A096A1
:10FAC000EEACFFACA097E114F10409F442C0D701F9
:10FAD00018968C918F708630E1F5F3016081718109
:10FAE000C7010E9441F94C01009799F1DC01189679
:10FAF0008C9118978F70F82C092D853029F4169663
:10FB0000FC90169717960C9169E776E08F2D902F51
:10FB10000E9441F9FC01892B09F497C080858F7000
:10FB2000823009F05EC081859285A385B4858215F7
:10FB30009305A405B50509F050C06596EEADFFAD7F
:10FB400065971082112329F06C96FFAD6C97F11127
:10FB500096C088E0FE01E75BFF4FDE015196019001
:10FB60000D928A95E1F729893A894B895C896D89DB
:10FB70007E898F89988DC559DF4F0FB6F894DEBF07
:10FB80000FBECDBFDF91CF911F910F91FF90EF90EE
:10FB9000DF90CF90BF90AF909F908F907F906F90AD
:10FBA0005F904F903F902F9008956B96AEADBFAD94
:10FBB0006B9712966D917C9140E051E0CE01875B8E
:10FBC0009F4F0E94512D7BCF6B96EEADFFAD6B9793
:10FBD0006281738140E052E0F1CF21863286438614
:10FBE00054861111B1CF6596AEADBFAD65978C91BE
:10FBF000882309F4AECF67E279E08F2D902F0E9421
:10FC000041F93C01009709F48CC0FC0180858F709C
:10FC1000823009F062C081859285A385B485821502
:10FC20009305A405B50509F058C063EC71E28EE6B2
:10FC300092E10F9406158EE692E10F94BA12659642
:10FC4000AEADBFAD65971C9284CF6AEE71E28EE6D1
:10FC500092E10F940615D3016D917C918EE692E1AD
:10FC60000F9410148EE692E10F94BA12A201910142
:10FC700069E776E08F2D902F0E9410FDB2CF62963B
:10FC80008FAD6297811108C06596EEADFFAD6597A7
:10FC90008081882309F45DCFB12CA12CD12CC12CFB
:10FCA0002A96EFAC2A972B96FFAC2B972C960FAD8C
:10FCB0002C972D961FAD2D972E962FAD2E972F9604
:10FCC0003FAD2F9760964FAD609761965FAD61979E
:10FCD0006FEFC4010E9428E13CCF6C96BFAD6C97DA
:10FCE000B11125C0F401808585958595859585950B
:10FCF00083FD2FCFD30119962D923D924D925C92A8
:10FD00001C9727CF19821A821B821C828A818F70CE
:10FD10008A831D821E821F82188688E0FE0131962A
:10FD20001CCF6C96FFAD6C97FF2309F412CFB12C5A
:10FD3000A12CD12CC12C2A96EFAC2A972B96FFAC84
:10FD40002B972C960FAD2C972D961FAD2D972E9699
:10FD50002FAD2E972F963FAD2F9760964FAD6097A2
:10FD600061965FAD61976FEFC4010E9428E1611455
:10FD7000710409F0B7CFEDCE2F923F924F925F9270
:10FD80006F927F928F929F92AF92BF92CF92DF92AB
:10FD9000EF92FF920F931F93CF93DF93CDB7DEB710
:10FDA00068970FB6F894DEBF0FBECDBF6115710521
:10FDB00009F48EC05E8B498B9D8B8C8BFB018680FA
:10FDC00097808114910409F483C0F40180858295A1
:10FDD000807F8595859585958595823031F0853034
:10FDE00031F1F40182809380ECCF6184728441E030
:10FDF00050E069897E89C3010E947E64882389F36B
:10FE0000B12CA12CCC24C39473018301298950E027
:10FE100040E0B3018C899D890E94667829873A87E2
:10FE20004B875C876D877E878F87988BDACFC4017D
:10FE30000E9485FA8230A9F660E0C4010E94F3F9BD
:10FE4000FC01C184D284E384F48461E0C4010E9493
:10FE5000F3F9FC012184328443845484388E2F8A40
:10FE6000DB8ACA8AA1014C195D094F5F5F4F69891E
:10FE70007E89C6010E947E64882309F4B2CF8EE693
:10FE800092E10F94BA12712C612C6A897B89660DFC
:10FE9000771D8F89988D861797070CF4A2CFB12C08
:10FEA000A12CCC24C39471010A891B892989A3013F
:10FEB0008C899D890E94667829833A834B835C8371
:10FEC0006D837E838F8398879FEF691A790ADDCFD0
:10FED00068960FB6F894DEBF0FBECDBFDF91CF910D
:10FEE0001F910F91FF90EF90DF90CF90BF90AF9058
:10FEF0009F908F907F906F905F904F903F902F904A
:10FF000008950895089508958F929F92AF92BF9299
:10FF1000CF92DF92EF92FF920F931F93CF93DF93D5
:10FF200000D000D0CDB7DEB72091660C3091670CC1
:10FF3000232B09F4CCC02091580C2111C8C04C01CE
:10FF40008091580C8F5F8093580C8091880C8F5F44
:10FF50008093880C0F94B4069B01AC016091540C03
:10FF60007091550C8091560C9091570CA12CB12C8E
:10FF700065011BE0E12EF12C00E010E00E9452D35D
:10FF8000882309F452C0E091660CF091670C068159
:10FF9000178101151105B9F1F80180858F70863040
:10FFA00071F565EB76E0C8010E9441F90097D1F048
:10FFB000FC0120852F702530A9F4E680F780E1143C
:10FFC000F104E9F0FA82E982B801CE0101960E94BB
:10FFD0005937B401CE0101960E946858F701E280BA
:10FFE000F380EDCF1A83098370E060E0CE010196C3
:10FFF0000E945937B401CE0101960E946858F80159
:020000021000EC
:1000000002811381C6CFF3E08F16910451F00F9453
:10001000B4066093540C7093550C8093560C9093D7
:10002000570C1092AD121092AE1283E08816910414
:1000300009F443C00F94B4069B01AC016091500CCD
:100040007091510C8091520C9091530CA12CB12CB9
:10005000650118E8E12E13E1F12E00E010E00E94A6
:1000600052D3882351F1E091660CF091670C068120
:10007000178101151105B9F0F80180858F70863060
:1000800071F41A83098370E060E0CE0101960E944A
:10009000593761E070E0CE0101960E946858F8017E
:1000A00002811381E6CF0F94B4066093500C7093D5
:1000B000510C8093520C9093530C8091880C81507A
:1000C0008093880C8091580C81508093580C269610
:1000D0000FB6F894DEBF0FBECDBFDF91CF911F9159
:1000E0000F91FF90EF90DF90CF90BF90AF909F90D7
:1000F0008F900895A89583E090E00C94847F809180
:10010000870C8F5F8093870CA89583E090E00E9416
:10011000847F0E9416BC8091870C81508093870C4D
:10012000089565E87DE18DEB91E10F94061562E796
:100130007DE18DEB91E10F94061564E67DE18DEB99
:1001400091E10F9406156CE57DE18DEB91E10F9443
:1001500006158DEB91E10F94BA126CE47DE18DEB05
:1001600091E10F94061560E47DE18DEB91E10F9430
:10017000061563E37DE18DEB91E10F9406156EE1C9
:100180007DE18DEB91E10F9406156FE07DE18DEB44
:1001900091E10F94061567E07DE18DEB91E10F94FD
:1001A000061566EF7CE18DEB91E10F94061560ED8D
:1001B0007CE18DEB91E10F94061563EC7CE18DEB16
:1001C00091E10F94061569EB7CE18DEB91E10F94C1
:1001D00006156AEA7CE18DEB91E10F94061562EA5F
:1001E0007CE18DEB91E10F94061566E97CE18DEBE6
:1001F00091E10F9406156CE77CE18DEB91E10F9492
:1002000006156DE57CE18DEB91E10F94061568E430
:100210007CE18DEB91E10F94061560E37CE18DEBC1
:1002200091E10F94061562E27CE18DEB91E10F9470
:10023000061566E17CE18DEB91E10F9406156EE009
:100240007CE18DEB91E10F94061563E07CE18DEB91
:1002500091E10F94061566EF7BE18DEB91E10F9430
:1002600006156EEE7BE18DEB91E10F94061563EEC2
:100270007BE18DEB91E10F94061564ED7BE18DEB55
:1002800091E10F9406156BEC7BE18DEB91E10F94FE
:1002900006156DEB7BE18DEB91E10F9406156FEA8E
:1002A0007BE18DEB91E10F9406158DEB91E10D94BF
:1002B000BA120F931F93CF93DF9300D000D0CDB726
:1002C000DEB70E94918064ED74E18DEB91E10F94B3
:1002D0000615CE0101960E948EFFCE0101960E9466
:1002E000C1D90DED15E01A8309838091BD0F90915E
:1002F000BE0FA091BF0FB091C00F8B839C83AD83C5
:10030000BE83CE0101960E94C1D91A8309831B8244
:100310001C821D821E8280E590E00E948BFF44E0DB
:1003200050E0BE016D5F7F4F81E090E00E94DEBF34
:100330000E94D5C0CE0101960E94C1D91A830983BB
:100340001B821C821D821E8280E590E00E948BFF32
:1003500044E050E0BE016D5F7F4F85E090E00E9479
:10036000DEBF0E94D5C0CE0101960E94C1D96AEFBE
:1003700074E18DEB91E10F94061588EC90E02696E0
:100380000FB6F894DEBF0FBECDBFDF91CF911F91A6
:100390000F910895FF920F931F93CF93DF9300D097
:1003A00000D0CDB7DEB78C01BC01CE0101960F9411
:1003B000CC0FBE016F5F7F4F8EE692E10F94F81471
:1003C0008EE692E10F94BA12CE0101960F94C40FFB
:1003D0001A8219821C821B821E821D826EE87AE1BB
:1003E000CE0101960F94670FF801248135818D812C
:1003F0009E81F12C2817390738F0BE016F5F7F4FBF
:10040000C8010F940B01F82ECE0101960F94C40F72
:10041000FF2069F0B801CE0101960F94CC0FCE01F8
:1004200001960F942A15CE0101960F94C40F2696BB
:100430000FB6F894DEBF0FBECDBFDF91CF911F91F5
:100440000F91FF900895AF92BF92CF92DF92EF92FB
:10045000FF920F931F93CF93DF93CDB7DEB76D97C6
:100460000FB6F894DEBF0FBECDBF0F94B4069B014C
:10047000AC016091610C7091620C8091630C909161
:10048000640CA12CB12C650118EEE12E13E0F12EC5
:1004900000E010E00E9452D3F82E882351F00F9410
:1004A000B4066093610C7093620C8093630C90931C
:1004B000640C8091880C8F5F8093880CE091F90D1B
:1004C000F091FA0D0681178194E0C92ED12CF1101C
:1004D00003C082E0C82ED12CA090F90DB090FA0D87
:1004E000A114B10429F10115110511F1F80180855C
:1004F0008F708530A9F7C8010E9485FA823080F399
:10050000B801CE0101960E94D632CE0101960E941A
:10051000CF26882329F0B601CE0101960E943652DB
:10052000F80102811381CE0101960E947831D4CF67
:100530008091880C81508093880C8091F70D909168
:10054000F80D0597D9F1FF20C9F110E06091DC0B9F
:100550007091DD0B6115710589F111112FC0FB013F
:1005600080858F70853091F4CE0101960E94D6323D
:1005700061E070E0CE0101960E94365211E0892BB5
:1005800009F410E0CE0101960E947831E091DC0B75
:10059000F091DD0B309791F0828193819093DD0B88
:1005A0008093DC0B892B91F6E091F90DF091FA0D17
:1005B000868197819093DD0B8093DC0B6D960FB64F
:1005C000F894DEBF0FBECDBFDF91CF911F910F9189
:1005D000FF90EF90DF90CF90BF90AF9008952F9253
:1005E0003F924F925F926F927F928F929F92AF92C3
:1005F000BF92CF92DF92EF92FF920F931F93CF9310
:10060000DF93CDB7DEB7C955D1090FB6F894DEBF79
:100610000FBECDBF0F94B4069B01AC0160915D0C81
:1006200070915E0C80915F0C9091600CA12CB12CAC
:10063000650110E3E12E15E7F12E00E010E00E94C5
:1006400052D3882309F42EC2E091F90DF091FA0DEE
:10065000309709F427C28091880C8F5F8093880CB3
:100660002680378010E02114310409F43AC1F101E9
:1006700080858F708530F9F460E0C1010E94F3F944
:10068000FC0181859285A385B4850597A105B105F7
:1006900091F4B101CE0101960E94D632CE010196AD
:1006A0000E94CF2666968FAF6697811108C0CE0153
:1006B00001960E947831F10122803380D4CF2596B3
:1006C0001CAE1DAE1EAE1FAE259729961CAE1DAEEC
:1006D0001EAE1FAE299740E052E0BE016F5F7F4F14
:1006E000CE018F5B9F4F0E94102ECE0101960E947B
:1006F00084276B017C0169966FAF69976A96DFAEBC
:100700006A9770E060E0CE0101960E94A0274C013C
:10071000CE018F5B9F4F0E942A1F65966CAF7DAF05
:100720008EAF9FAF6597CE0101960E94032E182FC2
:10073000B601DD0C880B990B0F942B3620E030E0CE
:1007400048EC52E40F9484382B013C01CE01019611
:100750000E94015168969FAF8EAF689761E37EE17A
:100760008EE692E10F94061565964CAD5DAD6EADCB
:100770007FAD65978EE692E10F94DE126BE27EE12B
:100780008EE692E10F940615B301A2018EE692E186
:100790000F94DE1265E27EE18EE692E10F9406157B
:1007A000612F70E04AE050E08EE692E10F94F7137B
:1007B000E114F10409F48EC088E00E94B4D39B01D7
:1007C000AC0144275527B70190E080E0AA24AA9401
:1007D000BA2CC12CD12C17E2E12E19E0F12E00E049
:1007E00010E00E9452D3882371F1F1016081718180
:1007F00087EC91E10F94101465E17EE187EC91E1C3
:100800000F940615F101608171818AE299E00F94DD
:100810006C0790E080E0BC0169964FAD69976A96DD
:100820005FAD6A97CE0101960E94242762E070E0D6
:10083000C4010E940370CE0101960E947831669631
:100840001FAD669738CF20E030E048E152E4C301A5
:10085000B2010F942C3918163CF4F10160817181BA
:1008600084EA96E00F946C0768968EAD9FAD68970A
:10087000892B19F461E070E0DBCF20E030E040E844
:100880005FE365966CAD7DAD8EAD9FAD65970F94C2
:1008900017389B01AC01C301B2010F94243670E0FC
:1008A00060E087FDC5CFA301920165966CAD7DAD7B
:1008B0008EAD9FAD65970F9424361816DCF666E072
:1008C0007EE18EE692E10F9406158EE692E10F949A
:1008D000BA12B1CF6CEF7DE18EE692E10F9406156E
:1008E000AACF8091880C81508093880C0F94B40615
:1008F00060935D0C70935E0C80935F0C9093600C22
:100900000E94AEDA2B013C010F94B4066B017C010E
:100910000E945FF9882309F489C08091870C8111B6
:1009200085C030E020E041E050E060E4CE01019677
:100930000E942DD94FE350E065ED7DE1CE01019697
:100940000F94483063EF79E0CE0101960F943C3C60
:100950004FE350E06CEC7DE1CE0101960F944830FE
:100960002AE0AE014F5B5F4FC301B2010F94D33059
:10097000BE016F5B7F4FCE0101960F94510730E0AF
:1009800020E041E050E060E4CE0101960E942DD9C4
:100990004FE350E065ED7DE1CE0101960F944830C4
:1009A00063EF79E0CE0101960F943C3C4FE350E0B9
:1009B00065EC7DE1CE0101960F944830C701B60188
:1009C00028EE33E040E050E00F946E37CA01B901E1
:1009D0002AE0AE014F5B5F4F0F94D330BE016F5BD7
:1009E0007F4FCE0101960F94510730E020E041E0A7
:1009F00050E060E4CE0101960E942DD94FE350E013
:100A00006EEB7DE1CE0101960F9448304FE050E04F
:100A100068EB7DE1CE018F5B9F4F0F946630BE0186
:100A20006F5B7F4FCE0101960F945107112309F49C
:100A300053C066EF7DE18EE692E10F9406150E94A9
:100A4000AEDAAB01BC012AE030E08EE692E10F9411
:100A5000B8126EEE7DE18EE692E10F94061560917C
:100A6000880C062E000C770B4AE050E08EE692E1EF
:100A70000F94F7136CED7DE18EE692E10F9406156D
:100A80004091590C50915A0C60915B0C70915C0C28
:100A90002AE030E08EE692E10F94B8128EE692E101
:100AA0000F94BA12C75ADF4F0FB6F894DEBF0FBECD
:100AB000CDBFDF91CF911F910F91FF90EF90DF900D
:100AC000CF90BF90AF909F908F907F906F905F90EE
:100AD0004F903F902F9008956CEE7DE18EE692E16D
:100AE0000F9406150E94AEDAAB01BC012AE030E09B
:100AF0008EE692E10F94B81264EE7DE1ACCF4F9296
:100B00005F926F927F92AF92BF92CF92DF92EF92FD
:100B1000FF920F931F93CF93DF93CDB7DEB76D97FF
:100B20000FB6F894DEBF0FBECDBF6FEB7EE18EE651
:100B300092E10F9406158EE692E10F94BA120F948B
:100B4000B4062B013C018091880C882381F10F941D
:100B5000B4069B01AC01A12CB12C650110E1E12E82
:100B600017E2F12E00E010E0C301B2010E9452D35F
:100B700081111DC00E9416BC8091FD0D81116DC0B8
:100B80000E94D5378091F70D9091F80D059741F0AF
:100B90008091F90D9091FA0D892B11F00E9423821A
:100BA0000E94EF8282E090E00E94847FCCCF80910F
:100BB000880CFF24F394882359F06CE97EE187ECDC
:100BC00091E10F94061587EC91E10F94BA12F12C84
:100BD00066E87EE18EE692E10F9406158EE692E1DC
:100BE0000F94BA128091690C8F5F8093690CE09129
:100BF000F90DF091FA0D3097D1F1068117810115A9
:100C00001105A9F1D80118968C918F708530B9F72C
:100C1000C8010E9485FA882391F3F80160817181EF
:100C2000CE0101960E94EC30CE0101960E94CF26A3
:100C3000882359F08A859B85009739F0DC01ED9176
:100C4000FC910284F385E02D1995CE0101960E9456
:100C50007831F80102811381D2CF8091FB0D909100
:100C6000FC0D892B09F48CCF0E9463DC89CF109294
:100C7000DD0B1092DC0B6EE77EE18EE692E10F94C5
:100C800006158EE692E10F94BA1264E670E080E0F9
:100C900090E00F9443041092820C1092680C66E668
:100CA0007EE18EE692E10F9406150E94AEDAAB016A
:100CB000BC012AE030E08EE692E10F94B8128091F8
:100CC000DA0B9091DB0B009711F00E94A4FE1092BA
:100CD000DB0B1092DA0B1092670C1092660C1092DC
:100CE000FA0D1092F90D1092860C1092850C10924C
:100CF000D90B1092D80B1092840C1092830C109286
:100D0000D70B1092D60B1092FC0D1092FB0D109287
:100D1000750C1092740C61E67EE18EE692E10F9400
:100D200006150E94AEDAAB01BC012AE030E08EE687
:100D300092E10F94B8128EE692E10F94BA121092DB
:100D4000650C8091690C81508093690C8F2D6D9694
:100D50000FB6F894DEBF0FBECDBFDF91CF911F91CC
:100D60000F91FF90EF90DF90CF90BF90AF907F906A
:100D70006F905F904F9008955F926F927F928F92E5
:100D80009F92AF92BF92CF92DF92EF92FF920F931A
:100D90001F93CF93DF93CDB7DEB7A3970FB6F89429
:100DA000DEBF0FBECDBF8091DA0B9091DB0B892B9C
:100DB00009F4B8C58091880C8111B4C58091880C64
:100DC0008F5F8093880C6BE079E18DEB91E10F945C
:100DD00006158DEB91E10F94BA120091DA0B109188
:100DE000DB0B66E379E0C8010E9441F99093FA0DAC
:100DF0008093F90D6CE379E0C8010E9441F990936A
:100E0000860C8093850C63ED76E0C8010E9441F961
:100E10009093670C8093660C63E479E0C8010E94AC
:100E200041F99093D90B8093D80B0E94581A68E42B
:100E300079E08091DA0B9091DB0B0E9441F990935D
:100E4000D70B8093D60B009709F4B3C00E9485FAA4
:100E5000082F10E00115110509F4ABC0000F111F98
:100E6000000F111F8091D40B9091D50B892B09F0A5
:100E70008FC0C8010F94F62D9093D50B8093D40B9F
:100E80001092970C1092960C10924F0C10924E0CE0
:100E90001092950C1092990C1092980C78010130D8
:100EA00082E018071CF0E12C82E0F82EC7010196C1
:100EB0000F94F62D90939B0C80939A0C9093940C26
:100EC0008093930C8E0D9F1D90938E0C80938D0CB0
:100ED0000F94B40660938F0C7093900C8093910CD8
:100EE0009093920C90E080E0E0919A0CF0919B0C32
:100EF000E80FF91F10820196E816F906ACF782E0B8
:100F000090E09093970C8093960C80914E0C90916A
:100F10004F0C009741F061E00F94FE0160E080917A
:100F20004E0C0F94D00180E98093C9001092C80044
:100F30001092CD0083E08093CC008EE08093CA00B5
:100F4000F0922F02E0922E0220919A0C30919B0C8D
:100F500080912E0290912F02820F931F90938E0CFE
:100F600080938D0C232B09F462C06BE978E18EE647
:100F700092E10F9406154AE050E0B8018EE692E146
:100F80000F94FE1382E999E190938C0C80938B0C63
:100F900061EF78E18DEB91E10F9406154AE050E0A6
:100FA000B8018DEB91E10F94F7138DEB91E10F9464
:100FB000BA126EE479E08091DA0B9091DB0B0E941B
:100FC00041F98C01009709F472C00E9485FA8823C8
:100FD00009F46DC06FEF680FC8010E94F3F9DC01DE
:100FE0001996ED90FC909091890C992359F080917D
:100FF00070008E7F809370001092890C10922A02EC
:101000001092290282E18093280291110E9404CE5D
:10101000C7010E942CCE01E010E0E016F10674F04A
:1010200060E0C8010E9460CE0F5F1F4FF6CF64E8FA
:1010300078E18EE692E10F94DA19A4CF66E778E1C1
:101040008EE692E10F9406150E94AEDAAB01BC0168
:101050002AE030E08EE692E10F94B8128EE692E13B
:101060000F94BA1265ED78E18DEB91E10F940615BE
:101070004AE050E0B7018DEB91E10F94F7138DEB4F
:1010800091E10F94BA126FEC78E18EE692E10F9441
:1010900006150E94AEDAAB01BC012AE030E08EE614
:1010A00092E10F94B8128EE692E10F94BA12009179
:1010B000DA0B1091DB0B62E579E0C8010E9441F97F
:1010C0009093750C8093740C69E777E0C8010E94D7
:1010D00041F99093FC0D8093FB0D009709F4BDC17D
:1010E0002091FD0D2111B9C1FC01E680F7808091AE
:1010F000F50D9091F60D892B51F081E08093FD0D57
:101100006FEB78E18DEB91E10F94061545C065E535
:1011100078E18EE692E10F9406158EE692E10F9447
:10112000BA126FE478E18EE692E10F9406150E9400
:10113000AEDAAB01BC012AE030E08EE692E10F941A
:10114000B8128EE692E10F94BA128FE090E00F94FD
:10115000F62D8C0188E1D80111968C931197129687
:101160001C9212971C921E961C921E921D970E9412
:101170008DFE1093F60D0093F50D012B09F0CBC0F9
:101180006DE378E187EC91E10F94061587EC91E12E
:101190000F94BA121092FD0D1092810C1092800CD7
:1011A000CC24C394D12CE114F10409F456C18091EC
:1011B000FD0D882309F451C1F70180858F708630B9
:1011C00009F0A5C000811181CE0101965C014801A2
:1011D00090E1890E911C3501D8018C910E9429DC87
:1011E000582EF80181810E9429DC5294A0EF5A22E6
:1011F000582AD5015D925D010E5F1F4F8016910642
:1012000059F76AEB77E18DEB91E10F940615609148
:10121000800C7091810C4AE050E08DEB91E10F94CD
:10122000F71363EB77E18DEB91E10F940615809155
:10123000800C9091810CF3E0880F991FFA95E1F7EB
:1012400020917E0C30917F0C820F931F0E9419FF1A
:101250008DEB91E10F94BA128091800C9091810CEA
:10126000843191050CF053C0A0917E0CB0917F0C9D
:1012700048E09C01E3E0220F331FEA95E1F72A0FD3
:101280003B1F415008F443C0F901E40FF11D5081A8
:101290005523B9F3880F991F20917A0C30917B0C5C
:1012A000820F931FFC01D182C0828091800C9091AB
:1012B000810C33E0880F991F3A95E1F7A80FB91F09
:1012C00088E0F30101900D928A95E1F78091800CFE
:1012D0009091810C43E0880F991F4A95E1F7E091C6
:1012E0007E0CF0917F0CE80FF91F8081883231F479
:1012F0008091F50D9091F60D0E94D1D18091800CD6
:101300009091810C01969093810C8093800CF70151
:10131000E280F38048CF80EA90E00F94F62D90931E
:101320007F0C80937E0C61E378E18EE692E10F946E
:1013300006150E94AEDAAB01BC012AE030E08EE671
:1013400092E10F94B8128EE692E10F94BA1288E2FD
:1013500090E00F94F62D90937B0C80937A0C64E2CE
:1013600078E18EE692E10F9406150E94AEDAAB01A9
:10137000BC012AE030E08EE692E10F94B8128EE6CE
:1013800092E10F94BA1280917E0C90917F0C892B80
:1013900031F080917A0C90917B0C892B89F46CE070
:1013A00078E187EC91E10F9406150E94AEDAAB016B
:1013B000BC012AE030E087EC91E10F94B812E6CE50
:1013C0008FE897E790937D0C80937C0C0E948DFEB4
:1013D0008091F50D9091F60D0E948ECE83EC9FE0EA
:1013E0000E943ED0811132C069EF77E18EE692E132
:1013F0000F94DA190091F50D1091F60DC8010E94B5
:101400008ECE40E060EFC8010E94DDD10E9415FF42
:10141000E091F50DF091F60D11E0108369ED77E1A3
:101420008EE692E10F94DA198091F50D9091F60D08
:101430000E9490D1882309F460CE6DEC77E18EE6AE
:1014400092E10F94DA191093FD0D5ACE6FEB77E10C
:101450008EE692E10F94DA199DCE1092DD0B109278
:10146000DC0BE091F90DF091FA0D309709F400C111
:10147000C680D7800091F90D1091FA0D0115110564
:1014800009F4EFC0C114D10409F4EBC0D6011896D9
:101490008C918F70853091F7C6010E9485FA823059
:1014A00068F3B601CE0101960E94D632CE010196B4
:1014B0000E94CF26882309F468C08A859B850097FF
:1014C00069F570E060E0CE0101960E94A0278C01D2
:1014D000912C812C97FF06C0119501951109882444
:1014E0008394912CCE0101960E94032EE82EF12CBC
:1014F0008985853009F452C0863009F046C0B02E87
:1015000061E0802F0F94FE0161E0892809F483C017
:10151000EA94EF2809F083C060E081C0DC01ED911E
:10152000FC910484F585E02D1995892B49F08A8575
:101530009B85DC01ED91FC910284F385E02D1995EA
:101540008A859B85DC01ED91FC910680F781E02D79
:101550001995892BD1F0CE0101960E94032E882384
:1015600041F040E051E060E070E0CE0101960E9461
:10157000BE298D819E81892B41F040E052E060E0E0
:1015800070E0CE0101960E94BE29D6011296CD9040
:10159000DC90CE0101960E9478316CCFEF2829F4BF
:1015A00062E0CE0101960E94202D40E051E060E013
:1015B00070E0CE0101960E94BE298D819E81892B0B
:1015C00041F040E052E060E070E0CE0101960E9400
:1015D000BE2961E0802F0F94FE0160E0802F0F9400
:1015E000D00167EB78E18EE692E10F9406154AE0B0
:1015F00050E0B8018EE692E10F94F71362EB78E1C8
:101600008EE692E10F94061560EB78E18EE692E1AA
:101610000F940615BACFEA94EF2809F07DCFE62E95
:10162000F12C8B2D0F94D0016BEA78E18EE692E1DC
:101630000F9406154AE050E0B8018EE692E10F944F
:10164000F71369EA78E18EE692E10F9406154AE015
:1016500050E0B7018EE692E10F94F71367EA78E164
:10166000D5CFF801868197819093DD0B8093DC0BB9
:101670008EE692E10F94BA12E091660CF091670C3D
:10168000309709F4ADC08091880C8F5F8093880CEF
:10169000068117815E01FEE1AF0EB11C5EE9652E89
:1016A00054E0752E66EB862E64E0962E011511052A
:1016B00009F491C0D80118968C918F70863009F08A
:1016C00068C01F8F0E8F70E060E0C5010E9459371F
:1016D0008AA19BA1892B09F45CC08091DA0B9091BF
:1016E000DB0B892B09F455C0EE8CFF8CF70180854C
:1016F0008F70863099F565EB76E0C7010E9441F95D
:101700000097F1F0DC0118962C9118972F70253076
:10171000B9F41696CD90DC90C114D104F9F0DA82B8
:10172000C982B701CE0101960E945937ED81FE8131
:101730001082118212821382F601C280D380ECCF14
:10174000FA82E98270E060E0CE0101960E9459378A
:1017500062E070E0CE0101960E946858EAA1FBA108
:10176000108211821282138288A1843068F462E0B0
:10177000823008F060E089A10F94FE01EAA1FBA18C
:101780008181807F818305C08630E1F038F4853027
:1017900081F0D80112960D911C9188CF803439F0D8
:1017A00060E08234B1F789A10F94FE01F2CF62E0CC
:1017B000FACFBC82AB829A828982CE0101960E94C6
:1017C0003D74E7CFBC82AB827A826982CE010196FA
:1017D0000E948873DECF8091880C81508093880CA2
:1017E00066EA77E18DEB91E10F9406156EE977E1FA
:1017F0008DEB91E10F94061581E02091F90D309168
:10180000FA0D232B09F480E00E94216465E977E159
:101810008DEB91E10F94061581E02091660C3091DB
:10182000670C232B09F480E00E94216466E877E1CD
:101830008DEB91E10F9406156BE777E18DEB91E16C
:101840000F94061581E02091740C3091750C232BB8
:1018500009F480E00E94216464E777E18DEB91E177
:101860000F94061581E02091D80B3091D90B232BD2
:1018700009F480E00E9421646BE677E18DEB91E151
:101880000F94061581E02091FB0D3091FC0D232B68
:1018900009F480E00E94216462E677E18DEB91E13A
:1018A0000F9406158091820C0E9421648DEB91E1CA
:1018B0000F94BA126DE577E18DEB91E10F94061567
:1018C0000E94AEDAAB01BC012AE030E08DEB91E181
:1018D0000F94B8128DEB91E10F94BA1281E08093CE
:1018E000680C8CE891E10E945DC5882351F08CE87A
:1018F00091E10E9415CC84E090E09093F80D8093E4
:10190000F70D8091F70D9091F80D079731F484E071
:1019100090E09093F80D8093F70D8091880C8150A2
:101920008093880CA3960FB6F894DEBF0FBECDBF90
:10193000DF91CF911F910F91FF90EF90DF90CF90AB
:10194000BF90AF909F908F907F906F905F90089521
:101950000F931F93CF93DF93CDB7DEB760970FB68A
:10196000F894DEBF0FBECDBF8091880C811172C08C
:1019700060E779E18DEB91E10F9406158DEB91E134
:101980000F94BA121092B9111092B81180E090E140
:101990009093B4118093B31184E890E09093BB11BD
:1019A0008093BA1181E08093B51182E78093BC11D6
:1019B00087EA91E10E94C6188B37910509F0E1C0D2
:1019C00068E579E18EE692E10F9406158EE692E1E4
:1019D0000F94BA121C821B8284EE94E09A8389834E
:1019E00087EA91E19E838D838FEF9FEF98878F83A6
:1019F0008091DA0B9091DB0B892B11F00E947F858F
:101A0000CE0101960E946DFF9093DB0B8093DA0B61
:101A100087EA91E10E94E9168091DA0B9091DB0B45
:101A2000892BD9F46CE479E187EC91E10F940615E8
:101A300087EC91E10F94BA1262E67AE0CE01099642
:101A40000F94D50FCE0109960F942A15CE01099651
:101A50000F94C40F90E080E014C069E379E18DEB4E
:101A600091E10F9406158DEB91E10F94BA120E944B
:101A7000BC868091991190919A11892B69F481E02B
:101A800090E060960FB6F894DEBF0FBECDBFDF9139
:101A9000CF911F910F9108950E9495FA882379F3B1
:101AA000A0919911B0919A1152961C921E92519741
:101AB00054961C921E92539784E890E01D969C9336
:101AC0008E931C971E961C921E9782E755968C93B8
:101AD0005597ED91FC9111970088F189E02D60E612
:101AE00070E0CD0119950091991110919A1162E65B
:101AF0007AE0CE0109960F94D50FC8010F94931187
:101B00001816190664F48F87188A41E050E0BE0168
:101B1000615F7F4FCE0109960F94F00EEECFBE01AC
:101B2000675F7F4F8BE991E10F941C0FCE010996FF
:101B30000F94C40F8091991190919A11DC01ED914D
:101B4000FC910488F589E02D19956BE179E18EE629
:101B500092E10F9406156BE971E1CE0109960F949D
:101B6000CC0FBE01675F7F4F8EE692E10F94F814B1
:101B70008EE692E10F94BA12CE0109960F94C40F2B
:101B80007ECF87EA91E10E94FA15892BA1F087EABE
:101B900091E10E94241662E67AE0CE0101960F944C
:101BA000D50FCE0101960F942A15CE0101960F9400
:101BB000C40F0F94351687EA91E10E94E91668E296
:101BC00079E18DEB91E10F9406158DEB91E10F9486
:101BD000BA1240CF0E94A88C892B49F486EF9FEF60
:101BE0009093F80D8093F70D84EF91E0089588ECC1
:101BF00090E008954F925F926F927F928F929F92A2
:101C0000AF92BF92CF92DF92EF92FF920F931F930A
